:020000040800F2
:100000000000011075C30608E91F00080D1C020856
:1000100015C4060815C4060815C40608000000002B
:10002000000000000000000000000000593B000834
:100030005D3B000800000000613B000825F400085B
:1000400015C4060815C4060815C4060815C4060814
:1000500015C4060815C4060839A600083DA6000800
:1000600015C4060841A6000845A600080D2800088A
:100070002128000835280008492800085D280008C4
:10008000712800088528000815C4060815C406084C
:1000900015C4060815C4060815C4060849A60008B4
:1000A000B9260008E126000809270008A52600084F
:1000B00031270008452700085927000815C40608FD
:1000C00015C4060815C4060815C4060815C4060894
:1000D00015C40608512100085D21000869210008A7
:1000E0004DA6000815C40608653B000895270008C2
:1000F000BD270008E5270008812700089928000887
:1001000015C4060815C406086D27000815C406089E
:10011000752100088121000815C4060815C40608C9
:10012000AD280008C1280008D5280008E9280008E3
:10013000FD28000815C4060815C4060815C40608DD
:1001400015C4060815C4060815C40608B93B0008FE
:100150000D2900081D2900082D2900088D210008FF
:1001600015C4060815C4060815C4060815C40608F3
:1001700015C4060815C4060815C4060815C40608E3
:0801800015C4060815C40608A9
:10019000D0E907239A422FBFD01AC0688018C01A2E
:1001A000704700BFD0E9092300699A4238BF12188E
:1001B000D31A0138C01A7047D0E90902101AB0FAF0
:1001C00080F04009704700BF0246036A4069D16869
:1001D000C05C01338B4228BF00231362704700BF0D
:1001E000436A8269D154436A0169426B01338B428D
:1001F00028BF00234362D36843F08003D360704775
:10020000436B188810F0100002D01A889B880120D8
:10021000704700BF436B99891A88890610B5044658
:100220000AD592B2900607D5E26A002A29D09888AA
:10023000216B80B29047636B99891A88090692B244
:100240000FD510060DD5D4E909128A4214D0A16940
:100250002069895C99800132B2FBF0F100FB112228
:10026000A262998A1A88C90592B204D5D20744BFFE
:100270004FF6F7721A8010BDDA6822F08002DA6059
:10028000EFE79B88E2696169DBB28B54E269E16860
:10029000636B0132B2FBF1F001FB1022E261CBE7AC
:1002A000036942681F2B10B40AD95468A3F1200CCB
:1002B000202101FA0CF1214207D15DF8044B70476F
:1002C0001468202199402142F7D081690024C86830
:1002D0000C7480684C68016821F00101016020689D
:1002E00094F805C00C4C818934F81C4089B221EA8D
:1002F00004011F2B818107D9A3F1200120238B400A
:100300005DF8044BD3607047202101FA03F35DF8D8
:10031000044B9360704700BFF820070882B00922A1
:10032000274B8DF80720DA68D00319D4DA68D10694
:1003300040D4DA68D20541D4DA6812F0E00F3BD13C
:10034000DB6813F0020F14BF082309238DF8073070
:100350009DF80730012B0AD09DF8070002B07047C6
:1003600001238DF807309DF80730012BF4D1144A92
:1003700012E0D368DB0519D4D36813F0E00F17D16E
:10038000D36813F0020F14BF082309238DF8073038
:100390009DF80730012BDFD1D168C8034FF001036E
:1003A000F4D4D368D906E4D50623EFE70223EDE7BA
:1003B0000723EBE70623D4E70723D2E70223D0E79E
:1003C000003C0240704700BF704700BF01207047EB
:1003D000044BD3E90003984288BF03F50063181A61
:1003E000704700BF98200020054AD2E900318B42B7
:1003F000FDD0D1180133C3F30A03087A13607047A4
:1004000098200020064BD3F8080800B97047D3F8AD
:100410000808A0F10500B0FA80F04009704700BF5D
:1004200098200020012380F849307047064BD3F80C
:100430000C08D3F81028431E90428CBF00200120E6
:100440009B1A03EBC02070479820002010B5D0F80D
:10045000E83504461B699847032384F812310020CD
:1004600010BD00BF08B5042290F81211D0F8E8358D
:1004700080F8131180F81221DB689847002008BD2E
:1004800008B5D0F8E435DB6903B19847002008BD12
:1004900008B5D0F8E4351B6A9847002008BD00BFB6
:1004A00008B5D0F8E4355B6A9847002008BD00BF66
:1004B000037830B403B30446C0F1010C04EB0C0321
:1004C00014F8015FDBB2002DF8D101335B00DCB220
:1004D000138003230C704B7004785CB10223002559
:1004E0005A1CD2B2CC548D5410F8014F0233DBB2F7
:1004F000002CF5D130BC704702242346E8E700BF4A
:1005000010B5074C2068FF2808D00649D1F81428F8
:1005100001F6180100F080F8FF232360002010BDD1
:100520000000002098200020432301480B807047E2
:1005300004000020122301480B807047480000206F
:10054000042301480B8070475C00002008B5044B71
:1005500004480A461946FFF7ABFF084608BD00BF2E
:10056000B8280020A4BE070808B5044B04480A4672
:100570001946FFF79DFF084608BD00BFB8280020B8
:10058000B0BE070808B5044B04480A461946FFF7F1
:100590008FFF084608BD00BFB8280020B8BE070876
:1005A00008B5044B04480A461946FFF781FF084680
:1005B00008BD00BFB8280020C4BE070808B5044B1A
:1005C00004480A461946FFF773FF084608BD00BFF6
:1005D000B8280020D0BE0708704700BF704700BF92
:1005E000704700BF704700BF704700BF704700BF33
:1005F000044B00200522C3F80828C3F82009C3F8DB
:100600002409704798200020024B0020C3F80808F6
:10061000704700BF98200020212838B50C4605D02F
:1006200022282DD0202813D0002038BD0029FBD04F
:10063000072AF9D1194BD3F8280993F82C1993F804
:100640002D2993F82E39206021716271A371EBE797
:100650000029E9D0072AE7D1104DD5F8243913B184
:10066000096800209847206821796279A379C5F844
:10067000280985F82C1985F82D2985F82E39D3E716
:100680000029D1D0022ACFD1044BD3F82039002B36
:10069000CAD0098800209847C6E700BF98200020EC
:1006A00010B4144CD4E900239A4286BF03F5006CC1
:1006B000ACEB02029A1A0A44B2F5006F13D8B1B13A
:1006C00001444A1E013810F801CFE118824203F1BB
:1006D000010381F808C0C3F30A03F4D1636000206A
:1006E0005DF8044B704702205DF8044B70470846E4
:1006F000F6E700BF9820002010B58121044669F07C
:10070000EBFF2046012169F0E7FF2046822169F0D6
:10071000E3FFFFF779FF002010BD00BFC169026948
:1007200010B4002340F20114A0F844410B60D169D9
:10073000846D21F002014FF0010CD161A0F89CC33F
:100740002360D169044821F4003180F82F395DF825
:10075000044BD1611846704798200020202301489F
:100760000B80704760000020122301480B80704707
:1007700080000020042301480B8070479400002073
:100780000A4608B5054920B90548FFF791FE034818
:1007900008BD0448FFF78CFE004808BDC8290020AA
:1007A000E0BE0708F8BE070808B5044B04480A462F
:1007B0001946FFF77DFE084608BD00BFC829002086
:1007C00010BF07082048D0F8E837D0F8EC2730B53C
:1007D0009B184FF01A040C8001D11C4830BD1B4AF5
:1007E000D0F8EA174FF0000E10467546B3F1204FCF
:1007F0004FEA137C0CF130040EF1020E2ABF0CF10B
:10080000370C847080F802C0BEF1100FC5704FEA3B
:10081000031300F10200E9D100200446B1F1204F9A
:100820004FEA117303F1300C00F102002ABF373395
:1008300082F812C093740828D4744FEA011102F1AF
:100840000202EBD1014830BD00F0FF1F98000020EC
:1008500008B5044B04480A461946FFF729FE084626
:1008600008BD00BFC829002024BF070808B5044BF5
:1008700004480A461946FFF71BFE084608BD00BF9C
:10088000C829002030BF0708034BD3F8D82AB3F893
:10089000DC3A138300207047982000204FF400704A
:1008A000034B1060D3F8883C0B600020704700BFFA
:1008B00098200020002070470120704701207047D9
:1008C0000020704710B51C6994420DD396468A18D3
:1008D0008C469442996938BFA4EB0E0C7144624671
:1008E000BDE8104071F032B910BD00BF2DE9F041F4
:1008F000204E96F8B83C002BFBD1B9B3014400F16F
:10090000FF384F1ED6F81018D6F80C3818F8010F1B
:100910004A1CC2F30A029A4234BF002401249B1AE3
:10092000314403EBC423012B81F8BC0CC6F810281A
:100930001AD10EF0C3FD04460D460EF0BFFD031B99
:1009400061EB0501B3F57A7F71F10003F5D3D6F8B9
:100950000C38D6F8102893428CBF002101219B1A35
:1009600003EBC123012BE4D0B845CBD10020BDE877
:10097000F08100BF982000200A4B10B5D3F808483A
:1009800004B910BDD3F80838052BFAD1064C002A5B
:100990000846D4F8C4331146F3DDFFF7A7FFD4F8B7
:1009A000C43310BD982000209031002090F84820DA
:1009B000531C0244DBB280F8483082F8341090F8BF
:1009C00049200AB1132B03D9002280F8482003B92B
:1009D00070470A4AD2F808180029F9D0D2F8082836
:1009E000052AF5D110B5064C19463430D4F8C43375
:1009F000FFF77CFFD4F8C43310BD00BF982000205F
:100A00009031002090F848100023A0F8483001B938
:100A10007047094BD3F80828002AF9D0D3F80838D2
:100A2000052BF5D110B5054C3430D4F8C433FFF79D
:100A30005DFFD4F8C43310BD982000209031002011
:100A40002DE9F0475D4E1F4606EB80039C68002CA5
:100A500000F0AD8004F13E03A36104F59F73E361F0
:100A60004FF48073C4E90433283623686660054672
:100A7000E16094F83D00A363904609F01DFE8146B5
:100A800094F8440294F83CA0261D00284FD194F815
:100A9000450268BBD4F8403283BB390734D418F020
:100AA000020F60D118F0010F44D194F9472294F855
:100AB0004712D4F84832002A10DB41481B01841841
:100AC000DBB284F800335209012301F01F0103FA5D
:100AD00001F140F822103046BDE8F087394A01F0B4
:100AE0000F010A441B01DBB213763046BDE8F087E4
:100AF00067F01CFAD4F84032002BCED0324A116B8A
:100B00000B4339071363CAD50135EDB2B9F1000FB4
:100B1000CBD04FF4E163FA0689F80850A9F8063003
:100B200036D4BB0694F8462245D4322133E067F030
:100B3000FDF9ACE7504609F0BFFD0135EDB20028E4
:100B4000B3D04FF4C1620572C28094F846220221EC
:100B500009F0AAFF94F9472294F84712D4F84832D2
:100B6000002AAADABAE76B1CDBB2B9F1000F99D000
:100B700089F808304FF4A163A9F8063094F84622AA
:100B80004846022109F090FF18F0010F8DD0D1E7FF
:100B900094F846220221484609F086FF94F947223C
:100BA00094F84712D4F84832002A86DA96E72646A7
:100BB0003046BDE8F0871221EDE700BFF8200708B6
:100BC00000E100E0FCEC00E0003802402DE9F047D5
:100BD000038A8489A4B21C4082B045D081468846ED
:100BE0004FF0004501F14C0701F13406B4FA84F3EB
:100BF00025FA03F2D24391B2A9F8101014401B3B1E
:100C0000B8F1000F5DD0042B2CD8DFE803F050467C
:100C10003B300300D8F80C30D9F82CA033B19B68D6
:100C200023B11FFA8AF108F104009847D8F824305C
:100C300033B19B6823B11FFA8AF108F11C00984771
:100C4000D8F83C302BB19B681BB11FFA8AF13046B3
:100C50009847D8F854302BB19B681BB11FFA8AF122
:100C600038469847002CC1D102B0BDE8F087D8F8CB
:100C70000C30D9F834105B6808F104009847002C58
:100C8000B4D1F1E7D8F82430D9F838105B6808F10E
:100C90001C009847002CA9D1E6E7D8F83C30D9F8D9
:100CA0003C105B6830469847002C9FD1DCE7D8F8B1
:100CB0005430D9F840105B6838469847002C95D1DD
:100CC000D2E7042B07D8DFE803F00319140F0A005A
:100CD000D9F840300193019B002C87D1C4E7D9F8A3
:100CE0002C300193019BF7E7D9F834300193019B35
:100CF000F2E7D9F838300193019BEDE7D9F83C30A1
:100D00000193019BE8E700BF38B5284C94F8B82C54
:100D1000012A034603D0022A09D0002038BD244905
:100D2000D1F8C823A2B984F8B82C002038BD00251A
:100D300040F20112C0E95455C0E95655A0F84421CB
:100D400000F5A27169F0D8FD84F8B85C002038BDC8
:100D5000402AD4F80C0819D9403AC1F8C8234022D7
:100D60008118C4F80C1880B2124940F201140144F1
:100D70000020C3E95411C3E95620A3F844411846A2
:100D800003F5A27169F0B8FD002038BD4FF00005F1
:100D9000C1F8C85302EB0001C4F80C1808BF0221C7
:100DA00080B208BF84F8B81CDEE700BF982000209E
:100DB00090310020542D002001EB810138B500EB6B
:100DC000C1010E4DB1F88C1304462846FFF768FCAC
:100DD000E378C4F8A85340210022C4E9EC120122B0
:100DE00093422046A4F89C2304F5677108BFC4F819
:100DF000AC5369F081FD002038BD00BF5C35002098
:100E000038B52A4BD3F80C240F2A04D0511CC3F850
:100E10000C14002038BD264A92F8B85C0021C3F8B3
:100E20000C14002DF5D1D2F80C18D2F81048B1F5F9
:100E3000006F30D0A14235D002F6BC4594BF641A91
:100E4000C1F5006415FA81F5402C19D82144C2F887
:100E50000C184FF00001C3F8C8130CBF0223012384
:100E600082F8B83C40F201120023C0E95455C0E9B1
:100E70005643A0F8442100F5A27169F03DFDC8E792
:100E8000403CC3F8C84340310123C2F80C1882F833
:100E9000B83C4024E6E7C2F80C581CB1294602F6DB
:100EA000BC45D1E7002382F8B83CB2E7903100207E
:100EB0009820002038B5224DD5F8183495F830C464
:100EC000044623B195F81C345CEA030331D00123B6
:100ED000E06984F8463140F20112A4F84421026826
:100EE0001849002AA8BFC2F380739B0301EA12418C
:100EF00043F020030B4363F31F42BCF1020F026077
:100F000000D038BDE278104BC4F8A8331F20002170
:100F1000C4E9EC01012A4FF00101A4F89C1308BFB9
:100F2000C4F8AC3304F567712046BDE8384069F079
:100F3000E3BC012166F0D2FD95F830C4C7E700BFDD
:100F400090310020DFBFFFFFA035002070B590F882
:100F5000CF2590F8D13590F8CE5590F8D0C590F8BF
:100F6000CC1590F8CD6505EB02250CEB032C90F821
:100F7000D32590F8D23503EB0223012284B080F808
:100F8000112101F01F029BB2ADB21FFA8CFC012AA5
:100F900004468DF80810ADF80A50ADF80CC0ADF855
:100FA0000E30C0F840318DF809600AD0022A57D0BF
:100FB000002A3CD001F0800166F090FD002004B0D2
:100FC00070BD90F81231032B2BD15FFA8CFCBCF171
:100FD000010F26D8D0F8E43502A99B689847BDF8E0
:100FE0000E30002BEAD1C4E94A33C4E94C33042162
:100FF0004FF4807284F81111A4F81C2104F58E714D
:10100000204669F00BFC636DC44A1A61E278012A3C
:10101000D4D104F2CC545C614FF0802219681A607C
:10102000CCE7204666F022FD002004B070BD092EFA
:10103000F7D801A252F826F0E3100008F3110008D7
:10104000231000082D120008231000085B1200086E
:10105000071100082310000871110008A1110008F1
:1010600001F0600120295FFA8CF334D0012E00F0EA
:101070006181032E00F09581002E9FD190F81221FE
:10108000022A00F01B81032ACBD11CF0800F40F014
:10109000A48103EB830300EBC30393F87633002BA7
:1010A00000F0A6819E4B0122C3F840249D4A0223F2
:1010B000C4E94E334FF48070002184F81131A4F854
:1010C0001C01C4E94C31C4E94A2204F58E71204662
:1010D00069F0A4FB72E7D0F8E43502A99B68984751
:1010E0006CE790F81231023B012B9AD88C4BD0F868
:1010F00018210021C3F8381412B10222C3F8382491
:10110000894A0223D4E72E0A022EADF8063000F0F9
:10111000CD81032E00F09181012E82D1D0F8EC35E3
:1011200080781B680DF106019847BDF80630002B4A
:101130003FF444AFBDF80E20002A3FF43FAF934286
:1011400028BF13464FF480720221A4F81C2100220C
:10115000C4E94A0084F81111C4E94E33C4E94C32A1
:1011600004F58E712046ADF8063069F057FB25E78F
:10117000012B7FF456AF90F81221022A00F049812A
:10118000032A7FF44EAF4FF4807100F5887202207D
:10119000A4F81C11C4E94E3384F81101002190E732
:1011A000EDB25F4E012D86F831543FF63AAF90F81C
:1011B0001231022B00F02181032B7FF432AF002D7E
:1011C00000F07F8190F81011012910D0D0F8E4359B
:1011D0005B68984796F83114D4F8E43584F8101118
:1011E0001B6820469847D4F8E8359B689847002349
:1011F000F9E690F81231023B012B3FF612AF012DB8
:101200007FF4DCAED0F8E43500259B68C0F81851B7
:1012100002A9984704224FF48073C4E94A55C4E9EF
:101220004C5584F81121A4F81C31E7E6012D00F09B
:10123000CC80022D7FF4C2AE5FFA8CF3002B7FF4DA
:10124000BDAE02694FEA1C23023B5268032B00F239
:101250005681DFE803F05B426B5F5CEA03037FF4D7
:10126000E0AE90F81221032A3FF4DBAE016905F0ED
:101270007F0680F8146108681A4665F30A12024373
:101280000A604FF480720421C4E94A33C4E94C3344
:1012900084F81111A4F81C2104F58E71204669F020
:1012A000BDFA636D1D4A1A61E278012A0DD0002E45
:1012B00000F01281022384F812317FE65A063FF4CF
:1012C0007DAE194666F00AFC78E604F2CC525A610B
:1012D0004FF0802219681A60E9E7032363F30612CE
:1012E00001210F4D84F816110421002384F81111F7
:1012F0004FF48071A4F81C11C4E94A33C4E94C339B
:1013000004F58E712046C5F83C247AE6022363F387
:101310000612E5E7052363F30612E1E7180008600B
:1013200090310020D0350020C8350020042363F31D
:101330000612D5E790F81221022ABFD0032A7FF4C3
:1013400070AE002D7FF43AAE13F07F023FF44FAF42
:101350001CF0800F40F0C48003EB830100EBC1015F
:1013600081F8742381F8765381F87553282101FBA5
:10137000030300EB820293F87713506D03688A1E13
:10138000012A6FF35553D4F8E4258CBFC3F30071E1
:10139000012161F31C739268036002A92046904703
:1013A00025E790F81221022A88D0032A7FF439AE6B
:1013B00025B9590602D0194666F090FBD4F8E435F9
:1013C00002A99B682046984711E7D0F8E43502A9A6
:1013D0009B68C0F81851984709E703F07F0303EBB7
:1013E000830300EBC30393F81E31002B7FF45AAE46
:1013F000454B0022C3F8402458E6002D3FF40AAFC5
:1014000001210322D0F8E43580F8101180F8122170
:10141000E6E63E4984F811214FF480700022C4E9C9
:101420004A11A4F81C01C4E94E33C4E94C3204F556
:101430008E71204669F0F2F9C0E5EDB2052D3FF658
:10144000F0ADDFE805F02B231B130B03D0F8EC35D0
:1014500080789B690DF10601984766E6D0F8EC3577
:1014600080785B690DF1060198475EE6D0F8EC35AF
:1014700080781B690DF10601984756E6D0F8EC35E7
:101480008078DB680DF1060198474EE6D0F8EC3520
:1014900080789B680DF10601984746E6D0F8EC3558
:1014A00080785B680DF1060198473EE6D0F8E43598
:1014B00080789B6A0DF1060198474670C4F8F005E4
:1014C00033E60222D0F8E43580F8122180F810517A
:1014D0005B68294698479DE6012384F812316DE543
:1014E000282303FB020181F81C2100EB820281F812
:1014F0001E5181F81D61906991F81F113EE701238B
:1015000063F30612ECE600BF90310020C4350020E2
:1015100010B5044629B990F81121032A0DD00020F6
:1015200010BDD0F8E4359B69002BF8D090F812215B
:10153000032AF4D19847002010BDD0F890230B4621
:10154000D0F87C138A4213D9C078521A0128C4F803
:10155000902336D08A4228BF0A4692B2C4E9E223D9
:1015600004F55D71A4F87433204669F057F9D6E7A5
:10157000D0F8E4351B691BB190F81221032A1ED064
:1015800000234FF480720421C4E94A33C4E94C3388
:1015900084F81111A4F81C2104F58E71204669F01D
:1015A0003DF9636D104A1A61E278012AB7D104F25D
:1015B000CC545C614FF0802219681A60AFE79847FD
:1015C000DEE78A42D4F88003A4F8743328BF0A46C1
:1015D000084492B2C4E9E22304F55D71C4F88003C3
:1015E000C4F88403C0E700BF1800086038B504469B
:1015F00049B990F81131022B11D094F81631012B12
:1016000040D0002038BDD0F8E4355B69002BF8D01D
:1016100090F81221032AF4D19847002038BDD0F861
:101620003831D0F82421934236D9C178012908BF36
:10163000D0F82811A3EB020318BFD0F82821C0F876
:10164000383108BF52189BB24FF480710025C0E9B1
:101650004C35A0F81C11C0E94A2200F58E7169F0E2
:10166000DDF8E378C4F88053012BC4E9E255A4F80F
:10167000745308BFC4F8845304F55D71204669F0C3
:10168000CDF8BAE72A4B2269D3F83C145160002305
:1016900084F81631002038BDD0F83C31B3FBF2F5A8
:1016A00002FB1535ADB99A4213D8D0F840219342C8
:1016B0000FD24FF48073A0F81C31C0E94A55C0E93D
:1016C0004C5500F58E7169F0A9F8E378C4F84051E3
:1016D000C8E7D4F8E435DB681BB194F81221032A7B
:1016E00023D0E2780023012A4FF0050108BFC4F897
:1016F0008433C4E9E23384F81111C4F88033A4F8C8
:10170000743304F55D71204669F088F8636D094A09
:101710001A61E278012A7FF470AF04F2CC525A6168
:101720004FF0802219681A6067E720469847D8E78B
:101730009031002018000860F8B50B7813F06006AF
:101740000D46044620D0202E25D1CE884EB31B0650
:1017500049D5384F687832463946FEF75DFFEB8849
:101760000222002684F811214FF48072C4E94E331E
:10177000C4E94A77C4E94C36A4F81C2104F58E71FB
:10178000204669F04BF80AE04B780A2B17D00B2B58
:101790000ED0062B03D1204666F068F902263046AB
:1017A000F8BD022248781144FEF736FF3046F8BDF6
:1017B0008B78002B3AD1204BC3F84464EFE7022228
:1017C00080F811214FF48072A0F81C211B4A0123DC
:1017D000C0E94E33C0E94A22C0E94C3600F58E71AB
:1017E00069F01CF8DBE7164B164A4978116003F6DE
:1017F00018020321C0E9E46680F81111C0F888637B
:10180000C0F88023C078C3F8146801284FF00003A3
:10181000C4F88C33A4F8743304F55D7108BFC4F8C0
:101820008423204668F0FAFF0026B8E766F01EF928
:10183000B5E700BFB028002090310020D43500204B
:101840009820002000000020002310B5194604460F
:10185000402268F073FF802120460023402268F078
:101860006DFFD4F8E835A078012284F812215B6876
:101870009847002010BD00BF10B502230446402247
:10188000812168F05BFF204602234022012168F09D
:1018900055FF204603230822822168F04FFF0E4B9C
:1018A0000222A3F84C20FEF7A3FEE2780B4BC4F80B
:1018B000A83340200021C4E9EC01012A4FF00101C6
:1018C000A4F89C13204604F5677108BFC4F8AC3334
:1018D00069F012F8002010BD000000205C350020E7
:1018E00070B5812182B00446314E68F0F5FE0121C9
:1018F000204668F0F1FE0025022340228121204687
:1019000086F82F5968F01AFF012102234022204651
:1019100068F014FF274B86F82F59D3F8482483F832
:1019200030541268284690470095009BE16843F0C8
:1019300010030093009B0B610A691F4B009203E0A8
:101940000A690092013B02D0009AD006F8D4002325
:101950000193019B43F020030193019A164B012050
:1019600060F38A120192019A0A610A69019203E006
:101970000A690192013B02D0019A9206F8D4E278FA
:101980000E4BC4F8A83300211F20C4E9EC01012A42
:101990004FF00101A4F89C1304F5677105D02046AF
:1019A00068F0AAFF002002B070BDC4F8AC33F6E7BF
:1019B0009820002090310020400D0300A035002029
:1019C0002DE9F047089F884615460021202204464D
:1019D0001E4670F0F4FA4FB13B68E3811B0C238282
:1019E0007B687A89E3821B0C62822383404669F01C
:1019F000E9FCEB0619D4431EB8B108EB000701E07F
:101A0000013B12D317F801CDBCF12E0FF8D1C01A4B
:101A1000421E032AA8BF0322082B03F1010AA8BF14
:101A200008239146C2441A4606E008280246C246E8
:101A3000A8BF08224FF000094FF020334146236031
:101A4000636004F10807204670F080F8174B23818B
:101A50005146BB704A46384670F078F8611EE31D67
:101A600011F801CFACF1610EBEF1190F9CBFACF1C2
:101A7000200C81F800C08B42F2D1384604F10B01F2
:101A800010F8013BA3F16102192A9CBF203B00F82A
:101A9000013C8842F4D118232373330CA382E572EE
:101AA000099B6683E361BDE8F08700BF202020002A
:101AB0002DE9F04FDFF89494D9F8D80AB9F8DC4A48
:101AC000448387B0002B00F0DE8001F5FE781344DC
:101AD000DFF87CB40393164601F12007C24621E0EB
:101AE000002E64D0D9F8943CB34200F0D180D9F8EC
:101AF000903CB34200F00481D9F8983CD9F89C1C82
:101B0000B3424BD8B14200F29E81711A204665F073
:101B10005BFF039B01369E4207F500770AF5007ACA
:101B200000F0AD80D9F8A05CB542A7F12004D7D869
:101B3000751BD9F8B08C05F00702EB080492D8F8B1
:101B400030200233934203D3D8F8382093420BD984
:101B500041461846059365F007FF059B804600281F
:101B600000F09181C9F8B00C98F80420002A40F0E8
:101B70003981D8F82850002D00F07E81D8F8302027
:101B80009B1A049A02EBC303D8F80C20204602EB00
:101B900043224FF400714346A847BAE7B142B4D993
:101BA00020464FF40072002170F009FAB1E74FF4BB
:101BB00000723146204670F002FA802387F89E3189
:101BC0000C2387F8A231D9F8903CD74AD9F8881C61
:101BD000C4F8C6319342C4F8CA1100F33981D34A1C
:101BE000D34C82FB03021A44D817C0EB621284FB69
:101BF0000254D04D85FB03C5C0EB2530C2EB8215E6
:101C000087F8A1015B1B801020F03F0001330343E4
:101C1000144487F8A031D317C3EBE4142244C24B19
:101C200087F89F214A1E9A4200F31E81BF4BC0488D
:101C300083FB02311144D317C3EB611180FB0140D8
:101C4000BC4C84FB0254C3EB2433C1EB811487F8F2
:101C5000A531121B9B1023F03F03013213430844AC
:101C600087F8A431CB17C3EBE010014487F8A31128
:101C7000552387F8DE31AA2387F8DF3149E7D9F801
:101C8000D80AB9F8DC4A0483002007B0BDE8F08F19
:101C90004FF0FF3384F8EC3184F8ED3184F8EE3105
:101CA00084F8EF31D9F8A83CC4F8E8315223237006
:101CB00063706123A37084F8E73141230025E3704A
:101CC00084F8E631722384F8E43184F8E5314FF486
:101CD000F0722946A7F11C0070F071F95523C7F87E
:101CE000D051C7F8D451C7F8D85184F8FE316FF0FD
:101CF000550384F8FC5184F8FD5184F8FF3108E75E
:101D000000214FF40072204670F059F98A4A03CA44
:101D100047F81D0CEB2007F8200C582007F81F0C83
:101D2000902047F8191C07F81E0C002302220821F6
:101D3000F820E372227307F8131CA273E37307F809
:101D4000102C07F80B0CD9F8900C84F82C20D9F83B
:101D5000882C6376121A2262D9F8980CD9F89C2C38
:101D6000E376121A3F2020764FF0FF30A0763E2017
:101D7000207701206377A377E37784F82D3084F808
:101D80002E3084F82F30626284F8300084F83130CD
:101D900087F82610802187F82010292187F8221043
:101DA000942187F823100E2187F824100D21634A0F
:101DB00087F82510552187F8DE11AA2187F8DF1151
:101DC00003CA5F4BC7F82700C7F82B1003CB138853
:101DD000A7F82F309378C7F83200C7F8361087F885
:101DE000313096E64FF400720021204670F0E7F89B
:101DF000049B002B4ED1D8F84030002B00F0AA8075
:101E0000049AD8F830304F49CDE9002220461122FB
:101E1000FFF7D6FDD8F840301A6C002A00F0AD80EC
:101E2000049A1B6BCDE90022474911223846FFF77F
:101E3000C7FDD8F8448007F120044FF4E075B8F1ED
:101E4000000F3FD165E6F11A204665F0BDFD60E662
:101E5000FF2387F89F3187F8A13187F8A031324BF3
:101E60004A1E9A427FF7E2AEFF2387F8A33187F834
:101E7000A53187F8A431FBE6294620464FF40072CD
:101E800070F09DF845E6A7F1240343F804BF9A4596
:101E9000FBD13EE6D8F84030049AD8F84480002BB5
:101EA0000CBF01230223C3EB02154346002B3FF472
:101EB00030AE013D9B6CF9D198464FF40075002B74
:101EC0003FF427AE2544203423462035444604966B
:101ED00098460EE05CF81C1B236BCDF800C0002672
:101EE0000196FFF76DFDA46C08F12008CCB14545C3
:101EF00017D02379A44604F11C0E1122A8F120006A
:101F0000002BE7D162792669236B216842F0210218
:101F1000CDE900E6FFF754FDA46C08F12008002C81
:101F2000E5D1049EF5E500BFFF03FB008320088296
:101F3000818080809755454140BF07084CBF070806
:101F400058BF0708F0C5070894C507089820002067
:101F5000DEADBEEF049BD9F88C1CCDE900332046E2
:101F60000822FFF72DFDD8F84480B8F1000F3FF4A8
:101F7000D0AD3C464FF4F075A4E7049BCDE90033A7
:101F800052E700BF8C46134601466246184648F0A9
:101F90000BBA00BF1049114BD1F8882042F47002EF
:101FA00010B4C1F888201A680D4C002042F00102DC
:101FB0001A6098601A6822F0847222F480321A60E3
:101FC0005C601A68074C22F480221A60D8608C602A
:101FD0005DF8044B704700BF00ED00E000380240A0
:101FE0001030002400000008704700BF2DE9F843BE
:101FF00046697EB9D0F80080C8F30D0904460F4643
:10200000B9F1000F26D03F68FEF788F9092804D0FF
:102010006FF001063046BDE8F8834A4D2B6923F482
:1020200040732B612B6943F400732B612B6943F0E0
:1020300001032B61C8F80070FEF770F92B690928BD
:1020400023F001032B61E3D123680433236030467E
:10205000BDE8F8833C4B98452AD303F58043984567
:1020600024D303F58043984554D3384B984554D92D
:1020700003F58033984553D903F50033984552D979
:1020800003F50033984551D903F5003398453ED9FF
:1020900003F5003398454CD903F5802398454BD977
:1020A000B8F1016F4BD305200DF064FA4FF0080929
:1020B000FEF734F9092804D04FF0FF363046BDE86A
:1020C000F883204D2B6923F440732B612B6943F473
:1020D00000732B612B6923F0F8032B612B6943EA12
:1020E000090343F002032B612B6943F480332B6116
:1020F000FEF714F92B6923F002032B612B690928E1
:1021000023F0F8032B61D7D1D4F800807BE74FF0A0
:102110003809CDE74FF01009CAE74FF01809C7E7B3
:102120004FF02009C4E74FF02809C1E74FF030090C
:10213000BEE74FF04009BBE74FF04809B8E74FF062
:102140005809B5E7003C024000400008FFFF0008C6
:102150000148FEF75FB800BFB80000200148FEF755
:1021600059B800BF040300200148FEF753B800BF70
:10217000500500200148FEF74DB800BF9C07002025
:102180000148FEF747B800BFE80900200148FEF704
:1021900041B800BF340C0020704700BFF0B5254B9C
:1021A0000268254983B00646002401E051F8343026
:1021B0009A4209D001340E2CF8D100211F4A052083
:1021C00004F0F6FF002113E01D4F07EB8407D7F85A
:1021D0004C5485B1717901EB410305EBC303002237
:1021E0001820C3E9032200FB01559E601A75291DC2
:1021F000084603B0F0BD0A21642005F0B9F8014695
:10220000C7F84C0470B1294664226FF0D8FE0A4B1F
:10221000D7F84C5403EBC404C5E90045ED616D6388
:10222000ED64D7E70190074A052004F0C1FF01994A
:10223000DEE700BF000001405021070864BF070827
:10224000903100208CBF0708704700BFB0B14B68C9
:1022500010B4A3B18B6813B343681A6881605879CE
:102260009189022383400B439BB2938193899BB254
:1022700043F0010393815DF8044B70477047436856
:102280001A685C7993894FF0020C0CFA04FC9BB23B
:102290008C6823EA0C039381A4B18160E6E744686B
:1022A0002268938923F001031B041B0C9381816036
:1022B000607991895DF8044B022383400B439BB204
:1022C00093817047938923F001031B041B0C9381B6
:1022D0008160D0E738B5D0E9004307EE902A1B684B
:1022E000354A20680139934204688DB216D002F550
:1022F0008062934212D002F5705293420ED002F5E2
:10230000806293420AD002F58062934206D02B4B42
:10231000D3F87C3E5B0807EE103A04E0274B03F647
:102320007C6393ED007ADFED266AB8EE477AF8EE2B
:10233000677A87EE270A30EE260A6CF019FC1E4AEF
:1023400023880138944280B29BB212D002F5806299
:1023500094420ED0B4F1804F0BD0A2F5803294425B
:1023600007D002F58062944203D002F58062944265
:1023700002D123F070039BB2124A944212D002F5AC
:10238000806294420ED023F4407302F56C429BB2FB
:1023900094422380E56220850AD10023238601230D
:1023A000A38238BD2380E56220850123A38238BD46
:1023B000054B9C42F1D0F8E70000014000000020EE
:1023C0000AD7233C001000400004014070B540686B
:1023D000837903F0020213F0040300F0C9804FF088
:1023E000000E134604247246754690F805C0BCF1F1
:1023F000030F30D8DFE80CF08E5F30020368188CD2
:1024000020F480500004000C1884188C9C8820F460
:10241000005000042A43000C40EA0232988B6C4DB5
:1024200020F4E6400004000CAB42A4B240F4C040EB
:1024300000F0B08005F58065AB4200F0AB809C8079
:10244000988319641A849A8B22F400621204120C85
:1024500042F400629A8370BD2A4305685C4E288C62
:1024600020F480700004000C2884288CB5F804C087
:1024700020F400700004000C40EA0222A88B20F037
:1024800073000004000CB5421FFA8CFC40F06000A1
:1024900073D006F58066B5426FD0A5F804C0A88356
:1024A000E9632A84AB8B23F008031B041B0C43F065
:1024B0000803AB8370BD2A430568454E288C20F085
:1024C00010000004000C2884288CB5F804C020F00B
:1024D00020000004000C40EA0212288B20F4E640A1
:1024E0000004000CB5421FFA8CFC40F4C04061D0DF
:1024F00006F58066B5425DD0A5F804C02883A963BF
:102500002A842B8B23F400631B041B0C43F400630D
:102510002B8370BD00682E4E2A43058C25F00105E3
:102520002D042D0C0584058CB0F804C025F002059F
:102530002D042D0C2A43058B25F073052D042D0C3D
:10254000B0421FFA8CFC45F0600528D006F5806685
:10255000B04224D0A0F804C0058341630284038BF9
:1025600023F008031B041B0C43F00803038370BD16
:102570004FF4807E1C46012537E722F4006242EAD0
:10258000032222F480622CF4405C42EA04224CEAEA
:102590000E1C82E724F4804444EA8E144FE74FF681
:1025A000F37616402CF4407C46EA03024EEA0C0C0B
:1025B0002243CFE722F0800242EA031222F04002D7
:1025C0002CF4406C42EA04124CEA8E0C94E700BFF3
:1025D0000000014070B4EFF31182102383F31288DE
:1025E000C4684668A5682B6823F001032B60356832
:1025F000114B767933F81660AB899BB223EA060358
:10260000AB81236965681F2B11D9203B202404FA74
:1026100003F3EB60D3B283F31188C3689B685960FE
:102620001A68012422431A60047470BC7047202485
:1026300004FA03F3AB60EDE7F820070803681A7D9E
:10264000012A04BF02221A7593F82C100CBF4FF414
:1026500000720022012904D1022183F82C1042F4D7
:10266000806293F84410012905D093F85C10012989
:102670000AD072B97047022183F8441093F85C10B5
:10268000012942F4006204D1022183F85C1042F473
:1026900080524168096800234B628B899BB21A43C0
:1026A0008A817047024B0348D3F84C14FEF78EBA68
:1026B000903100200000014010B5064C0648D4F8C7
:1026C0004C14FEF783FAD4F86C140448BDE81040AB
:1026D000FEF77CBA9031002000000140004001402C
:1026E00010B5064C0648D4F84C14FEF76FFAD4F82F
:1026F00070140448BDE81040FEF768BA903100201D
:10270000000001400044014010B5064C0648D4F8D2
:102710004C14FEF75BFAD4F874140448BDE810407A
:10272000FEF754BA903100200000014000480140FB
:10273000034B4FF08040D3F85014FEF747BA00BF68
:1027400090310020024B0348D3F85414FEF73EBAF0
:102750009031002000040040024B0348D3F8581485
:10276000FEF734BA9031002000080040024B0348C5
:10277000D3F85C14FEF72ABA90310020000C004018
:10278000024B0348D3F86814FEF720BA90310020BA
:102790000004014010B5064C0648D4F86814FEF752
:1027A00015FAD4F878140448BDE81040FEF70EBAC4
:1027B00090310020000401400018004010B5064C84
:1027C0000648D4F86814FEF701FAD4F87C140448DB
:1027D000BDE81040FEF7FAB9903100200004014036
:1027E000001C004010B5064C0648D4F86814FEF7EB
:1027F000EDF9D4F880140448BDE81040FEF7E6B9BE
:102800009031002000040140002000400348D0F82F
:102810008C3E13B100F56860184770470000002037
:102820000348D0F8AC3E13B100F56A601847704712
:10283000000000200348D0F8CC3E13B100F56C60D6
:1028400018477047000000200348D0F8EC3E13B151
:1028500000F56E6018477047000000200348D0F86C
:102860000C3F13B100F5706018477047000000205E
:102870000348D0F82C3F13B100F572601847704739
:10288000000000200348D0F84C3F13B100F57460FD
:1028900018477047000000200348D0F86C3F13B180
:1028A00000F5766018477047000000200348D0F814
:1028B0008C3F13B100F57860184770470000002086
:1028C0000348D0F8AC3F13B100F57A601847704761
:1028D000000000200348D0F8CC3F13B100F57C6025
:1028E00018477047000000200348D0F8EC3F13B1B0
:1028F00000F57E6018477047000000200248C3685A
:1029000003B11847704700BF001000200248C36A97
:102910000BB1203018477047001000200248C36CEC
:102920000BB1403018477047001000200248C36EBA
:102930000BB160301847704700100020026836491C
:10294000002310B422F001022124884202600360B7
:1029500043608360C3600361446138D02F4B984269
:102960002ED02F4B98423CD02E4B984240D02E4B2D
:10297000984232D02D4B984241D02D4B984246D0B0
:102980002C4B984217D02C4B98423CD02B4B984262
:1029900016D02B4B984224D02A4B984228D02A4B51
:1029A00098421AD0294B984229D0294B98422ED0D0
:1029B000284B984208D14FF03D5243F8AC2C03E02D
:1029C0004FF4746243F8202C5DF8044B7047224B9F
:1029D0005DF8044B3D229A607047204A43F8642C0E
:1029E000F2E74FF474125DF8044B43F8382C70474B
:1029F0004FF074625DF8044B43F8502C7047184A4E
:102A000043F87C2CE0E73D2243F8082CDCE7154A2C
:102A100043F8942CD8E700BF1060024028600240C1
:102A2000406002405860024070600240886002408E
:102A3000A0600240B8600240106402402864024076
:102A4000406402405864024070640240886402405E
:102A5000A0640240B8640240006002403D000020D3
:102A6000400F002000003D2000222DE9F0471346D2
:102A70000D684FF0010E032604E00133102B02F124
:102A8000020239D00EFA03FC3CEA0504F5D10768CE
:102A900006FA02F427EA040707600F79D0F800A0CD
:102AA00007FA02F9013F49EA0A09012FA046C0F8D6
:102AB00000906FEA040411D887683C4084604C7928
:102AC000876894403C438460446824EA0C04446072
:102AD0008C7947689C40A4B23C434460C46824EAB3
:102AE0000804C460CC79C768944001333C43102B80
:102AF000C46002F10202C5D1BDE8F0872DE9F041C2
:102B00002348244F244E254C82B0382200216FF0F8
:102B100056FA002557F825103246002301E054F8F4
:102B2000332091422ED001330E2BF8D100200535F1
:102B300065F0FCF94B2DEDD1DFF85880184F08F502
:102B400096754FF0007698F8040007F0B5FD08F18F
:102B50001408044688B1036803F13F4303F57E037C
:102B600007EB932393F8C80065F0E0F9A38801967A
:102B7000206800936946FFF777FFA845E3D102B0CC
:102B8000BDE8F081064A02EBC30393F85C00CEE790
:102B9000DC35002080100020000001405021070893
:102BA000F8200708224A936803F00C03042B10B4A2
:102BB00021D0082B22D01F4B03601D4C1E4AA16858
:102BC000C1F30311114491F8B410CB404360A168E4
:102BD000C1F38221114491F8B41023FA01F181600C
:102BE000A1685DF8044BC1F342310A4492F8B42065
:102BF000D340C3607047114B0360DEE753685168F0
:102C000013F4800F01F03F01536814BF0B4A094AC7
:102C1000B2FBF1F1064A5268C2F30142C3F38813D2
:102C2000013201FB03F35200B3FBF2F30360C4E78C
:102C3000003802400024F400F810002000127A004E
:102C400070B5446B8668A38923F400531B041B0CE6
:102C5000A38182790546407912F0040F14BF4FF426
:102C6000805C4FF0000C110310F0010F4FEA0222BC
:102C70000CBF0023042302F48062800748BF43F0A6
:102C8000080342EA0C021343228A92B201F4005173
:102C900022F440520A432282A28922F4B05222F046
:102CA0000C021204120C1A43A281A38A23F440736B
:102CB0001B041B0C84B0A3826846FFF773FF244BF0
:102CC0009C4205D003F580639C4201D0029A00E04B
:102CD000039AA3891F491B0402EB82024CBF7300B5
:102CE000B30002EB8202B2FBF3F3A1FB0302A08963
:102CF00052096426000406FB12334FEA02121FD465
:102D00001B013233A1FB0313C3F3431313439BB2E1
:102D10002381AB796A6B13F0080F938A0AD09BB2B8
:102D200043F00803938293899BB243F40053938149
:102D300004B070BD23F008031B041B0C9382F2E760
:102D4000DB003233A1FB0313C3F342131343DEE76B
:102D5000001001401F85EB512DE9F843394C9DF8D7
:102D600020509DF82490A0420F4690461E4649D020
:102D7000354B98424ED0354B984253D0344B984205
:102D80002BD0344B984255D0334B984221D14B46EF
:102D90002A4631460520FDF753FE04460023C4E9C8
:102DA0000B78C4E90733C4E909336571A66084F878
:102DB00006902046FFF744FFEA07616B1AD4AB0781
:102DC00013D48B899BB243F400538B812046BDE81A
:102DD000F88300242046BDE8F8834B462A46314656
:102DE0000320FDF72DFE0446D8E7CB6843F08003AF
:102DF000CB60E6E74FF6DF730B80CB6843F0200330
:102E0000CB60DCE74B462A4631460020FDF718FE32
:102E10000446C3E74B462A4631460120FDF710FE23
:102E20000446BBE74B462A4631460220FDF708FE22
:102E30000446B3E74B462A4631460420FDF700FE20
:102E40000446ABE700100140004400400048004049
:102E5000004C004000500040001401408160EFE64B
:102E60004171EDE62DE9F043DFF8148208EBC0096B
:102E700085B00546C70099F8C80007F01DFC044658
:102E800099F8C90007F018FC064699F8CA0065F0E1
:102E90004DF86B1CDBB2002C00F0AD8040F60E123A
:102EA0002372E280002E00F0C380337240F60E23BE
:102EB0002046F38004223A2107F0F6FD0422304632
:102EC0003A2107F0F1FD08EB0703624AD3F8C4404A
:102ED000944200F09880604B9C4200F09E805F4BD3
:102EE0009C4200F0AB80474497F8CB20022A5CD08C
:102EF000032A7ED05A4B5B4E012A18BF1E46A78874
:102F00006846FFF74FFE27F03F07029B564AB3FB88
:102F1000F6F63F04A2FB03233F0C47EA9347A78042
:102F2000228822F001021204120C2280B2B2C6F3EF
:102F30000B069B0C002E59D04FF4967101FB03F346
:102F40004A49A1FB03139B0901339BB242F400429F
:102F50002384A2832388464A9BB243F00103238043
:102F6000238823F4816323F002031B041B0C4FF41A
:102F7000804143F4806323802181238823F08003F0
:102F80001B041B0C238023889BB202EB451243F0E9
:102F9000010323800121002382F8885482F88914D8
:102FA00082F88A3405B0BDE8F083A6886846FFF74A
:102FB000F9FD26F03F06029A2B4B3604A3FB0213C1
:102FC000360C46EA9346A680218821F001010904C7
:102FD000090C21809B0C2749013392092384A1FB12
:102FE00002329209042A38BF0422B2E742F00102F9
:102FF000A2E7214E83E7002E3FF465AF337240F61F
:103000000E23F3805AE71D4B1A6A42F400121A622B
:103010001A6A22F400121A6265E703F5F0331A6A9D
:1030200042F480021A621A6A22F480021A625AE793
:10303000042220463A2107F037FD44E703F5EE333A
:103040001A6A42F400021A621A6A22F400021A6230
:1030500049E700BF0054004000580040005C0040B9
:10306000804F1200009F240083DE1B43D34D62106B
:1030700090310020632D3E05C02709000038024032
:10308000F81000202DE9F047954D90F9001080468A
:10309000807805EBC1060138CC0090B0D6F8C4109A
:1030A00014282ED8DFE810F0530126011500570030
:1030B0006100A200AA00CB01BD017D00870045028E
:1030C0000D02E001C500D50030003800AA019C01C6
:1030D0005B01888A0C8B81B2824841EA044130EA64
:1030E000010100F02681D8E90210521A42F2107153
:1030F00063EB00038A4273F1000302D3152388F8BF
:10310000023010B0BDE8F08798F813000882C8E9D3
:103110000223122088F80200888A0C8B80B240EAD1
:103120000440714C34EA000000F0B68000200E909C
:103130000F9001200F910E900E99002900F01E8231
:103140000F9914310F910F9909684905CBD51423B4
:1031500088F80230D5E798F8110000F0FE000882E8
:10316000C8E90223052088F80200888A0C8B80B207
:1031700040EA04405D4C34EA000000F0A4800020E6
:10318000009001900120019100900099002900F029
:103190000182019914310191019909684F05D6D432
:1031A000A1E798F8110040F001000882C8E9022365
:1031B0000B2088F80200888A0C8B80B240EA044019
:1031C0004B4C34EA00006FD00020049005900120A1
:1031D000059104900499002900F0D68105991431D5
:1031E0000591059909684D05B1D47CE798F813005D
:1031F0000882C8E90223072088F80200888A0C8B1D
:1032000080B240EA0440384C34EA00005FD000202D
:10321000029003900120039102900299002900F08E
:10322000C581039914310391039909684E058ED421
:1032300059E7088820F480600004000C088098F8A2
:10324000110000F0FE000882C8E90223102088F86F
:103250000200888A0C8B80B240EA0440234C34EA96
:10326000000012D000200C900D9001200D910C90C8
:103270000C99002900F094810D9914310D910D994C
:10328000096848053FF563AF2DE798F81330FF2B29
:1032900006D198F810301BB1132388F8023030E7BC
:1032A000112388F802302CE7D8F81400012800F028
:1032B0009381022800F049820E20098B88F80200D1
:1032C000C8E902231DE7062388F8023019E7D8F879
:1032D0001400002800F07081082388F8023010E7FD
:1032E000F81000200100030084000700820007009E
:1032F00002000300088820F400600004000C08802D
:10330000088880B240F480600880088880B240F469
:1033100080700880032088F80200888A0C8B81B2B4
:10332000AB4841EA0441C8E9022330EA01037FF4D3
:10333000E8AE98F81230002B40F0D38198F81330A3
:10334000FF2B00F04682042388F80230D9E6098872
:1033500089053FF5C8AE002388F80230D1E62C4439
:1033600094F8C80007F0A8F9064694F8C90007F0D9
:10337000A3F9984AB2F8E83401339BB28246A2F826
:10338000E83416B13368B2881A83BAF1000F04D05A
:10339000DAF80030BAF804201A831121304602F01E
:1033A0008BFA1121504602F087FA4FF00909652780
:1033B0002EB13368B28819690A4240F02881013F72
:1033C00000F022810CF07AF804460D460CF076F8F5
:1033D000001B61EB0501052871F10003F6D3E7E757
:1033E000088880B240F4007008804FF6FF30888271
:1033F0000121C8E9022388F8021082E6D8F81400F7
:10340000002800F07281D8F8184014F8016B0E8281
:1034100001381225C8E90504C8E9022388F80250DA
:103420006FE6888A0C8B81B2694841EA044130EA30
:1034300001017FF458AE0A2388F8023061E608885B
:1034400080B240F480700880092088F80200888AE1
:103450000C8B81B25E4841EA0441C8E9022330EA9C
:1034600001037FF44EAEE6E7002401250A940B9495
:103470000B910A950A98002800F04A810B981430A5
:103480000B900B98006846077FF52DAED8F8140016
:10349000032800F07281022800F24681088820F497
:1034A00080600004000C0880088880B240F400703E
:1034B0000880098A88F81C40C8E9022388F802506D
:1034C0001FE60020012408900990099108940898AB
:1034D000002800F0178109981430099009980068B5
:1034E00047077FF500AEEFF31185102080F31288B7
:1034F000088880B240F400700880D8F818000E8A5E
:10350000471CC8F81870EDB2067085F311880D8A53
:10351000D8F818106FF001004E1CC8F818600D7034
:10352000C8E90223C8F8140088F81C4088F8024053
:10353000E7E5002006900790012007910690069C81
:10354000002C00F0EB80079C14340794079C24683F
:1035500064067FF5C8AD0C8AD8F818104D1CC8F861
:1035600018500C70D8F8141088F81C000139C8E9FC
:103570000223C8F8141088F80200C2E50F99183128
:103580000F910F990968AEE50599183105910599D4
:103590000968A8E501991831019101990968A2E526
:1035A0000D9918310D910D9909689CE50399183111
:1035B00003910399096896E5088880B240F4007089
:1035C00008800121C8E9022388F8021099E500BFAC
:1035D0000100030090310020088820F4806000047E
:1035E000000C0880EFF31184102080F31288088B00
:1035F000088880B240F40070E4B2088084F3118837
:103600000C2188F802105BE616B13368B2885A8341
:103610000BF054FF04460D460BF050FF031B61EB0B
:103620000501052B71F10003F6D316B13368B2889A
:103630001A830BF043FF04460D460BF03FFF031BBC
:1036400061EB0501052B71F10003F6D3B9F1010916
:103650007FF4ADAE16B13368B2885A830BF02EFFFB
:1036600004460D460BF02AFF031B61EB0501052BF9
:1036700071F10003F6D3BAF1000F04D0DAF800308C
:10368000BAF804205A830BF019FF04460D460BF0DC
:1036900015FF031B61EB0501052B71F10003F6D348
:1036A00016B13368B2881A830BF008FF04460D4642
:1036B0000BF004FF031B61EB0502052B72F1000305
:1036C000F6D3BAF1000F04D0DAF80030BAF80420CB
:1036D0001A8398F90000441C3FF43DAEFFF7C2FB8B
:1036E00039E60F2388F802300BE5088880B240F4F1
:1036F000007008800121C8E9022388F81C1088F8AE
:103700000210FEE409991831099109990968EAE45F
:103710000B9918310B910B990968E4E4079918315A
:10372000079107990968DEE4D8F81800098A441C53
:10373000C8F818400170D8F81410C8F808200139EA
:10374000C8F81410C8F80C30DBE4088880B240F4E4
:1037500000600880EFF31184102080F31288088B3A
:10376000088820F480600004000CE4B2088084F330
:1037700011880D2188F80210A2E5088820F48060E5
:103780000004000C0880EFF31184102080F31288ED
:10379000D8F818000D8A461CC8F81860057008880B
:1037A00080B240F40070E4B2088084F31188D8F845
:1037B0001800098A441CC8F818400170D8F8141081
:1037C0000C200239C8E90223C8F8141088F8020056
:1037D00097E498F81030002B3FF4B5AD2BE600BF0E
:1037E00038B5184D9DF814E005EB40144FEA401C25
:1037F00094F8890400B938BD490084F89B24C4F8C2
:103800009C3484F899140023049984F898E40222E3
:1038100005F5916584F89A34C4F8A01484F8A434AA
:1038200084F88A2465440BF049FE02460B4628467C
:10383000FFF728FC94F88A34002BF4D194F8A40400
:1038400038BD00BF9031002038B5184D9DF814E008
:1038500005EB40144FEA401C94F8890400B938BDC8
:1038600084F89B24C4F89C3401220023490005F508
:10387000916584F89A2484F8A434049A84F898E42E
:10388000022384F89914C4F8A02484F88A34654487
:103890000BF014FE02460B462846FFF7F3FB94F8A4
:1038A0008A34002BF4D194F8A40438BD9031002060
:1038B000F0B587B00023834A00930193136843F463
:1038C0008033136003E0009BB3F5A04F09D0136869
:1038D00003F400330193009B01330093019B002B01
:1038E000F1D0784B1B6813F4003318BF0123019308
:1038F000019B012B01D000BFFDE7724B72491A6C8E
:10390000724842F080521A640A6842F440420A60E7
:103910009A689A609A6842F400429A609A6842F4FF
:10392000A0529A6058601A6842F080721A601A6851
:103930009201FCD5664A40F205711160996821F048
:1039400003019960996841F00201A2F580629960D3
:10395000936803F00C03082BFAD1936803F00C036F
:10396000042B00F08D80082B00F08F80594D5A4BAE
:10397000C5F87C3E534B59499868D5F87C2E584C75
:10398000C0F303100144574891F8DC10CA4056496F
:10399000C5F87C2EE160554A596FA260596B544AB4
:1039A00021F080015963596F41F080715967196B9B
:1039B0000A431A635A6B5A639A6B9A631A6C4D499D
:1039C0000A431A64596C4C4A0A435A6402A948F2E1
:1039D000FF73002602934FF6FF770396FFF744F834
:1039E00000F580600297FFF73FF800F580600297CE
:1039F000FFF73AF800F58060FFF736F800F58060D1
:103A0000FFF732F800F58060FFF72EF800F58060D0
:103A1000FFF72AF800F58060FFF726F800F58060D0
:103A2000FFF722F80846FFF7BDF8D4F8FC30029AF9
:103A30003249334843F08073C4F8FC30314BC3F84B
:103A4000B01F5E60196841F001011960D5F87C3E35
:103A50004FF47A71B3FBF1F3013BB3F1807F2A4954
:103A6000B2FBF1F2C0F8EC2408D24FF0E022F021D2
:103A70005361072384F823109661136107B0F0BDEA
:103A8000144D224BC5F87C3E74E753685168114DC4
:103A900013F4800F01F03F01536814BF1B4A0E4A14
:103AA000B2FBF1F1074A5268C2F30142C3F3881333
:103AB000013201FB03F35200B3FBF2F3C5F87C3E85
:103AC00058E700BF0038024000700040085440072B
:103AD000003C0240000000200024F400F810002008
:103AE00000ED00E0000002400003FA0500000008BD
:103AF000FF916700FFC9FE103357070055CEACC5D4
:103B000090310020001000E040420F0000127A00C7
:103B100082B0064B002201920193019B03EB8000CF
:103B20000190019B196002B0704700BF502800400F
:103B300010B51C2006F0C0FD1121044601F0BCFEAA
:103B400014B12368A2885A83C8200BF0E5FC2046F4
:103B5000BDE8104004F08AB9704700BF704700BF4D
:103B6000704700BF10B5124C94F8FA3423B9114BCA
:103B70004FF480225A6110BD4FF0E022D2F8103D80
:103B800023F00603C2F8103DFEF704FA94F8FA3465
:103B9000002BECD0D4F800359B68DB07E7D5D4F8D0
:103BA000FC25136823F0030161F307031360DEE7CC
:103BB00090310020003C01402DE9F04FB34CD4F887
:103BC000FC345A69D2078BB002D50BB0BDE8F08F38
:103BD0005A699B6912EA0309F7D0C9F3074319F43C
:103BE000002F009340F0E180009B590743D419F067
:103BF000020F5FFA89F603D0D4F8FC3402225A612E
:103C0000B9F1000FC0F2EE8119F4006FC9F3072576
:103C100040F04A81330708D59D4B9E48D3F8F830D1
:103C20009847D4F8FC3408225A61F70600F1C481A1
:103C3000EE0600F16F81A90600F1E880009BDA062C
:103C400009D5934B9348D3F808319847D4F8FC34FE
:103C50004FF480125A61009B9B06B6D58C4B8D4861
:103C6000D3F80C319847D4F8FC344FF400125A6161
:103C70000BB0BDE8F08FD4F800259369D2691340EA
:103C80001FFA83FABAF1000FB1D0DFF81882CDF82D
:103C90000C90A8F1180500271AF0010F78D0FEB299
:103CA000D4F8002504EB86031069D3F80815536B8C
:103CB0008968F340DB01DBB203430B4013F00109D9
:103CC000D9B240F0AB810A0740F1C881D8F8002092
:103CD00008239360994619F0800F59D0D5E94CC05C
:103CE000D5F82431D8F800E0ACEB00018B42DEF8C7
:103CF000182028BF0B4692B20333B2EB930F47D97B
:103D0000D4F8002594F8F394323604EB8603CDE919
:103D10000178674698469446874237D9D5F82431CA
:103D2000391A994228BF194601F1030BD5F82831F9
:103D30004FEA9B0BB9F1000F10D18AB203329210F7
:103D4000D8F8F8640AD04846013053F8047B37604D
:103D50008242F9D1D5E94C70D5F8283108440B449A
:103D6000B842C5F82831C5F83401DEF818300AD158
:103D700095F81C11012202FA01F1DCF8342022EA44
:103D80000102CCF834209BB29B45C5D3DDE9017814
:103D90005FEA5A0A07F1010708F1040805F128054E
:103DA0007FF47AAFDDF80C9021E7D4F800359D69F7
:103DB000DB691D402D0C3FF417AF04F59E68DFF85A
:103DC000D0B004F244560027C24608E06D0807F15F
:103DD000010706F1040608F128083FF405AFEB07D8
:103DE000F4D5F9B204EB8103D4F80025D3F84435B7
:103DF0009B6852691340D807DAB200F13F819307FC
:103E000040F16781336802229A60DFE7D4F8003519
:103E1000D4F808159A680868C2F34102022A06BF5E
:103E2000032262F30A006FF30A0008605A6842F442
:103E300080725A6006A8FEF7B5FED4F8FC24D4F8C8
:103E40000015D368079D6FF38D23D36088681249EE
:103E5000C0F34100014491F8D010032900F05F81C4
:103E60000E490F480126294484F8F26481424FF03C
:103E70004006A4F8F46400F2AC810E2161F38D23B6
:103E80004FF40051D3605161D8E600BF903100205B
:103E9000F810002080360020F8200708401E1BFF85
:103EA0003F420F009836002000238DF8133094F81D
:103EB00002368DF81330B64BB648D3F80031984728
:103EC000D4F80035D4F8FC24986894F8FA344FF408
:103ED00000615161002B3FF49DAEC2077FF59AAEA1
:103EE00094F80536012B7FF495AE9DF81330032B23
:103EF0007FF490AED4F8FC35A7491A6842F001026D
:103F00001A601A6842F003021A600B6943F0060354
:103F10000B617FE6D4F80065D4F8FC1473680027C1
:103F200023F0010373600597059B43F0200305937D
:103F3000059B67F38A130593059B0B610B6905933A
:103F4000BC46964B03E00A690592013B02D0059AF4
:103F50009006F8D494F8F12452B1914B03EB820E01
:103F6000FF2253F8040F8260D86B73458260F8D14A
:103F70000B2363F3070763F3070C4FF0FF33B361C1
:103F80004FF00113F3617761C6F810C033688548BC
:103F90006FF30A13336094F8F324D4F84435012AFC
:103FA000186100F0B5804FF480534B61784B79482D
:103FB000D3F8FC3098473EE6D4F8FC349A6922F0F6
:103FC00010029A611A6AC2F34340022802F00F01FC
:103FD00000F0B080062800F087809A6942F0100255
:103FE0009A6125E694F8FA343BB1D4F8FC251368BD
:103FF00023F0030161F307031360D4F80025644B39
:104000006448D3F80411536823F0010353608847D0
:10401000D4F8FC344FF000425A61F5E5516BD8F802
:1040200000005B4B4FF0010C0CFA07FC21EA0C017D
:1040300051630122D3F8F0308260314655489847E9
:1040400094F8F334012B00F0B18019F0020F3FF423
:1040500042AED8F8003002229A6099E6CB0604D529
:10406000D8F8003010229A6092E6480658BF894678
:10407000EBD5D8F8003040229A6089E694F8F32412
:10408000336801208242986007D11A69D8F87C33DE
:10409000C2F312029B1AC8F88C33DBF8EC3050469E
:1040A000984794F8F334012B7FF490AE002F7FF4FF
:1040B0008DAE94F80136052B7FF488AED4F84435E4
:1040C000384A1A61384A5A611A684FF080221A60D9
:1040D0007CE610077FF57AAEDBF8F430504698475F
:1040E000336808229A6071E601EB810104EBC1019B
:1040F000D4F8C065D1F87C08C2F30A1202443068D3
:10410000C4F8BC0A3068C4F8C00AC1F87C2864E767
:10411000254A5A611A684FF080221A6043E700214D
:1041200084F8F2144FF40071A4F8F414092161F337
:104130008D23A5E647F6F07010423FF44EAFC2F370
:104140000A1201EB810004EBC00002F1030C5FEAEC
:10415000AC0CD0F87068D4F8C0E54FEA810818BFFD
:10416000002006D00130DEF8007046F8047B84455C
:10417000F8D1414404EBC101D1F870081044C1F8F2
:104180007008D1F87C080244C1F87C2825E700BFFC
:10419000F81000208036002000ED00E0400D030004
:1041A00094360020180008604C3C0020002F7FF45B
:1041B0004CAF94F80136042B7FF447AFD4F8443564
:1041C0002B4A1A612B4A5A611A684FF080221A60F2
:1041D0003BE72948A5F57401A1F51051814203D8A8
:1041E0000D2161F38D234BE6244925482944814262
:1041F00003D20C2161F38D2342E62248A5F18C7194
:10420000A1F54341814203D80B2161F38D2337E6A9
:104210001D491E482944814203D20A2161F38D239E
:104220002EE61B491B482944814203D2092161F330
:104230008D2325E61848A5F1B771A1F558518142A3
:1042400003D2082161F38D231AE614491448294446
:10425000814203D2072161F38D2311E611491248EF
:104260002944814234BF0621052161F38D2307E6ED
:10427000180008604C3C0020DFC810002013FBFE33
:1042800020D61300FF69180000D3CEFE40771B0034
:10429000C05BB3FEC091210040AC2700C01D6AFE88
:1042A00040E13300803C36FEE09C410070B51A4D81
:1042B0001A4BC5F8E43A1A4B85F8F01A002683F831
:1042C0002F6905F6E423C0E954330D230446C0F8F2
:1042D000583140F20113C0F85C6100F5A271A0F8FA
:1042E000443166F009FBE378C4F8B4631F22C4F8D4
:1042F000B023012205F582659342C4F8A853A4F8BF
:104300009C2308BFC4F8AC5304F567712046BDE890
:10431000704066F0F1BA00BF90310020555342530F
:1043200098200020F0B50B7813F0600683B00C469F
:10433000054633D0202E2DD14A78FE2A6BD0FF2A95
:1043400063D14A88002A40F08B80CA88002A40F056
:104350008780190600F184806148624B80F82F291C
:10436000C5F8B423EA78012183F83014A5F89C132A
:1043700003F582631F21012AC5F8B013C5F8A833DD
:1043800005F5677108BFC5F8AC33284666F0B4FA86
:10439000002600E00026304603B0F0BD4B780A2B23
:1043A0006AD00B2B63D0012BF5D18B88D9B21B06B9
:1043B00076D40196019BC06843F010030193019BE2
:1043C000036103690193484B03E002690192013BD9
:1043D00002D0019AD206F8D42846424F66F07CF902
:1043E000022321794022284666F0A8F997F8303454
:1043F000022B6DD094F90420002ACCDA012BCAD00C
:1044000001212846FFF752FFC5E763F02FFB022684
:10441000304603B0F0BD4E8816BBCC88012C1FD1AE
:1044200018061DD52F4FD7F848349B699847C0B25E
:1044300087F8F40AA0B1022307F6F42785F81131B2
:104440004FF48073C5E94E44C5E94A77C5E94C4647
:10445000A5F81C3105F58E71284666F0DFF99AE75C
:10446000284663F003FB0226304603B0F0BD1D4B27
:104470004A8883F8F52A8EE7022280F811214FF44A
:104480008072A0F81C21194A0123C0E94E33C0E90B
:104490004A22C0E94C3600F58E7166F0BFF97AE722
:1044A0000096009BC06843F020030093009B61F3DB
:1044B0008A130093009B0361036900930A4B03E096
:1044C00002690092013B87D0009A9706F8D483E7EF
:1044D0008121284663F002FB002387F830345AE735
:1044E0009820002090310020400D0300853C0020E2
:1044F00010B50D4B93F82F39022B07D0033B012B3E
:1045000002D80021FFF7D2FE002010BD074B93F820
:104510001D14044666F0A2FA0028F5DA01212046AF
:10452000FFF7C4FEF0E700BF982000209031002084
:10453000F8B5404E96F82F59074655B1012D06D1D2
:104540003D4B93F81D1466F089FA002832DB0020F9
:10455000F8BD394CB0F8B433D4F81424C4F8E82AC0
:104560001F2BD4F81824C4F8EC2A08D1334BD4F804
:1045700010249A4203D194F81D1401291FD994F8EC
:10458000F63A04EBC3020133DBB2042B4FF0050112
:1045900008BF002382F8F81A4FF4005184F8F63A65
:1045A00038460223C2F8FC1A84F83034FCF782FC47
:1045B0000020F8BD29463846FFF778FEC7E794F893
:1045C0001E34013B0F2BDAD866F048FA002827DBAF
:1045D00096F82F39013B022BB9D9B4F8183B1BB31D
:1045E000042286F82F29164AC7F85C51C7E95422DD
:1045F000D4F8182484F8F05A934228BF1346D4F80C
:10460000EC2AC7F8583140F20111A7F84411D31A27
:1046100007F5A2713846C4F8EC3A66F06DF996E7F2
:104620003846FCF747FC92E719463846FFF73EFE4E
:104630008DE700BF98200020903100205553424361
:10464000D46000202DE9F04F93B045F061FF45F0B4
:1046500025FFAB4B0793B0F1000940F329814FF0E0
:10466000000A9B46A74BA84CCDF804A002935646DF
:10467000D04604E008F50068C14540F38F80202251
:104680000AA9404645F090FEA04912220AA86DF002
:10469000E5FC05460028EDD1B04521D0019A9C4F9C
:1046A0009C49CDF80CB002EB420307EB83070132C3
:1046B0003846019202F064FDDBF81C20039B43F8AE
:1046C0004C7BCBE90822944ACBF80C60CBF828202D
:1046D000A8EB06060122CBE90466CBF808209B462E
:1046E000029BD3F81831CBF81C304646122212AB8D
:1046F000991814F80A3011F8201C994202F10102AD
:104700000CD04FF0000A202AF1D12036B1450AA979
:10471000304639DB45F048FE0022E8E70AF1010A9D
:10472000BAF1150FEFD190190AA9202245F03CFEED
:104730007A4909AA0AA86DF0E8FB28B30027CDE959
:104740000477039706973E46731E042B00F29F8161
:10475000DFE803F09A8DA29E030003F08BFA054672
:10476000069989B1DDE90423039843EA42127B01EB
:1047700043EAC023A1F2BC7143EA650342EA412245
:1047800043EA0243CBF81C30019B642B00F0B48059
:10479000464608F50068C1453FF771AF019A642AA3
:1047A00000F0AA80B0457BD0594C5A495A4F0C238F
:1047B00003FB0244531C1A462046A8EB060501934E
:1047C00002F0DEFCDBF81C30CBF80040CBE90365DF
:1047D000CBE908330123CBF81450CBF82870CBF881
:1047E0000830019B1D1D4E4C0299D4F84C61C1F854
:1047F00018614C2202FB05F56319002118466DF083
:10480000DEFB4C2200216DF0DAFBDFF820A144F83A
:1048100005A0019D8762C0E90499C0E907664FF0D1
:104820000108C0F80880466205354FEA4903B3F134
:10483000805F42DB029B3B493948D3F818514FF463
:1048400098726DF083F93649079A0C460B465D6203
:10485000C3E907554C339A42F9D1A66826B92379A2
:1048600013B12368002B63D113B0BDE8F08F03F0C0
:1048700001FA05902949002009AA6DF046FB01368E
:1048800000287FF461AF6BE703F0F4F90490F1E7DF
:1048900003F0F0F90746EDE703F0ECF90390E9E7E0
:1048A000019B1D1D002B40F0F0801D4C0425BCE732
:1048B000144A02920425A3F598744C2202FB05F5D4
:1048C0006319184600216DF07AFB4C2200216DF02F
:1048D00076FB0299C9F1006203465200124860510A
:1048E000D1F818115962C3E9042202225A71012237
:1048F000C3E907119A609DE76423074F019370E7AE
:104900008C420020F8100020CCBF0708A8BF070881
:10491000AC3C0020BCBF0708851F0008E4BF0708A7
:104920005C410020CC210708FCBF0708ECBF07084A
:10493000C4E91166584A2664E663304637468E4617
:10494000D56C02F14C0355B3D3F808C01F64451E63
:10495000AC45C3E91177DF6313D0451CAC4517D0D4
:10496000844581D10546002D3FF47EAF106CC16BAC
:1049700001F1010CC0F83CC01864936428461A4643
:10498000DEE700283FF470AF854253F80C2CEAD1E3
:10499000107900283FF468AF53641A64EEE771465B
:1049A00002222F46A64613E0CB6B0A635B011DBFB4
:1049B00003F6FF7002F1FF3303EB10331346C1E936
:1049C0000477C1E90D3351F84C0F5A1C0136C8B1B8
:1049D0000B79002BE8D10B690A63002B48D14C6995
:1049E0001046531E4863002C4BD004F6FF7C03EBAB
:1049F0001C33281A8B63C51851F84C0F5A1C01360A
:104A00000028E5D125493E22C1F8902C3F22013BE8
:104A1000C1F8942CC1F8A85C4022214DC1F8982C13
:104A20007446C1F8B46CC1F8A43C980F9A00C1F860
:104A30008C5C43B340F2FF15521940F10000520A5A
:104A400042EAC05202F14000024402EBC303C1F843
:104A5000A02C144AC1F89C0CC1F8AC4CC1F8B04C65
:104A6000D80D5C02C1F8883CC1F8804C5060FBE670
:104A700003F6FF7C4C69531E03EB1C304863002C8B
:104A8000B3D11346B5E70122DCE7074FABE603F0ED
:104A9000F1F80690EEE600BF5C410020982000206F
:104AA0000CC00708182D0020851F000800797047EA
:104AB0000079C0F34010704700794009704700BF8B
:104AC000704700BF704700BFD0ED007AD0ED036A99
:104AD00030EE677AE6EE877AB0EE670AC0ED007ACC
:104AE000704700BFD0ED017AF5EE407AF1EE10FA92
:104AF00005D19FED0C7AC7EE207AC0ED017A31EE38
:104B0000277AD0ED007A80ED021AC1EE076A30EE06
:104B1000677AC0ED036AE6EE877AB0EE670AC0ED09
:104B2000007A704783F9223E9FED047AC7EE007A3F
:104B300077EEA07A80EEA70A704700BF72C7D13D1A
:104B400000230360436080ED020A704790ED017A14
:104B5000D0ED036AD0ED027A30EE470AA6EE807AF5
:104B600090ED000A80ED017A37EE676AE6EE867A0C
:104B700037EEC07AC0ED027AA6EE870A80ED000A11
:104B8000704700BFD0ED056AD0ED017A90ED007A54
:104B900090ED066AD0ED025A90ED035A80ED050AB9
:104BA00066EEA77AC0ED066AE7EE007A90ED077A26
:104BB000E5EE867A90ED086AD0ED045A80ED087A29
:104BC000E5EE477AE5EEC67AB0EE670AC0ED077A01
:104BD000704700BFD0ED057A90ED006A90ED067A3F
:104BE000D0ED035AE6EE007A90ED016AF0EE406AED
:104BF000A6EE267AB0EE670AD0ED047A90ED026A4E
:104C000067EEC07AA5EEC07AE6EE267A80ED057AE8
:104C1000C0ED067A704700BF03685A1C0260197025
:104C2000704700BF03690133012B03611CD0D0ED35
:104C3000005AD0ED026A07EE903A30EE656AF8EE5F
:104C4000E77A86EE277A77EE257AB0EE667A30EE4E
:104C5000670AC0ED017AA6EE007AC0ED007A80ED19
:104C6000037A80ED027A7047002380ED010A80ED1F
:104C7000000A8360704700BF03685A1C0260197005
:104C8000704700BF024B186803681B68184700BFD5
:104C9000D8700020024A536823EA00005060704731
:104CA000D870002050F8043C012202770BB118386C
:104CB0001847704790F83420034602F0FF0012B105
:104CC000002283F8342070474FF48053838170476B
:104CD0004FF40063838170470120704701207047C3
:104CE0002DE9F84F6D4DD5F808C0A889B5F9169093
:104CF000B5F812E0C0EB2C1303FB03F4B5F9103048
:104D0000241303FB04F44000B5F90E30C0EBEC00B3
:104D100003FB00F0A41304EBE024B5F914306C623B
:104D20000F46A4F5FA31164683FB013281FB018C54
:104D300012034FEAE97B42EA13524FEA033A09FBB6
:104D40000CF308FB0B3BA9FB0839D9441B0A43EAC7
:104D5000096313EB0A0342EB292202F50042A3FB8D
:104D60000E390EFB029E4FEAEE734FEA6E0253EAD3
:104D70006E0E4FF0000000F08580B5F91C9009FB25
:104D80000CFEB5F91AC08CFB011C4FEAE97A4FEA18
:104D90004C4C08FB0AEE4CEAD13CA9FB08984904AC
:104DA00011EB0901F04448EB0C0C4018A96AC1F55D
:104DB0008019B5F9181009F0004E4FEAC978B8EB20
:104DC00000080CEBC1014EEA590E6EEB010E18EB18
:104DD000080C4EEB0E011CEB080C4EEB01014FEAE8
:104DE00081194FEA8C1049EA9C691CEB000C41EBDD
:104DF0000901890041EA9C714FEA8C0C1CEB080CFC
:104E00004EEB01014FEA8C00890010EB080041EAEB
:104E10009C714EEB010167F0C7F8B5F92220B5F996
:104E200020E0B5F91E504FEA6138430B43EAC14315
:104E300002FB08FC4FEAE27903FB09C9A2FB032C41
:104E4000CC4402FB08F803FB0C88A2FB032CC444EF
:104E5000520E42EACC12121841EB6C6C4FEAEE7320
:104E60000EFB01F103FB0011AEFB00300144DB0C33
:104E700043EA4133D0184CEBE141000A40EA0160BB
:104E800000EB05100FB1000A386026B104EB840472
:104E90008034241234600120BDE8F88FD8700020DF
:104EA00031B10A4BD3ED117AFDEEE77AC1ED007A0C
:104EB00052B1064B9FED067AD3ED127A67EE877AF0
:104EC000FDEEE77AC2ED007A01207047D87000202D
:104ED0000000C8422DE9F04F624D85B0B5F85A3058
:104EE000E86CB5F8588001911B02B5F85410B5F87C
:104EF0005660B5F85C40C01A67EB07074FEA014EF1
:104F0000A8FB001CB5F8523008FB07CCC90941EAE0
:104F10004C6111EB0E0193464FEAC332A6FB003EF3
:104F200006FB07EE4FEA132343EA0E634FEAEC1C3D
:104F30004CF1000C9B18A4FB002604FB07644FEA0D
:104F4000D25242EA44224FEA2E2E4FEAE4544EF166
:104F5000000E12F5FA6944F10006B9F5FA6F0294F1
:104F600076F10004039631DA029CA2FB02A602FB52
:104F700004F806EB48044FEA84084FEA8A0616EB69
:104F80000A0648EA9A7844EB08084FEA560A4AEAC1
:104F9000C87AB608344CB1EB0A0146EA88766CEB65
:104FA000680C9B1B039E6EEBA80EA1454FF0FF34CF
:104FB00076EB040426DB00FB07F7A0FB000202EB04
:104FC0004707C00F40EA4700B9EB0009019C84B1D4
:104FD000286EA0FB033200FB0E2E5B0D43EACE23AE
:104FE0005B1A4FEA6E5E6EEB0C0CDB0B43EA4C4334
:104FF0002360BBF1000F01D0CBF80090012005B079
:10500000BDE8F08F40F6AC56029C921944F10004C2
:1050100002FB04F4A2FB028202EB4404E6004FEA26
:10502000C802B8EB020246EA587664EB060651184D
:105030004CEB060C18EB080644EB040A16EB0806CA
:1050400044EB0A0A4FEA8A0A4AEA967AB600B6EBB5
:1050500008026AEB0404520842EAC4729B1A6EEB1F
:10506000640EA8E7D870002024FAFFFF01207047E3
:105070000C4B0D481B6810B4446E1B1BFA2B09D84F
:1050800009B1836E0B604AB1C36E5DF8044B1360C7
:105090000120704700205DF8044B704701205DF847
:1050A000044B704754350020D8700020034B002279
:1050B000C3E91C22C3E91E2201207047D8700020DA
:1050C000094B0A4A1B68D16F5B1AFA2B0AD810B435
:1050D000D2E91C41936FC486018743875DF8044B76
:1050E000012070470020704754350020D870002000
:1050F000004870471412002070B5224E224C3546ED
:105100003622002104F180006CF059FF55F8103F61
:1051100000209847336BC4F8B850984783683BB376
:1051200004F1800206889446104600210578032D7C
:1051300000F106001ED001310929F7D1701E80B29E
:1051400000231178022902F1060209D00133092B4C
:10515000F7D1D4F8BC30082B0AD05A1CC4F8BC20B4
:10516000062202FB03C30221002219705A80988094
:10517000012070BD062303FB0141B1F88200013814
:1051800080B2DDE714120020D87000202DE9F04134
:105190000C4E356873691D4011D0DFF82C80012753
:1051A000B5FA85F4C4F11F0408EB840307FA04F48C
:1051B000D3F8C00003689847A5437461F0D1BDE8F7
:1051C000F08100BF003C0140D870002010B54D4C6C
:1051D00094F80031C0B223B9EE283FD0BB2848D0A4
:1051E00010BD494AD4F804111268521A0A2A30D85C
:1051F000012B12D194F8083123B984F80C0184F8FA
:10520000003110BD012BEBD10022022384F82201D2
:1052100084F8232184F8003110BD022BE0D194F8EA
:10522000233194F82221E1180133DBB29A4281F84C
:105230000C0184F82331D3D194F824310022012BBE
:1052400084F800212ED0022B1DD0002384F82431B5
:1052500010BD0023EE2884F80031BFD12A4B012273
:105260001968C4F80411002384F8002184F8083177
:1052700010BD254A01231268C4F8042184F80031C6
:1052800084F8083110BD94F80C31204AC3F3810131
:1052900003F003001172C3F301119B095072D17125
:1052A0009371D2E7B4F90E31DFED195A9FED195A17
:1052B00007EE103AB4F91031B8EEC77A07EE903A1B
:1052C000B4F90C31C7EE256A06EE103AF8EEE77A2B
:1052D000B8EEC66A87EE857A0C4BC6EE257AFDEEEF
:1052E000E66ABDEEC77A16EE902AFDEEE77A1A80DE
:1052F00017EE102A5A8017EE902A9A802EF030FC72
:10530000A3E700BFD8700020543500200000001033
:10531000CDCCCC3FCDCCCCBF38B51446002944D041
:10532000344B9FED356AD3ED4A7AB3F9402193EDC2
:105330004C0AB8EEE77AD3ED517AC7EE066A0D460D
:1053400004EE902AB3F93C21F8EEE77A05EE902AB4
:10535000B3F93E2187EE864AF8EEE44A05EE102ABC
:10536000F8EEE55AB3F93A21D3ED4D7AB3F9383175
:10537000E6EEA45A06EE102AB8EEE77AB8EEC55A61
:10538000B8EEC66AA6EEA57AA6EE856A07EE903A52
:10539000B8EEC00AF8EEE77AA6EE870AE6EE867A5D
:1053A000A4EE270A69F0E4FB28600CB3114BDFED93
:1053B000125A93ED517AB3F92E21B3F92C319FEDA6
:1053C0000F0AB8EEC76A07EE902A86EE257A06EE37
:1053D000903AF8EEE77AF8EEE66A67EE277AB6EEEC
:1053E000006AE6EE867A27EE800A69F0C1FB20604B
:1053F000012038BDD87000200000F04A0000C842EB
:10540000234B244A30B5D3F8484194F91030A168B1
:1054100003EB830302EB830383B08A078DF8070055
:10542000586B0AD501230DF10702002165F02AFE11
:10543000A3689B0714D503B030BD636913B11A6824
:105440009B885383144B15491A68154B4D68D2003D
:10545000A3FB023292094B685B1B9A42FBD2E1E745
:105460000D4B0E491A680E4B4FF4FA7000FB02F216
:10547000A3FB0232486892094B681B1A9A42FBD27E
:105480006369002BD7D01A689B88138303B030BDA3
:10549000D8700020141200207C360020001000E09C
:1054A000D34D621070B52B4C94F84C3182B023B9B7
:1054B000012084F84C3102B070BDD4F84851264A1E
:1054C00095F91030A96803EB830302EB83030522EF
:1054D000ADF800208A07586B11D502236A4601A94E
:1054E00065F0D0FDAB689B071CD59DF8053003F037
:1054F000010383F0010084F84C3102B070BD6B6988
:1055000013B11A689B885383144B15491A68154BBD
:105510004E68D200A3FB023292094B689B1B9A4251
:10552000FBD2DAE70D4B0E491A680E4B48684FF470
:10553000FA7606FB02F2A3FB023292094B681B1AB1
:105540009A42FBD26B69002BCFD01A689B881383D9
:10555000CBE700BFD8700020141200207C3600205A
:10556000001000E0D34D62102DE9F04383B0002815
:1055700061D1334DD5F8506195F84C31314F324CF3
:10558000DFF8D08033B900230120C5F8503103B0D3
:10559000BDE8F083D5F8489199F91030D9F8082082
:1055A00003EB830307EB830305219207586BADF8E8
:1055B000001018D502236A4601A965F063FDD9F8E9
:1055C00008309B0721D59DF8053003F0010385F8CD
:1055D0004C31002BD7D01D4A12689642D2D80020F9
:1055E00003B0BDE8F083D9F8143013B11A689B8872
:1055F0005383174B61681A68D200A8FB02329209E4
:1056000063685B1A9A42FBD2D4E7114B61681A684F
:105610004FF4FA7303FB02F2A8FB023292096368AB
:105620005B1A9A42FBD2D9F81430002BCBD01A68FF
:105630009B881383C7E7054B014D1E6806449BE713
:10564000D870002014120020001000E05435002013
:105650007C360020D34D6210F0B5404C83B094F8F6
:105660005421D8250021034600958DF8041082B1FD
:10567000020C050E8DF8022008461A0A8DF801501A
:105680008DF803208DF80430FFF76EFF90BB03B058
:10569000F0BD050C010A10468DF801508DF802107E
:1056A0008DF80330FFF760FF0028F0D00620FFF7E9
:1056B000A7FE0123D4F8485184F84C31042395F90E
:1056C0001020274902EB820201EB8202A968506B8D
:1056D0008A0719D56A46002165F0D4FCAB689B07A0
:1056E00025D5204B1B6803F59C530833C4F8503173
:1056F00003B0F0BD0620FFF783FE012384F84C3190
:10570000D4F848510523DAE76A6912B11168928822
:105710004A83154A154E1168154A7768C900A2FBDD
:10572000012189097268D21B9142FBD2D2E70E4B4C
:105730000E491A680E4B48684FF4FA7606FB02F2DF
:10574000A3FB023292094B681B1A9A42FBD26B6987
:10575000002BC6D01A689B881383C2E7D87000203C
:1057600014120020543500207C360020001000E088
:10577000D34D621010B50020FFF7F6FE00B910BD42
:10578000084C0620FFF73CFE0123C72084F84C316B
:10579000FFF736FE044B1B6803F5A4430833C4F837
:1057A000503110BDD87000205435002070B588B03D
:1057B00002260096204ECDF80CD0154696F85421BE
:1057C000002304468DF804300293AAB1CDE90615F2
:1057D00005930522030E8DF8013004920DF10203AA
:1057E000220C1A70220A5A7000209C70FFF7BCFE2F
:1057F00050B9204608B070BDCDE9052104220795B7
:105800000DF101030492EBE70620FFF7F9FDD6F84E
:105810004801012386F84C310379022B08D0074B4D
:105820001B682C4406332046C6F8503108B070BDC2
:1058300002A965F077FCF2E7D8700020543500200B
:1058400070B588B0032600961A4ECDF80CD01446D9
:1058500096F85421002503468DF804500295A2B114
:10586000CDE90654020E059105218DF80120049121
:105870000DF10202190C1170190A51700020937079
:10588000FFF772FE48B908B070BDCDE905120421DA
:1058900007940DF101020491ECE7D6F84801037971
:1058A000022B18BF2046EED102A965F03BFC204632
:1058B000E9E700BFD870002028B30368124A30B56A
:1058C00003F13F4303F57E039B0A054683B00C4674
:1058D000D05C62F02BFBA988009104F00303C4F3B1
:1058E00081028DF8043028688DF80520C4F3001378
:1058F0006946C4F341148DF806308DF80740FDF772
:10590000B3F803B030BD7047C0210708F8B503688D
:1059100004469869002871D040F615030021C38021
:105920000172FFF7C9FF2268444B9269A361002A04
:1059300064D09388B3FA83F3202BC3F11F0C50D0AB
:1059400012683F493F4D0CF0FC0E0EF1804E0EF5F3
:105950009C3E02F13F420CF0030002F57E02DEF8AD
:10596000086080000F27C2F38722824007FA00F008
:1059700026EA000001EB8C0604F11807C6F8C07097
:10598000CEF80800DEF808002F4E15F80CC00243D0
:10599000CEF808204FF000402C4A20FA03F3536160
:1059A000106820EA03001060506820EA030050608D
:1059B000D6F8000C1843C6F8000C906820EA0300E3
:1059C0009060D06820EA0300D060D6F8082C6144CB
:1059D0001343C6F8083C91F85831042B0FD82368BC
:1059E0009A695AB193884FF00042B3FA83F332FABE
:1059F00003F303D015490A6813430B60F8BD6544EF
:105A0000042295F9103081F85821002B2A7C0DDBF7
:105A10000F480121C51802F01F025B0901FA02F2CA
:105A2000402185F8001340F82320D8E7094B02F005
:105A30000F02134440221A76D1E700BFA54C00089C
:105A4000D8700020F82D070800300140003C0140CC
:105A500000E100E0FCEC00E082B08DED010A01986D
:105A600002B07047C31783EA400070479FED087A81
:105A7000C0ED020AC7EE007A0023036030EEA77A79
:105A8000C0ED017AC0EE877AC0ED037A704700BF9F
:105A900083F9223E80ED010A704700BF90ED017A44
:105AA000D0ED007AC0ED020A30EE877AC0EE876A48
:105AB00030EE677AE6EE877AB0EE670AC0ED007ADC
:105AC000704700BF80ED000A704700BF9FED047A69
:105AD000C7EE007A77EEA07A80EEA70A704700BF83
:105AE0004E2DA63D002303604360836080ED030AD2
:105AF000704700BFF5EEC00AF1EE10FA06DCF0EEDA
:105B0000407A80ED000AB0EE670A704760EE810AC5
:105B100090ED007A77EE607AF4EEC07AF1EE10FA4A
:105B20000ADC77EE200AF4EEC00AF1EE10FA8CBF20
:105B3000F0EE407AF0EE607AC0ED007AB0EE670ADF
:105B4000704700BFB4EEE00AF1EE10FA07D4B4EEED
:105B5000C10AF1EE10FA88BFB0EE410A7047B0EE0C
:105B6000600A7047894BB3FBF2F399420DD30023CF
:105B70004FF07E52026043608360C3600361002384
:105B8000836143610362C361704707EE902ADFEDD2
:105B9000806AB8EE677A07EE901A27EE267AF8EE5A
:105BA000677A27EE277AFDEEC77A17EE903A203310
:105BB000402B00F2DA80DFED777AB4EEE77AF1EE8F
:105BC00010FAF0EE477A0CDDDFED735A9FED736A41
:105BD000F0EE676AF4EEC66AF1EE10FA77EEE57A57
:105BE000F6DCDFED6F6AF4EEE67AF1EE10FA0CD532
:105BF000DFED695A9FED6B6AF0EE676AF4EEC66AF4
:105C0000F1EE10FA77EEA57AF6D4DFED676AF4EEDE
:105C1000E67AF1EE10FA00F39C80DFED646AF4EEB0
:105C2000E67AF1EE10FA44BFDFED5D6A76EEE77AD0
:105C300027EEA76ADFED5E5ADFED5E6A9FED5E5AE2
:105C4000DFED5E4AE6EE256ADFED5D5AA6EE265AE6
:105C500027EE864AE6EE055AF7EE006AE4EE257A6C
:105C6000F0EE665AE7EEA45AE7EEE46A86EEA54A3D
:105C7000DFED4D6A77EE267ABDEEE76A16EE103A52
:105C80002033402B6AD8B4EEE67AF1EE10FA0CDD40
:105C90009FED416ADFED416AB0EE677AB4EEE67AD5
:105CA000F1EE10FA77EEC67AF6DC9FED3D7AF4EE6F
:105CB000C77AF1EE10FA0CD59FED376ADFED396A3D
:105CC000B0EE677AB4EEE67AF1EE10FA77EE867A05
:105CD000F6D49FED357AF4EEC77AF1EE10FA49DD8D
:105CE0009FED2C7A77EE677A67EEA76A9FED306AB0
:105CF0009FED307ADFED304A9FED315AA6EE867A7D
:105D000027EEA63AE6EE874AB7EE006AA6EEA45A58
:105D1000B6EE007AE3EE057AF8EE003A36EE676A00
:105D200067EEA37A26EE077AB7EE005AC5EE256A2B
:105D300080ED044A26EE877A26EE866A66EEA77A1A
:105D400080ED007A80ED016A80ED027AC0ED037A81
:105D500015E7DFED106A76EEE77A69E7DFED197A8D
:105D6000B6EE007AB7EE006ADEE7B7EE004AF0EE74
:105D7000445A7DE79FED0D7AF4EEC77AF1EE10FA02
:105D800044BF9FED077A77EE677AADE720A1070061
:105D900027D4D236DB0F4940DB0FC940E4CB164194
:105DA000DB0F49C0E4CB16C1DB0FC93FDB0FC9BF16
:105DB0009A7C2E36FAAF4FB93587083CF304353F4D
:105DC000A4AA2ABE00000000FDEEC07A17EE903AA9
:105DD0002033402B53D8DFED2B7AB4EEE70AF1EEF7
:105DE00010FA0CDDDFED286A9FED287AF0EE407A9C
:105DF000F4EEC77AF1EE10FA30EE660AF6DCDFED6B
:105E0000247AB4EEE70AF1EE10FA0CD5DFED1E6A43
:105E10009FED207AF0EE407AF4EEC77AF1EE10FAB8
:105E200030EE260AF6D4DFED1C7AB4EEE70AF1EE86
:105E300010FA1FDCDFED197AB4EEE70AF1EE10FA82
:105E400044BFDFED137A37EEC00A60EE007A9FEDB3
:105E5000147A9FED146ADFED146AA7EE876A9FED4E
:105E6000137AE7EE866A60EE275AA7EEA67AA5EEC9
:105E7000870A7047DFED037A37EEC00AE5E79FED4A
:105E80000C0A7047DB0F4940DB0FC940E4CB1641D9
:105E9000DB0F49C0E4CB16C1DB0FC93FDB0FC9BF25
:105EA0009A7C2E36FAAF4FB93587083CA4AA2ABE91
:105EB000000000009FED307A70EE077AFDEEE76A91
:105EC00016EE903A2033402B53D8B4EEC70AF1EEC9
:105ED00010FA0CDD9FED296ADFED296AB0EE677AD2
:105EE000B4EEE67AF1EE10FA77EEC67AF6DC9FEDC4
:105EF000257AF4EEC77AF1EE10FA0CD59FED1F6A01
:105F0000DFED216AB0EE677AB4EEE67AF1EE10FAD0
:105F100077EE867AF6D49FED187AF4EEC77AF1EE32
:105F200010FA21DC9FED197AF4EEC77AF1EE10FA3F
:105F300044BF9FED147A77EE677A27EEA77ADFEDFC
:105F4000146ADFED145A9FED146AE7EE265ADFED6E
:105F5000136AA7EE256A27EE875AE7EE066AE5EE92
:105F6000267AB0EE670A70479FED0D7A77EE677A72
:105F7000E3E79FED0C0A7047DB0FC93FDB0FC94019
:105F8000E4CB1641DB0F49C0E4CB16C1DB0FC9BF20
:105F90009A7C2E36FAAF4FB93587083CA4AA2ABEA0
:105FA000DB0F494000000000B5EE400AF1EE10FAA8
:105FB00025D007EE902AF8EE670ADFED117A08B5D2
:105FC000034660EEA70A0846F0EE406A13B9FFF7F1
:105FD0004DFD0CE0022B06D0032B08D1FFF776FD18
:105FE000BDE808407EE5FEF79FFDFEF7A9FDFCEE4B
:105FF000E66A16EE903A99B2BDE80840B2E57047FD
:10600000BD378635B5EE400AF1EE10FA01D1044BEA
:1060100003E003280CBF034B034B0B60704700BF2A
:10602000C14A00084D4B0008D54B000890ED0E7A90
:10603000B5EEC07AF1EE10FA00F3988030EE607A97
:10604000D0ED015A037867EE255A002B5BD101F0A1
:106050000103D0ED117A002B61D077EE677AF0EE74
:10606000470A87EE816AD0ED0F6AC0ED110AF5EE9E
:10607000C06AF1EE10FA57DCD0ED037A26EE276AFB
:10608000D0ED056A90ED105A60EE266A76EE857ABC
:1060900077EEA57A77EE867AF4EEE71AF1EE10FA4B
:1060A00000F38480B4EEE72AF1EE10FA8CBFB0EE74
:1060B000670AB0EE420A70EE677A90ED044AD0EDBE
:1060C000024AC0ED135A67EE847A4A07E7EE247A53
:1060D000B0EE457AA1EE277A80ED125A80ED146A6F
:1060E000C0ED156A80ED160A08D5F0EEC77AF0EE1D
:1060F000C56AF4EEE67AF1EE10FA6BD580ED107A0F
:106100000B0756D4704711F001034FF000020CBF8B
:10611000F0EE607AF0EE477A0270002B9DD177EEB8
:10612000E07A87EE816A9EE7D0ED0B7AD0ED034AE4
:10613000F5EE407AF1EE10FA05D19FED285AC5EE42
:10614000267AC0ED0B7A71EE276AD0ED0A7A80EDDF
:106150000C1A81EE265A36EE676A80ED0D5AE5EE8E
:10616000067A24EEA76AC0ED0A7A89E7D0ED077AAD
:10617000F5EE407AF1EE10FA70EE606A05D19FED0F
:10618000176AC6EE077AC0ED077A71EE277A90EDAE
:10619000067A80ED081A81EE276A76EEC77A80EDDE
:1061A000096AA6EE277A80ED067A49E7B0EE610A21
:1061B00081E7F4EEC71AF1EE10FA08DCB4EEC72A54
:1061C000F1EE10FA8CBFF0EE471AF0EE421AC0ED75
:1061D000101A7047B0EE457A92E700BF83F9223E6D
:1061E000002301220270C364836403650364436473
:1061F0004365836283657047DFED1B7A80ED010A9A
:10620000F4EEE70AF1EE10FAC0ED020A80ED031A8F
:10621000C0ED051A12DC0023836003610023012214
:1062200080ED0F2AC0ED0E2A0270C36483640365FB
:10623000036443644365836283657047B4EEE70A91
:10624000F1EE10FA0CDD81EE007AC0EE207AF0EE6D
:10625000006A77EE877A86EEA77A80ED047ADDE72A
:1062600000230361DAE700BFBD378635F0EEC07A60
:10627000B0EEE07AB4EEE77AF1EE10FAB4BFB0EE29
:10628000676AB0EE476AB5EE406AF1EE10FA46D0A2
:10629000B4EEE77AF1EE10FA8CBFF0EE675AF0EE4A
:1062A000475AC5EE866ADFED1F2ADFED1F3ADFEDA4
:1062B0001F4A9FED1F5A9FED1F3A9FED1F4ADFEDCA
:1062C0001F5AE6EEE23AA6EE834AE6EEA34AB7EE9E
:1062D000006AA6EEA45AA6EE846AE6EE855AC5EEDA
:1062E000866AB4EEE77AF1EE10FA48BFDFED147A71
:1062F000F5EEC00A48BF77EEE66AF1EE10FA48BF45
:10630000DFED107AB5EEC00A48BF77EEE66AF1EE2F
:1063100010FA48BFF1EE666AB0EE660A7047DFED2C
:10632000076ADEE739094E3DE3B59E3E88FA163E20
:1063300045FE7F3F99FB243F69A2163EA7DFA834A4
:10634000DB0FC93FDB0F4940B7EE007AF0EEC07AB1
:10635000F4EEC77AF1EE10FA77EE676A1DD8B1EE67
:10636000E67ADFED0F5ADFED0F6A9FED0F6AE7EE79
:10637000A65ADFED0E6AA7EEA56AE7EE866A67EE1B
:10638000266AB5EEC00AF1EE10FA44BF9FED087A16
:1063900077EE666AB0EE660A7047DFED066AF0E7F0
:1063A0002716983D306E99BC843459BEA40DC93F60
:1063B000DB0F494000000000B0FBF1F301FB1303C9
:1063C00008463BB11946B0FBF1F301FB1303084645
:1063D000002BF7D1704700BF44F25063984203DDB1
:1063E000A0F50C40A0387047034B9842BCBF00F5A5
:1063F0000C40A030704700BFB0B9FFFF48F6A04383
:10640000984203DDA0F50C40A03870470028B8BFC3
:10641000C018704780EAE073A3EBE0738B4203DBA4
:10642000002803DD401A704700207047FDD0084463
:10643000704700BF884203DB9042A8BF10467047F8
:106440000846704700230361704700BF036970B5B9
:106450000446A3B1214DD4ED067A77EE807A01335C
:1064600004F11C062361C4ED067A3046FEF7DAFB20
:1064700062682B689B1AA268934207D870BD426875
:10648000164D002AE7D12A684260E4E7E06A94EDFD
:106490000A0A64F0EDF8D4ED057AB4EEE70AF1EEFD
:1064A00010FA04DD237B7BB10323237070BDD4ED90
:1064B000047AD4ED066AF8EE677A022386EEA77AAC
:1064C000237084ED067A70BD296861600022236123
:1064D000A2613046BDE87040B4E700BF54350020EB
:1064E0002DE9F04100F11C0604463246054600F154
:1064F000640752ED017AB1EC010A77EE807A10461A
:1065000042ED017A1832FEF78DFB9742F1D12369F3
:10651000264F6268013323613B689B1AA26893424D
:1065200029D904F14808E86A95ED0A0A64F0A0F850
:10653000D4ED057AB4EEE70AF1EE10FA05F118058C
:106540001BDCA845EFD1D4ED047AD4ED066A94EDB6
:106550000C7AD4ED125AF8EE677A022386EEA76A17
:106560002370C7EE276A85EEA77A84ED066AC4ED2C
:106570000C6A84ED127ABDE8F081237B1BB1032302
:106580002370BDE8F08139682361002230466160E4
:10659000A261FFF757FF04F134002263FFF752FFB7
:1065A000A26404F14C00BDE8F0414BE754350020F3
:1065B00010B4019C401AA4EB030C00FB0CFC511A14
:1065C0005DF8044B9CFBF1FC0CEB0300704700BF33
:1065D00030EE600A32EE612A71EE600A22EE002A85
:1065E00082EE200A30EE210A704700BFD1ED007A1A
:1065F000DFEDE36A37EEA67ABDEEC76A16EE103A13
:106600002033402B00F25D82F4EEE67AF1EE10FAD0
:106610000CDDDFEDDC5A9FEDDC6AF0EE476AF4EE4C
:10662000C66AF1EE10FA37EE657AF6DCDFEDE26A63
:10663000B4EEE67AF1EE10FA0CD5DFEDD25A9FED0A
:10664000D56AF0EE476AF4EEC66AF1EE10FA37EE5C
:10665000257AF6D4DFEDCA6AB4EEE67AF1EE10FAE6
:1066600000F30D82DFEDD36AB4EEE67AF1EE10FAB4
:1066700044BFDFEDD16A36EEC77A67EE076A9FED59
:10668000C76A9FEDC75ADFEDC75AA6EE865A9FED3F
:10669000C66AE6EE855A27EE264AA6EEA56AA4EE5D
:1066A000067AF0EE474ABDEEE77A17EE103A20334D
:1066B000402B00F203829FEDBD7AF4EEC77AF1EE33
:1066C00010FA0CDD9FEDAF6A9FEDAF7AF0EE676ACE
:1066D000F4EEC76AF1EE10FA77EEC67AF6DC9FEDBB
:1066E000B67AF4EEC77AF1EE10FA0CD59FEDA56AF2
:1066F0009FEDA87AF0EE676AF4EEC76AF1EE10FA41
:1067000077EE867AF6D49FED9E7AF4EEC77AF1EEB4
:1067100010FA40F309829FEDA57A77EE677A27EEAB
:10672000A77ADFED9E6ADFED9E5A9FED9E6AE7EE47
:10673000265ADFED9D6AA7EE256A27EE874AE7EE27
:10674000066AE4EE267AB0EE675A91ED017ADFED43
:106750008C7A77EE276ABDEEE66A16EE103A2033A1
:10676000402B00F2A481B4EEE77AF1EE10FA0CDDD2
:10677000DFED845ADFED847AB0EE666AB4EEE76A44
:10678000F1EE10FA76EEE56AF6DCDFED8B7AF4EEE8
:10679000E76AF1EE10FA0CD5DFED7A5ADFED7D7A7B
:1067A000B0EE666AB4EEE76AF1EE10FA76EEA56A2C
:1067B000F6D4DFED737AF4EEE76AF1EE10FA40F307
:1067C000A781DFED7A7A77EEE66A66EEA67ADFEDEC
:1067D000735A9FED734A9FED736AA7EEA54ADFEDEA
:1067E000725AA7EE846A66EEA73AE7EE865AE3EE9F
:1067F000A56A66EEC52A24EEA63AB0EE666AFDEEFC
:10680000C77A17EE903A2033402B00F24D81DFED2E
:10681000677AB4EEE77AF1EE10FA0CDDDFED595A43
:10682000DFED597AF0EE476AF4EEE76AF1EE10FA1E
:1068300037EE657AF6DCDFED607AB4EEE77AF1EEFA
:1068400010FA0CD5DFED4F5ADFED527AF0EE476AC1
:10685000F4EEE76AF1EE10FA37EE257AF6D4DFEDC2
:10686000487AB4EEE77AF1EE10FA40F34581DFEDB5
:106870004F7A37EEC77A67EE077ADFED485A9FED19
:10688000484ADFED486AA7EEA54ADFED475AE7EE32
:10689000846A67EE273AE7EEA65AA3EEA57AF0EEF1
:1068A000476AD1ED027ADFED365A37EEA57ABDEEB2
:1068B000C74A14EE103A2033402B00F2EA80F4EE7F
:1068C000E57AF1EE10FA0CDDDFED2E3A9FED2E4A5F
:1068D000F0EE475AF4EEC45AF1EE10FA37EE637A4E
:1068E000F6DCDFED355AB4EEE57AF1EE10FA0CD5B0
:1068F000DFED243A9FED274AF0EE475AF4EEC45AF2
:10690000F1EE10FA37EE237AF6D4DFED1D5AB4EE2D
:10691000E57AF1EE10FA40F3E380DFED245A35EE2C
:10692000C77A67EE075A9FED1D4A9FED1D2ADFEDDE
:106930001D3AA5EE842A9FED1C4AE5EE823A67EEE9
:10694000251AA5EEA34AA1EE847A25EE072A64EE65
:10695000871A26EE821A26EE077A26EEA10AFDEEA7
:10696000E75A15EE903A2033402B00F28D80DFED90
:106970000F5AF4EEE57AF1EE10FA2CDD1EE000BFBE
:10698000DB0FC93FDB0FC940E4CB1641E4CB164116
:10699000DB0FC940E4CB16C1DB0FC93F9A7C2E3612
:1069A000FAAF4FB93587083CA4AA2ABEDB0F49408D
:1069B00000000000DB0FC9BFDB0F49C05FED0C3AE0
:1069C0001FED0E4AF0EE675AF4EEC45AF1EE10FADB
:1069D00077EEE37AF6DC5FED085AF4EEE57AF1EE55
:1069E00010FA0CD55FED163A1FED164AF0EE675A15
:1069F000F4EEC45AF1EE10FA77EEA37AF6D45FED16
:106A00001A5AF4EEE57AF1EE10FA5DDD5FED195AEF
:106A100075EEE77A27EEA74A5FED205A5FED203A40
:106A20005FED200AE4EE253A67EE845AE4EE230A8D
:106A30005FED233AE4EE203AE5EEA37A64EEA74A4E
:106A400065EE275AA6EEA42AE6EEE51A67EEC67AA8
:106A500031EE241A75EEC05A80ED007AC0ED017A4D
:106A6000C0ED026A80ED031AC0ED041AC0ED052ADC
:106A7000C0ED065A80ED072A80ED083A70475FEDB9
:106A8000356A36EEC77AF8E55FED375AF0EE657A8B
:106A9000E0E71FED392AF0EE421AB0EE420AB0EEFE
:106AA000421AB0EE427A5AE75FED3F6AF9E61FED0F
:106AB000403AF0EE432AB0EE436AA0E61FED445A96
:106AC00043E65FED454AEEE55FED465AF4EEE57AC2
:106AD000F1EE10FA44BF5FED485A75EEE77A99E798
:106AE0005FED4C5AB4EEE57AF1EE10FA44BF5FED7B
:106AF0004E5A35EEC77A14E75FED527AB4EEE77A74
:106B0000F1EE10FA44BF5FED547A37EEC77AB2E681
:106B10005FED587AF4EEE76AF1EE10FA44BF5FEDEC
:106B20005A7A77EEE66A50E61FED5E7AF4EEC77A9F
:106B3000F1EE10FA44BF1FED607A77EE677AEEE56A
:106B40000023036143618361C361036003624362A5
:106B50008362C3624360036343638363C36383608D
:106B6000036443648364C364C3607047D1ED017AF6
:106B700091ED007AD0ED044A90ED065AD0ED075A17
:106B800090ED050AD0ED080AD0ED0A1AD0ED0C2AD6
:106B900090ED0D3AD0ED0E3A90ED091A90ED0B2ADA
:106BA000F8EEE76AD1ED027AB8EEC77AF8EEE77A46
:106BB00026EEA64AA7EE275AE7EE074AB0EE446A49
:106BC00075EE875AA7EE076AE7EE272AE7EEA73A9F
:106BD000A7EE260AE7EE260AE6EEA71AA6EEA73AE1
:106BE00031EE041AC0ED044A90ED0F4AD0ED104A80
:106BF00080ED065AC0ED075A90ED115AD0ED125AA9
:106C0000C0ED0E3AA7EEA76A34EE274A74EE874A23
:106C100075EEA75A35EE265A32EE262A80ED0F4A37
:106C2000C0ED104A80ED115A80ED050AC0ED080A4A
:106C300080ED091AC0ED0A1A80ED0B2AC0ED0C2A6E
:106C400080ED0D3AC0ED125A90ED004A90ED025AD7
:106C5000D0ED014AD0ED133AD0ED035AA7EE064A23
:106C6000B0EE457AA7EE867AE6EE864AF7EE007A2F
:106C700073EEA77A35EE866AC0ED137A80ED004A8E
:106C8000C0ED014A80ED027A80ED036A704700BFD3
:106C900010B50024034684468646002C00F00E8181
:106CA000DEED006A9CED007AD3ED007AE6EEC77A5D
:106CB000012CC3ED007A00F01081DEED016A9CED3D
:106CC000047AE6EEC77A032CC3ED007A6CD1DEEDD0
:106CD000026A9CED087AE6EEC77AC3ED007AD2ED3F
:106CE000007A90ED085AD0ED0C5AD0ED044A92ED9E
:106CF000017AD2ED026A92ED036AA7EEE47AE7EE3A
:106D0000C56AA7EEE56A90ED095AD0ED0D5AE7EE97
:106D1000456AA5EEC76AD0ED0E5AA5EEE66A81ED8A
:106D2000036A90ED0F5AC1ED026AC6EE055AC1ED35
:106D3000035A90ED0B6AE5EEC66AC1ED026A90ED6A
:106D40000A5A81ED017A86EE856A81ED026AD0EDFC
:106D5000066AA6EE667A81ED017AD0ED076AA5EEA5
:106D6000E67A81ED017A90ED055AC1ED007AC7EE21
:106D7000056AC1ED016A90ED017AE7EE667AC1ED30
:106D8000007A90ED027AE7EE467AC1ED007A90ED56
:106D9000037AE7EE657AC1ED007AD0ED006A87EEFE
:106DA000A67A81ED007A10BD9EED007ADCED016AD5
:106DB000D3ED017AE7EE667A022CB1EE476AC3EDB5
:106DC000017ADEED016A9CED057AE6EEC77AC3ED45
:106DD000017A40F0B580DEED046A9CED007AD3EDD7
:106DE000047AE6EEC77A012CC3ED047A40F288807B
:106DF000DEED056A9CED047AE6EEC77A032CC3ED5E
:106E0000047A40F08480DCED086A9EED066A93ED1A
:106E1000007AE6EE667AC7EE876AC3ED046A9EEDF5
:106E2000086ADCED006AD3ED087AE6EE667A012C9A
:106E3000C3ED087A74D99EED096ADCED046AE6EECA
:106E4000667A032CC3ED087A07D19EED0A6ADCED61
:106E5000086AE6EE667AC3ED087A93ED086AD3ED28
:106E60000C7AC6EE076A032CC3ED086A9CED006A33
:106E7000DEED0C6AE6EE667AC3ED0C7A9CED046AF0
:106E8000DEED0D6AE6EE667AC3ED0C7A07D19EED73
:106E90000E6ADCED086AE6EE667AC3ED0C7AD3ED95
:106EA0000C6AC6EE877AC3ED0C7A013414330EF106
:106EB000100E0CF1040C002C7FF4F2AED3ED047A2A
:106EC00093ED007A93ED086AC7EE876AC6EE077AFB
:106ED000C3ED046AC3ED087AE1E7DEED006A9CEDDC
:106EE000016A93ED017AD3ED027AA6EEC67A83EDBC
:106EF000017A9CED027AE7EE667AC3ED027A6AE7E0
:106F000093ED007AC7EE876AC3ED046A87E793EDD5
:106F1000007AC7EE876A022CC3ED046AC5D07EE70B
:106F2000C7EE876AC3ED086ABFD09CED006ADEED4C
:106F30000C6AD3ED0C7AE6EE667AC3ED0C7AAEE716
:106F40009CED027AD3ED027AE6EE077A032CC3EDCC
:106F5000027ADCED066A9EED017AE6EEC77AC3EDB1
:106F6000027A7FF438AFDEED026A9CED0A7AE6EE33
:106F7000C77AC3ED027AB2E610B584B00C46024679
:106F800069461030FFF784FEDDED006A9DED017A61
:106F9000DDED027AB6EE006A66EE866A27EE067AC4
:106FA00067EE867A0120C4ED006A84ED017AC4EDB3
:106FB000027A04B010BD00BF20EE000AFEEE007A97
:106FC00060EE277A60EEA00A9FED020AC7EEA00AE3
:106FD00067F0B6BF54F82D4008B564F087FE07EEA1
:106FE000900AF5EEC07AF1EE10FAACBFB1EEE70A06
:106FF0009FED010A08BD00BF0000000060EEA00A7E
:10700000E0EE000AB1EEE00A704700BF21EE011A7F
:10701000A0EEA01AA0EE001AB1EEC10A704700BFA0
:107020002DE9F04F83B005469DF830400D9E01924A
:10703000002C14BF4FF030094FF020091C1E884669
:107040004ADB16F8010B014600286CD0002C65D0F5
:107050004FF0000A324601E0002C34D012F8013B18
:107060002746013C002BF7D1BAF1000F3CD1023F7B
:10707000002C65D0BA4645450AF1FF3A49462846F4
:1070800001D2019B9847BAF1FF3FF4D10D9A1078D5
:1070900023463C1B01469B4688B14FF0000A013352
:1070A0009F1B454506EB070B284601D2019B9847DD
:1070B00016F8011B0029F4D1BAF1000F18D1584677
:1070C00003B0BDE8F08FBAF1000F31D0014683461E
:1070D0000028F4D02346E2E716F8010B634258B3C8
:1070E0001C464FF0010AB5E7014683460028D6D179
:1070F000002C04F1FF36E2DD3446454506F1FF364B
:107100004946284601D2019B9847731CF5D10BF1E3
:10711000010BA344584603B0BDE8F08F2346A246B6
:107120004FF0FF34BBE7671EA346002CA2D1C6E791
:1071300023464FF0FF34ADE7E64383463446DCE7B1
:1071400023463C46A6E700BF0FB430B583B006AB7C
:107150000A4C53F8042B0193D4E9580160F0DAFF8C
:107160000546206803685B6998470028F9D02846DF
:1071700003B0BDE8304004B0704700BFD8700020B5
:107180000EB410B583B005AB044653F8042B074981
:10719000009301A8019460F0BDFF019B00221A70CA
:1071A00003B0BDE8104003B0704700BF794C000841
:1071B0000CB470B5334CD4F86831A4B0002B4AD06D
:1071C00094F8703199423ED82F4B304A1B68A2FB8D
:1071D000031292094FF47A7101FB123304A82C496F
:1071E000FFF7CEFF04AA29AB0244CDE902322949B8
:1071F000289A064603A860F08DFF039BD4F86851D7
:107200005A1C03920A221A70039B5A1C03920022F2
:107210001A702DB32B681B6A1BB128469847D4F807
:1072200068519DF8101049B10DF111042B682846E2
:107230001B68984714F8011B0029F7D124B0BDE85A
:10724000704002B07047D4F87421012303FA00F0B3
:107250001042B9D1F2E7D4F86C31002BB0D1EDE790
:10726000D4F86C31002BE9D030440222009204A9FA
:107270008218FD2032F098FE24B0BDE8704002B0C4
:10728000704700BFD870002054350020D34D6210E5
:1072900038C00708194C000830B54FF4004087B0DB
:1072A0002DF000F958B14FF4004104462DF0B0FC28
:1072B000022806D1226848F201039A4224D007B07E
:1072C00030BD00234FF46121022294F904008DE8BF
:1072D0000E001A464FF4004130F012FE1C4BC3F86A
:1072E00068010028EBD01B4A1B4B1C4C1C481D4955
:1072F0000091CDE90332CDE901041B4B1B4A022169
:107300000020FFF755FFDAE7114C00254FF400404D
:1073100084F80C545FF044FA0028D0D0D4F87831C7
:1073200083420AD0D4F8543283420BD0D4F830339D
:1073300098420AD0C4F86C51C1E704F5BC73C4F894
:107340006C31D0E704F51573F9E704F54C73F6E7F3
:10735000D87000205CC0070868C0070874C0070820
:1073600080C0070888C00708B0BE070844C00708E7
:1073700038B5174CD4F81054033005EB9003B3F52F
:10738000007F18D804EB810120F00302D1F8140C1F
:10739000C4F810341044C3F5007304F21444C1F867
:1073A000140C0C4A04EB85049B0004210020FFF719
:1073B000FFFE204638BD00210846074AFFF7F8FEC9
:1073C000064A1369002443F000731361204638BD58
:1073D000D870002094C00708B8C00708000000104B
:1073E00038B50568EB69044653B1987800B938BDE3
:1073F0009A88E281DA8822821B896382012038BD63
:107400000C211420FFF7B4FF0346E861EDE700BF4D
:107410002DE9F041944603EB43031CF8068B86B03C
:10742000144602EB430315464FFA88F69CF80070A9
:10743000A0EB070E821BBEF1000FB8BFCEF1000E0D
:10744000002AB8BF52429645B8BF65460CF1060CFB
:10745000B8BF7EB26345E9D1B0456F88A3F106029B
:1074600006D0BE46A24216D014F8068FB045F8D119
:10747000B4F80280CB1BA1EB080C002BB8BF5B4219
:10748000BCF1000FB8BFCCF1000C6345BE46E9DD8E
:1074900047462546E5E76B7904932B7903932B78D0
:1074A000064A0091CDE9013E032103460120FFF782
:1074B0007FFE284606B0BDE8F08100BFC8C00708BF
:1074C00003681A46591C016012F8021B02605878C2
:1074D00041EA0020704700BF02681146531C036058
:1074E00011F802CB0160D31C5178036093781B0420
:1074F00043EA0123111D0160D07843EA0C0343EAFB
:107500000060704712B370B50446864604E0981BCD
:1075100017D114EB0C0C15D01EF8013BA3F1410060
:10752000192811F8010BA0F1410598BF2033192D3E
:10753000A2EB0E0C00F12006E9D91B1A04D1002899
:10754000E7D170BD604670BD184670BD10467047EB
:1075500010B40288C378174CA2F5FA6202F0030156
:1075600040F2B55C9208013B0CFB0233827801EBE0
:107570004101013A02EB810204EB420102790C8BDA
:107580004179234403EB430302EBC30384790A4AA2
:107590000089C3EB031301EB8303C3EB0313224402
:1075A00002EB830200214FF47A73C2FB03015DF802
:1075B000044B7047F82D070880436D382DE9F041E2
:1075C00017461E4605464FF47A7200233846314668
:1075D00064F0EAFC4349444A014482FB0143C81772
:1075E0000B44C0EB631382FB03021A44D8173F4CD1
:1075F000C0EB621284FB02044FEAE27C3C48CCEB15
:10760000A40C80FB0C404FEAEC74C4EBE010C3EB1D
:107610000314A1EB8401A971C2EB0211A3EB810356
:107620006B710CEB4C03A2EBC30240F2B55303FBAE
:1076300010CCBCF5896F2A714FEA800043DA40F222
:10764000DA239C4546DCBCF5B77FB4BF002201229B
:10765000284B02EB420103EBC1034FEA4208DB8DEA
:1076600091B2254C08EB020E04EBCE0416344FF019
:107670000B0E01E034F8023D63451FDDBEF1010E43
:10768000F8D11C4B424403EBC2024FF0010E138BA6
:1076900085F802E000F5FA600CF1010C0844ACEB4F
:1076A000030C288085F803C04FF47A720023384613
:1076B000314664F079FC2A81BDE8F0810EF1010EBB
:1076C0005FFA8EFEE4E7032140F296530A464FF03C
:1076D0000608C6E7022140F229430A464FF0040893
:1076E000BFE700BF80BC92C789888888ABAAAA2A56
:1076F00073B06D16F82D0708102E070830B52E4D03
:1077000084468E460FCD8DB06C460FC40FCD0FC48E
:1077100095E80F001CF0030F84E80F000DD1274BF4
:10772000274A03FB0CF3B2EBB30F43D3254AB2EB6A
:10773000331F2CBF1D241C2400E01C240CF1FF333C
:10774000002B40F26D12194602FB0CF2B8BF0CF18F
:10775000020102EBA1021C491C4D019481FB0301B3
:10776000DB17A3EB61100244C3EBE1131A4425328B
:1077700085FB02301044D317C3EBA000C0EBC00060
:10778000ADF10403101A0DF1040C03EB8E0E01E0B1
:107790005CF8044F031985FB0320C218D817C0EB0F
:1077A000A200C0EBC000E645A3EB0000F0D1201A18
:1077B0000DB030BD1D24C1E7702E0708295C8FC2B3
:1077C000285C8F020AD7A3001F85EB5193244992AE
:1077D00008B50C4B53E9022352EA030C09D10023EC
:1077E00040F2011242808380837103800381184636
:1077F00008BD054909688A1843F10003FFF7DEFE5A
:10780000012008BD887D0020543500208842F0B555
:107810004FF0010461D301FB04F4B0FBF4FC8C4590
:10782000F9D284B3002A45D0002511E0BCF1090F3C
:107830002646CCBF372230229444B14283F800C0A0
:10784000744603F1010305F101051CD8B0FBFEFCF1
:10785000B4FBF1FE04FB1C00002DE7D1BCF1000FCE
:10786000E4DCA1420BD8B0FBFEFCBCF1000F744677
:107870000EFB1C00BEFBF1FED8DCA142F3D90CF1DB
:10788000300C03F801CB00221A70F0BDBCF1090FD7
:107890002646CCBF4FF0570E4FF0300EF444B142A5
:1078A00083F800C02C4603F1010302F10102EAD87B
:1078B000B0FBF5FCB4FBF1F504FB1C00002AE5D19C
:1078C000BCF1000FE2DCA142D9D8B0FBF5FC2C469C
:1078D00005FB1C00B5FBF1F5F2E78446002AA3D1B5
:1078E000E8E700BF002870B503DA2D2301F8013B5B
:1078F0004042092804464FF0010307DD03EB8303F0
:107900005B00B0FBF3F2092AF8D83BB3164D4FF0F9
:10791000000C0AE0092A8CBF572130210A44092BA8
:107920000EF8012B16D971460346A5FB0320B4FBC4
:10793000F3F25CEA02068E464FEAD00003FB1244E3
:107940000CF1010CE6D1092B01D9B446EBE730323A
:107950000EF8012B00238EF8003070BD8E460023F8
:107960008EF8003070BD00BFCDCCCCCC90422DE95C
:10797000F0410B46044615460AD2B0FBF5F6134A11
:1079800005FB16441846135D00F8013BBDE8F08185
:10799000B0FBF2F69642B6FBF2F706D20B4A05FBB5
:1079A0001767D15D03F8011BEAE7BA42B7FBF2F8AB
:1079B00007D9064A05FB187812F8081003F8011BCE
:1079C000EDE74046FFF7D2FF0346F2E704C10708A0
:1079D000B5EEC00ADFED347AF1EE10FACCBF30EE2E
:1079E000270A30EE670ADFED317A20EE270A70B5FC
:1079F000FDEEC07A86B017EE904A054684EAE47040
:107A0000002303A9A0EBE470CDE90033029360F0FA
:107A1000D9FD002CACBF20232D2303A88DF8003006
:107A200063F0D0FC01286E4628D0022832D003280B
:107A30001CD003A930466AF0CAFA304663F0C2FC93
:107A40000338C4B22246314628466AF07FF8002344
:107A50002B55284663F0B6FC2E232B5401303119E8
:107A600028446AF0D0FA284606B070BD302303A936
:107A700030468DF801306AF0AAFADEE743F23002B0
:107A8000302303A93046ADF801208DF803306AF0A9
:107A90009EFAD2E743F2300303A93046ADF8013035
:107AA0006AF095FAC9E700BF6F12033A00007A4402
:107AB0000378202B024600F10100F9D0092BF7D002
:107AC0002D2B28D02B2B03BF5378B7EE000A02468C
:107AD000B7EE000AA3F13001C8B209289FED567A2B
:107AE00010D8F2EE046A07EE901AF8EEE77A12F870
:107AF000013FE7EE267AA3F13001C8B20928B0EEC3
:107B0000677AF0D92E2B5ED003F0DF03452B07D028
:107B100020EE070A70475378BFEE000A0246D9E705
:107B200010B451782D2978D02B296AD0A1F13003D7
:107B3000092B02F101026BD80024002303EB83031D
:107B400001EB430312F8011FA1F130000928A3F152
:107B50003003F3D9B3F59A7F1A4628BF4FF49A72CF
:107B6000072B66D9DFED356A1346F7EE007A083B3E
:107B7000072B67EEA67AFAD802F00702DAB1F2EE26
:107B8000046A012A67EEA67A15D0022A67EEA67A61
:107B900011D0032A67EEA67A0DD0042A67EEA67AE2
:107BA00009D0053A67EEA67A05D067EEA67A012AD3
:107BB00018BF67EEA67A6CB387EE277A5DF8044BA0
:107BC00020EE070A70475378A3F13001C8B20928A4
:107BD00002F1010298D8F2EE046AF0EE665A07EE5E
:107BE000901AF8EEE77A12F8013F87EEA66AA3F141
:107BF0003001C8B2092866EEA56A37EE067AEED9DA
:107C000082E79178A1F13003092B02F1020293D9A6
:107C1000F7EE007A27EE277AD0E79178A1F13003CA
:107C2000092B02F1020288BFF7EE007AC4D80124C2
:107C300083E7F7EE007AA1E70000000020BCBE4C0D
:107C40000378202B024600F10100F9D0092BF7D070
:107C5000303BDBB2092B4FF000000AD812F8011FAD
:107C600000EB8000303903EB4000CBB2092BF5D993
:107C7000704770470378202B024600F10100F9D0CD
:107C8000092BF7D02D2B0CBF0246012092F800C023
:107C9000ACF13001CBB208BF4FF0FF30092B4FF0F1
:107CA00000030CD812F801CF03EB830301EB43036D
:107CB000ACF130015FFA81FCBCF1090FF2D903FB92
:107CC00000F07047F0B5384D2B78082141F22100C3
:107CD0008B4002E0013993B209D013F4004F4FEA10
:107CE0004302F7D080EA430301399BB2F5D1B5F8DE
:107CF0000120002A55D0DFF8C0C02C4EB4452DD24B
:107D0000ACF1060C0CEB0204B44227D2052A41F276
:107D1000210022D9A44514D00CF1FF3C04F1FF3E10
:107D20001CF8011F082283EA012313F4004F80EAA4
:107D300043010ABF5B008BB29BB2013AF5D1E64525
:107D4000EED1228862B1A11DB14206D2A118B14282
:107D5000A44602D2052A0C46DCD800210846F0BD14
:107D6000A71C264641F2210016F8011B082283EACF
:107D7000012313F4004F80EA43010ABF5B008BB27A
:107D80009BB2013AF5D1B742EED16188084AC91ACF
:107D9000B1FA81F1231D49095B1BA2F8B03C0846EA
:107DA000F0BD044FBC1EDCE700000E080000100808
:107DB000D870002003000E0807000E082DE9F041DE
:107DC0000446D0E90030134483421DD88E188E42F9
:107DD00017D00D4604F10C08002701E0AE4210D088
:107DE00023695A1C2261234415F8010B1873042AD5
:107DF000F4D141462046FAF7F9F8AE42C4E90470DE
:107E0000EED16069BDE8F0814FF0FF30FAE700BFC6
:107E100070B545880B460446C5F30B052A4600217C
:107E200018466AF0CCF82169084A9142034602D309
:107E3000074A914205D319B1BDE87040184608477A
:107E400070BD2A46BDE8704069F080BE082C080865
:107E50008230080810B50446C06900B110BD0C217D
:107E60001420FFF785FAE06110BD00BF10B1036870
:107E700082881A83704700BF2DE9F041154E002714
:107E80000546D6F8B40C86F8007103680C461B68EA
:107E9000AA2190469847D6F8B40C036839461B6867
:107EA0009847D6F8B40C036829461B689847D6F85B
:107EB000B40C036841461B6804EB08079847D6F8E2
:107EC000B40C14F8011B03681B689847A742F6D14D
:107ED000BDE8F081D870002070B5104C0022D4F8B5
:107EE000B43C84F800211A6806460D461846AA21BB
:107EF00013689847D4F8B40C036801211B689847AD
:107F0000D4F8B40C036831461B689847D4F8B40C15
:107F1000036829461B68BDE870401847D8700020E8
:107F200084B0F0B58FB014AC554D9DF8686084E80E
:107F30000F0000244FF08070C5F8B44C2CF0B2FA5A
:107F4000F8B1032390F904004E4ACDE901344FF40F
:107F5000E13300934FF0807123462FF0D1FFC5F835
:107F6000B40C70B120460121FFF7B6FF052007F0E1
:107F7000D3FA95F80841012C03D195F80C31A02BC8
:107F800005D000200FB0BDE8F04004B0704795F870
:107F90000051002DF5D13E20224608A98DF8205031
:107FA000FFF76AFF192007F0B7FA66B90C23012220
:107FB00008A93D208DF82030FFF75EFF192007F05B
:107FC000ABFA0120DEE7224608A93D208DF82050BB
:107FD000FFF752FF192007F09FFABDF95430BDF9A1
:107FE00056208DF814301B128DF8153013128DF8B1
:107FF0001730BDF958308DF8183014AD1B128DF8BC
:1080000016208DF819300FCD08AC0FC4BDF92A30F9
:10801000BDF95070BDF9526095E803008DF81A3033
:108020001B128DF81B30BDF92C308DF81C301B1243
:1080300044F8040B8DF81D30BDF92E3021808DF8E9
:108040001E3005A91B120C2255208DF81F30FFF79A
:1080500013FF192007F060FA3B128DF8153005A9BF
:108060003312672004228DF814708DF816608DF895
:108070001730FFF701FF192007F04EFA96E700BF0F
:10808000D8700020CD51000810B5184C04EB8000CA
:10809000D0F8B80C30B300EB400004EB800393F948
:1080A000C9CCBCF1FF3F1ED093F8D10CD0B104EB8A
:1080B0000C0293F8D00C92F804ED6423142103FB16
:1080C0000CFC00220CEB000304EB43030139B3F872
:1080D000083D704412FA83F2F4D10548A0FB023047
:1080E000C0F30F1010BD002010BD00BFD8700020DD
:1080F000CDCCCCCC70B5114B114CA34203D319E0BD
:108100000C33A34216D293F805C08C45F8D193F8EE
:1081100004C0844501D00028F2D193F807E09645C9
:10812000EED11D6895F804E0E645E9D12E689E423F
:10813000E6D100E00025284670BD00BF8430080865
:10814000043208080379022B00D0704710B582B0C2
:1081500090F910208DF8023002A801441E4802EB6D
:10816000820203244FF0000C4FF0010E00EB82025C
:108170008DF800C08DF801E08DF80340526B11F8C6
:10818000084C16498A4222D0A1F578418A4220D073
:1081900001F580618A4218D1118821F0400109045B
:1081A00003EB8303090C118000EB83001388016C3F
:1081B00023F0380331F824101B041B0C0B431380ED
:1081C00013889BB243F04003138002B010BD634696
:1081D000E2E77346E0E700BF1412002000300140E0
:1081E00070B50446234894F91030A66803EB830366
:1081F00000EB83031546B207586B82B00CD5019093
:1082000062F0DEFF0198294662F0DAFFA3689B075F
:1082100017D5012002B070BD636913B11A689B883D
:108220005383154B154A1B6856684FEAC30C144B11
:10823000A3FB0C3C4FEA9C1C53689B1B9C45FBD248
:10824000DDE70D4B0D491A680D4B4FF4FA7000FB3A
:1082500002F2A3FB0232486892094B681B1A9A4249
:10826000FBD26369002BD4D01A689B88138301204A
:1082700002B070BD141200207C360020001000E017
:10828000D34D621010B50379012B84B08E460DD00A
:10829000022B08D18368DB0758BF01F07F0104B0CF
:1082A000BDE810409CE7002004B010BD1446826871
:1082B0008DF80F4002F0010201920DF10F020092C1
:1082C000417C90F910007246FBF7BEFA04B010BD75
:1082D0002DE9F041046888B00546FDF717FBB6228A
:1082E0007E212046FFF7CEFF4FF0640807F0E6F846
:1082F00006460F4607F0E2F8831B61EB0701B3F572
:108300007A7F71F10003F5D3B8F10108EED10221B3
:108310002046FFF717FF636913B11A689B885383E0
:1083200007F0CCF806460F4607F0C8F8831B61EB50
:108330000702B3F57A7F72F10003F5D3636913B1D5
:108340001A689B8813834FF00A0807F0B7F80646AF
:108350000F4607F0B3F8831B61EB0701B3F57A7F93
:1083600071F10003F5D3B8F10108EED142467C214A
:108370002046FFF787FF07F0A1F806460F4607F0F3
:108380009DF8831B61EB0702B3F57A7F72F100035E
:10839000F5D3002259212046FFF774FF07F08EF82D
:1083A00006460F4607F08AF8831B61EB0702B3F518
:1083B0007A7F72F10003F5D35E22002371498DF8B4
:1083C00007200DF10702CDE902320122CDE9053186
:1083D000049202A94FF4A4722046079262F0A2FE12
:1083E0004FF00A0807F06AF806460F4607F066F8ED
:1083F000831B61EB0701B3F57A7F71F10003F5D3BD
:10840000B8F10108EED1012259212046FFF73AFFC9
:1084100007F054F806460F4607F050F8831B61EB4F
:108420000702B3F57A7F72F10003F5D38C22402165
:108430002046FFF727FF07F041F806460F4607F0F2
:108440003DF8831B61EB0702B3F57A7F72F10003FD
:10845000F5D3022241212046FFF714FF07F02EF842
:1084600006460F4607F02AF8831B61EB0702B3F5B7
:108470007A7F72F10003F5D32A6B434E95F82D00F5
:10848000B6FBF2F2092391B2404AFEF7C1FF4388DE
:10849000B6FBF3F6AE630279422142F0C0022046F9
:1084A000FFF7F0FE07F00AF805460E4607F006F85B
:1084B000431B61EB0602B3F57A7F72F10003F5D33B
:1084C000082243212046FFF7DDFE06F0F7FF0546B0
:1084D0000E4606F0F3FF431B61EB0602B3F57A7F0D
:1084E00072F10003F5D3042258212046FFF7CAFE9B
:1084F00006F0E4FF05460E4606F0E0FF431B61EB85
:108500000602B3F57A7F72F10003F5D30A225321F4
:108510002046FFF7B7FE06F0D1FF05460E4606F0EF
:10852000CDFF431B61EB0602B3F57A7F72F10003C6
:10853000F5D300227C212046FFF7A4FE06F0BEFF03
:1085400005460E4606F0BAFF431B61EB0602B3F583
:108550007A7F72F10003F5D306227D212046FFF7D2
:1085600091FE06F0ABFF04460D4606F0A7FF031B85
:1085700061EB0502B3F57A7F72F10003F5D308B021
:10858000BDE8F081A02E070840420F00E82F070841
:108590000C4B70B502463D21D3F8600FFFF772FE19
:1085A000192606F08BFF04460D4606F087FF031BD5
:1085B00061EB0502B3F57A7F72F10003F5D3013E5A
:1085C000EFD170BDD8700020F8B5782204460021A4
:1085D0000068FFF757FE052706F070FF05460E46B8
:1085E00006F06CFF431B61EB0602B3F57A7F72F174
:1085F0000003F5D3013FEFD1206820220121FFF7CE
:1086000041FE052706F05AFF05460E4606F056FFC6
:10861000431B61EB0602B3F57A7F72F10003F5D3D9
:10862000013FEFD120683A460221FFF72BFE642676
:1086300006F044FF04460D4606F040FF031B61EBC5
:108640000502B3F57A7F72F10003F5D3013EEFD155
:108650000120F8BD70B52422044641210068FFF7CF
:1086600011FE90B9052606F029FF04460D4606F0D6
:1086700025FF031B61EB0502B3F57A7F72F100035E
:10868000F5D3013EEFD1012070BD206820223021BA
:10869000FFF7F8FD0028E5D0206806223121FFF71A
:1086A000F1FD0028DED0206800223421FFF7EAFD2A
:1086B000D8E700BFF8B5072204460A210068FFF793
:1086C000E1FD052706F0FAFE05460E4606F0F6FE29
:1086D000431B61EB0602B3F57A7F72F10003F5D319
:1086E000013FEFD1206824224121FFF7CBFD052770
:1086F00006F0E4FE05460E4606F0E0FE431B61EB85
:108700000602B3F57A7F72F10003F5D3013FEFD192
:108710002068C0224221FFF7B5FD052606F0CEFEF7
:1087200004460D4606F0CAFE031B61EB0502B3F5D5
:108730007A7F72F10003F5D3013EEFD10120F8BD3D
:1087400010B50446002221210068FFF79BFD206838
:10875000FC222021FFF796FD206840222421FFF70C
:1087600091FD20680C222321FFF78CFD2068002258
:108770002221FFF787FD012010BD00BFF8B50122BF
:10878000074610210068FFF77DFD00B9F8BD1426EB
:1087900006F094FE04460D4606F090FE031B61EBC6
:1087A0000502B3F57A7F72F10003F5D3013EEFD1F4
:1087B0003868A022BDE8F840112163E510B50468CF
:1087C0002379012B84B010D0022B0BD1A368DB07D7
:1087D0004FF0F0024CBFFF217F21204604B0BDE8DE
:1087E0001040FDE4002004B010BDA268617C94F943
:1087F000100002F0010201920DF10F020092F0242C
:10880000FF228DF80F40FBF71FF804B010BD00BF2A
:1088100010B504682379CA4341EA0211012B84B0E0
:10882000CAB20ED0022B09D1A368DB074CBFD221FC
:108830005221204604B0BDE81040D1E4002004B02D
:1088400010BD8DF80F20A268617C94F9100002F031
:1088500001020DF10F04CDE90042D222FAF7F4FF34
:1088600004B010BD10B504682379012B84B010D07A
:10887000022B0BD1A368DB074FF0B4024CBFFF21E2
:108880007F21204604B0BDE81040A9E4002004B0D8
:1088900010BDA268617C94F9100002F001020192FF
:1088A0000DF10F020092B424FF228DF80F40FAF769
:1088B000CBFF04B010BD00BF10B504682379012BB5
:1088C00084B00FD0022B0AD1A368DB070A462046EA
:1088D0004CBFA521252104B0BDE8104080E4002054
:1088E00004B010BDA26894F910008DF80F1002F0CA
:1088F0000102617C0DF10F04CDE90042A522FAF7D7
:10890000A3FF04B010BD00BF10B504682379012B8C
:1089100084B010D0022B0BD1A368DB074FF0960276
:108920004CBFFF217F21204604B0BDE8104057E432
:10893000002004B010BDA268617C94F9100002F020
:10894000010201920DF10F0200929624FF228DF890
:108950000F40FAF779FF04B010BD00BF10B50468EE
:108960002379012B84B00FD0022B0AD1A368DB0737
:108970000A4620464CBF8721072104B0BDE81040BD
:108980002EE4002004B010BDA26894F910008DF808
:108990000F1002F00102617C0DF10F04CDE90042DD
:1089A0008722FAF751FF04B010BD00BF10B504686C
:1089B0002379C901012B84B0CAB20AD0022B05D198
:1089C0007821204604B0BDE8104009E4002004B03E
:1089D00010BD8DF80F20A268617C94F9100002F0A0
:1089E00001020DF10F04CDE900427822FAF72CFFC5
:1089F00004B010BD10B504682379012B84B011D0E8
:108A0000022B0CD1A368DB074FF055024CBFA52108
:108A10002521204604B0BDE81040FFF7E1BB00204F
:108A200004B010BDA268617C94F9100002F001024C
:108A300001920DF10F0200925524A5228DF80F40EE
:108A4000FAF702FF04B010BD10B504682379012BBA
:108A500084B00ED0022B09D1A368DB074FF031029E
:108A60004CBFF42174212046FFF7BAFB012004B06B
:108A700010BDA268617C94F9100002F0010201921D
:108A80000DF10F0200923124F4228DF80F40FAF715
:108A9000DBFE012004B010BD10B504682379012B62
:108AA00084B00CD0022B07D101225821204604B0FB
:108AB000BDE81040FFF794BB002004B010BDA268D1
:108AC00094F91000617C8DF80F3002F001020192E0
:108AD0000DF10F0200925822FAF7B6FE04B010BD55
:108AE00010B504682379012B84B00CD0022B07D178
:108AF00001224821204604B0BDE81040FFF770BBBA
:108B0000002004B010BDA26894F91000617C8DF8BB
:108B10000F3002F0010201920DF10F020092482283
:108B2000FAF792FE04B010BD10B504682379012B4A
:108B300084B00CD0022B07D11A460821204604B07D
:108B4000BDE81040FFF74CBB002004B010BDA26888
:108B5000617C94F9100002F0010201920DF10F0204
:108B60000092022408228DF80F40FAF76DFE04B03F
:108B700010BD00BF10B504682379012B84B00CD060
:108B8000022B07D101220821204604B0BDE8104085
:108B9000FFF726BB002004B010BDA26894F91000B6
:108BA000617C8DF80F3002F0010201920DF10F028D
:108BB00000920822FAF748FE04B010BD30B50568EF
:108BC0002B79012B85B0044612D0022B0DD1012246
:108BD0000B212846FFF704FB38B120681D2209212C
:108BE00005B0BDE83040FFF74DBB002005B030BDFB
:108BF000AA6895F91000697C8DF80F3002F0010227
:108C000001920DF10F0200920B22FAF71DFEE3E72D
:108C100010B5154BD3F8644F84B024B12379012BE0
:108C200010D0022B02D0002004B010BDA16811F0BA
:108C30000101024618BF8021204604B0BDE8104063
:108C4000FFF7CEBAA268617C8DF80F0002F0010236
:108C500094F910000DF10F04CDE900428022FAF7DB
:108C6000F3FD04B010BD00BFD8700020F0B505467C
:108C700090F91000244C00EB800004EB8000AC68FD
:108C8000406BA40785B010D5CDE90223019062F0B6
:108C900097FADDE902230198002162F0F3F9AB684D
:108CA0009B0718D5012005B0F0BD6C6914B126688A
:108CB000A4887483154C164E246877684FEAC40E56
:108CC000144CA4FB0E4E4FEA9E1E7468A4EB070CD6
:108CD000E645FAD2D8E70D4B0D491A680D4B4FF413
:108CE000FA7000FB02F2A3FB0232486892094B685B
:108CF0001B1A9A42FBD26B69002BD3D01A689B884F
:108D00001383012005B0F0BD141200207C36002032
:108D1000001000E0D34D621030B50579012D83B00D
:108D20008E460DD0022D08D18468E40758BF41F06B
:108D3000800103B0BDE8304098E7002003B030BDAB
:108D400014468268009402F00102417C90F9100000
:108D500001927246FAF778FD03B030BDF0B50546D2
:108D6000164695F91020244802EB820200EB82029D
:108D700083B0506BAA6892070FD5CDE9000362F06B
:108D80001FFA019B00980022314662F07BF9AB6824
:108D90009B0718D5012003B0F0BD6A6912B11468B1
:108DA00092886283154A1468154A4FEAC40E154C1E
:108DB0005768A4FB0E4E4FEA9E1E5468A4EB070CA6
:108DC000E645FAD2D9E70D4B0D491A680D4B4FF421
:108DD000FA7000FB02F2A3FB0232486892094B686A
:108DE0001B1A9A42FBD26B69002BD3D01A689B885E
:108DF0001383012003B0F0BD141200207C36002044
:108E0000001000E0D34D621030B50579012D83B01C
:108E10008E460DD0022D08D18468E40758BF41F07A
:108E2000800103B0BDE8304098E7002003B030BDBA
:108E300014468268009402F00102417C90F910000F
:108E400001927246FAF7CCFC03B030BD10B504466F
:108E50000068037982B0022B0CBF43210321062353
:108E60006A46FFF7D1FF68B1BDF80010BDF80220D7
:108E7000BDF8043049BA52BA5BBAE18662872387EB
:108E800002B010BDE086A06302B010BD70B50668E8
:108E9000F46982B005466CB33379012B04F1030207
:108EA00005D0022B1AD00020A07002B070BDB368AC
:108EB000717C96F91000009203F0010301930C22DB
:108EC0000D23FAF78DFCA0700028EED063892B8467
:108ED000A3896B84E389AB8402B070BDB36813F0DF
:108EE000010F30464FF00D0314BF0C218C21FFF70A
:108EF00035FFE8E70C211420FEF73AFAF06104464A
:108F00002E68C9E710B500680379012B84B00C46C0
:108F100018D0022B13D1836813F0010F14BF222144
:108F2000A221032303AAFFF719FF30B1BDF90D30C9
:108F300003EB83031B12E633238004B010BD002033
:108F400004B010BD8368417C90F9100003F0010368
:108F5000019303AB009322220323FAF741FC00287C
:108F6000E4D1EAE710B5044600680379012B84B028
:108F70001ED0022B19D1836813F0010F02AA4FF003
:108F8000060314BF1F219F21FFF7E8FE58B1BDF86B
:108F90000810BDF80A20BDF80C3049BA52BA5BBAC5
:108FA000E1812282638204B010BD002004B010BDB4
:108FB0008368417C90F9100003F00103019302AB38
:108FC00000931F220623FAF70BFCDFE710B50446D7
:108FD00000680379012B84B01ED0022B19D183685D
:108FE00013F0010F02AA4FF0060314BF2521A5219B
:108FF000FFF7B4FE58B1BDF80810BDF80A20BDF85F
:109000000C3049BA52BA5BBA21846284A38404B09A
:1090100010BD002004B010BD8368417C90F91000A1
:1090200003F00103019302AB009325220623FAF714
:10903000D7FBDFE700B500680379012B85B032D09C
:10904000022B25D1062302AAF721FFF787FEF8B1EC
:109050009DF809209DF808C09DF80A109DF80C3075
:109060009DF80BE0120142EA0C3242EA1112154956
:109070001B018A62C1F8682F9DF80D2043EA0E3368
:1090800043EA12138B60C1F86C3F05B05DF804FB36
:109090000C4BD3F8681FD3F86C2F996200209A60AC
:1090A00005B05DF804FB8368417C90F9100002AACA
:1090B00003F00103CDE900230623F722FAF790FB22
:1090C000C5E700BFD870002000B500680379012B08
:1090D00085B01CD0022B0AD1836813F0010F03AABC
:1090E0004FF0030314BF00218021FFF737FE9DF8E6
:1090F0000D309DF80C009DF80E100C4A1B0243EA3F
:1091000000430B430120D36405B05DF804FB836882
:10911000417C90F9100003AA03F00103CDE900237C
:1091200003230022FAF75CFBE1E700BFD8700020C0
:1091300000B500680379012B85B01CD0022B0AD141
:10914000836813F0010F03AA4FF0030314BF00213B
:109150008021FFF703FE9DF80D309DF80C009DF86F
:109160000E100C4A1B0243EA00430B430120136616
:1091700005B05DF804FB8368417C90F9100003AAF8
:1091800003F00103CDE9002303230022FAF728FBB3
:10919000E1E700BFD870002010B500680379012B0B
:1091A00084B029D0022B24D1836813F0010F4FF033
:1091B000030303AA14BF19468321FFF7CFFDB0B103
:1091C0009DF80C309DF90C109DF80D209DF80EC0F7
:1091D0001B04002943EA0223B8BF4FF07F410D4A28
:1091E000A8BF002143EA0C030B43C2F8443104B08A
:1091F00010BD002004B010BD8268417C90F91000C1
:1092000002F00102032303ACCDE900421A46FAF74B
:10921000E7FAD4E7D870002000B500680379012B85
:1092200085B02BD0022B25D1836813F0010F03AA40
:109230004FF0030314BF00218021FFF78FFDB0B171
:109240009DF80C309DF90C109DF80D209DF80EC076
:109250001B04002943EA0223B8BF4FF07F410E4AA6
:10926000A8BF002143EA0C030B43C2F8283105B024
:109270005DF804FB002005B05DF804FB8368417CC9
:1092800090F9100003AA03F00103CDE900230323A2
:109290000022FAF7A5FAD2E7D870002010B50446EC
:1092A00000680379012B84B03DD0022B36D183684E
:1092B00013F0010F02AA4FF0060314BF11219121F0
:1092C000FFF74CFD50B3BDF9083006EE903ABDF9FA
:1092D0000A30F8EEE66A07EE103ABDF90C30B7EE48
:1092E000086A07EE903A66EE866AB8EEC77AFDEE37
:1092F000E66A27EE067AF8EEE77A16EE903A67EE1F
:10930000867ABDEEC77AFDEEE77AE38617EE103A6D
:10931000238717EE903A638704B010BD0020E086E3
:10932000A06304B010BD8368417C90F9100003F085
:109330000103019302AB009311220623FAF750FABE
:10934000C0E700BF10B5044600230068E386A363AE
:109350000279012A84B022D0022A1DD1836813F039
:10936000010F02AA4FF0060314BF03218321FFF768
:10937000F5FC78B1BDF90A30BDF80810BDF80C2035
:109380005B4201EB410103EB430302EB4202E18646
:109390002387628704B010BD184604B010BD8368EF
:1093A000417C90F9100003F00103019302AB00939C
:1093B00003220623FAF714FADBE700BF70B5044670
:1093C000244894F91030A66803EB830300EB830371
:1093D0001546B207586B82B00ED5019061F0F0FED1
:1093E000012301980022294661F04CFEA3689B07E7
:1093F00017D5012002B070BD636913B11A689B884C
:109400005383154B154A1B6856684FEAC30C144B1F
:10941000A3FB0C3C4FEA9C1C53689B1B9C45FBD256
:10942000DBE70D4B0D491A680D4B4FF4FA7000FB4A
:1094300002F2A3FB0232486892094B681B1A9A4257
:10944000FBD26369002BD4D01A689B881383012058
:1094500002B070BD141200207C360020001000E025
:10946000D34D621010B50379012B82B08E460DD01A
:10947000022B08D18368DB0758BF41F0800102B09E
:10948000BDE810409AE7002002B010BD1446826883
:10949000009402F00102417C90F9100001927246A2
:1094A000FAF79EF902B010BD70B504682379012B5C
:1094B00084B00D4615D0022B10D1A368E122DB0742
:1094C0004CBF114661212046FEF78AFE30B12A4684
:1094D000FF21204604B0BDE87040C3E7002004B07F
:1094E00070BDA26894F91000617C02F001020DF1D8
:1094F0000F0601920096E1228DF80F20FAF7A4F9E9
:10950000E4E700BF30B504682379012B85B00D4630
:1095100016D0022B11D1A368DB074FF0C3024CBF5A
:10952000E12161212046FEF75BFE30B12A46FF2192
:10953000204605B0BDE8304094E7002005B030BDBE
:10954000A26894F91000617C02F0010201920DF111
:109550000F020092C3228DF80F20E122FAF774F96E
:10956000E3E700BF70B505682B79012B84B0044692
:109570000E4619D0022B14D1AB68DB074FF0F00276
:109580004CBFE12161212846FEF72AFE48B1221D89
:10959000FF212846FFF766FF18B12379337004B026
:1095A00070BD002004B070BDAA6895F91000697CF8
:1095B00002F0010201920DF10F020092F0228DF8EB
:1095C0000F20E122FAF740F9E0E700BF2DE9F04172
:1095D0006C4A0468016B6C4FB7FBF1F182B0064630
:1095E00089B20F2390F82D00FDF712FF4388B7FBD7
:1095F000F3F70546B7633046FCF788F900212046AB
:10960000FEF7A0FD0F224E212046FEF73BFE4FF055
:109610000F0805F053FF06460F4605F04FFF831B6A
:1096200061EB0701B3F57A7F71F10003F5D3B8F16F
:109630000108EED16A794F2102F00F022046FEF7B1
:1096400021FE4FF00F0805F039FF06460F4605F0E2
:1096500035FF831B61EB0701B3F57A7F71F10003DE
:10966000F5D3B8F10108EED16A79502102F00F026A
:109670002046FEF707FE4FF00F0805F01FFF0646D5
:109680000F4605F01BFF831B61EB0701B3F57A7FE3
:1096900071F10003F5D3B8F10108EED16A7942EA1D
:1096A00002125221D2B22046FEF7ECFD0F2705F040
:1096B00005FF05460E4605F001FF431B61EB060260
:1096C000B3F57A7F72F10003F5D3013FEFD10322A6
:1096D00014212046FEF7D6FD0F2705F0EFFE0546C4
:1096E0000E4605F0EBFE431B61EB0602B3F57A7FF5
:1096F00072F10003F5D3013FEFD13A4663212046D2
:10970000FEF7C0FD642705F0D9FE05460E4605F0BC
:10971000D5FE431B61EB0602B3F57A7F72F10003BD
:10972000F5D3013FEFD1082265212046FEF7AAFDBF
:109730000DF1070264212046FFF794FE9DF80720F3
:1097400022F0100242F06002642120468DF80720CA
:10975000FEF798FD0F2705F0B1FE05460E4605F011
:10976000ADFE431B61EB0602B3F57A7F72F1000395
:10977000F5D3013FEFD103212046FEF7E3FC02B011
:10978000BDE8F0812030070840420F002DE9F0418C
:10979000804682B00527962605F090FE04460D46C9
:1097A00005F08CFE031B61EB0501B3F57A7F71F1C7
:1097B0000003F5D3013EEFD10DF1070231464046DB
:1097C000FFF750FE08B9013FE5D102B0BDE8F081D6
:1097D000F0B583B015460DF107021C4606460F464C
:1097E000FFF740FE9DF8072005EA0203A34201D1DE
:1097F00003B0F0BD22EA050222433946304603B0E9
:10980000BDE8F040FEF73EBDF0B5044683B00D461E
:109810001746061D20680379012B18D0022B13D19F
:109820008368DB0732464FF0FF015CBF3246FF2101
:10983000FFF7C4FD30B115B12379DB07EAD40FB1CE
:1098400023793B7003B0F0BD002003B0F0BD826807
:10985000417C90F9100002F00102CDE90062FF2284
:10986000F9F7BEFFE6E700BF30B5044683B0051D3B
:1098700020680379012B14D0022B0FD18368DB07FA
:109880002A464FF0FF015CBF2A46FF21FFF796FDF5
:1098900010B12379DB07EBD403B030BD002003B057
:1098A00030BD8268417C90F9100002F00102CDE9E0
:1098B0000052FF22F9F794FFEAE700BF30B50246F5
:1098C000044652F8040B0379012B83B00ED0022B0F
:1098D00009D1FF21FFF772FD18B12079C04300F0D4
:1098E000010003B030BD002003B030BD8568417C6D
:1098F00090F91000009205F001050195FF22F9F79B
:109900006FFFE9E730B5B42283B00446FF21006859
:10991000FEF7B8FC10B9002003B030BD2068037911
:10992000012B04F1040514D0022BF4D18368DB076A
:109930002A464FF0FF015CBF2A46FF21FFF73EFD9C
:109940000028E8D02379DB07E6D520680379012BCE
:10995000EAD18268417C90F9100002F00102CDE961
:109960000052FF22F9F73CFFEAE700BF30B50A4694
:1099700083B00446A5210068FEF784FC10B90020DE
:1099800003B030BD20680379012B04F1040514D025
:10999000022BF4D18368DB072A464FF0FF015CBF3E
:1099A0002A46FF21FFF70AFD0028E8D02379DB07CC
:1099B000E6D520680379012BEAD18268417C90F9D1
:1099C000100002F00102CDE90052FF22F9F708FF72
:1099D000EAE700BF70B582B0CDE900230446FFF787
:1099E00091FF10B9002002B070BD20685522A5215A
:1099F000FEF748FC0028F5D0251D20682A46FF21E7
:109A0000FFF730FD0028EDD02379DB07F5D40DF109
:109A1000FF350DF1070615F8011F2046FFF7A6FFD9
:109A20000028DFD0B542F6D1DDE700BF002A37D0ED
:109A3000F0B5013A83B004464E1E51FA82F7051D77
:109A400016F8012F2068A521FEF71CFC90B9002014
:109A500003B0F0BD8268417C90F9100002F0010271
:109A6000CDE90052FF22F9F7BBFE0028EFD02379A1
:109A7000DB0710D520680379012BEBD0022BE6D150
:109A80008368DB072A464FF0FF015CBF2A46FF21AF
:109A9000FFF794FCE9E7B742D2D1012003B0F0BD53
:109AA0000120704770B5962282B004460E460068C9
:109AB000FF21FEF7E7FB10B9002002B070BD251DA5
:109AC00020680379012B1FD0022BF5D18368DB07B7
:109AD0002A464FF0FF015CBF2A46FF21FFF76EFCCC
:109AE0000028E9D02379DB07EAD42468E122114673
:109AF0002046FEF7C7FB0028DED03246FF21204675
:109B000002B0BDE87040ADE48268417C90F910007D
:109B100002F00102CDE90052FF22F9F761FEDFE712
:109B2000002A4BD02DE9F041013A4F1C82B0044687
:109B30000E4657FA82F7051D20689622FF21FEF790
:109B4000A1FB98B9002002B0BDE8F0818268417C99
:109B500090F9100002F00102CDE90052FF22F9F75E
:109B60003FFE0028EED02379DB0710D5206803796B
:109B7000012BEBD0022BE5D18368DB072A464FF09F
:109B8000FF015CBF2A46FF21FFF718FCE9E7D4F884
:109B90000080E12211464046FEF774FB0028D1D038
:109BA00032464046FF21FFF75DFC0028CAD001364F
:109BB000BE42C1D1012002B0BDE8F0810120704752
:109BC00070B505460B460446164655F8040B82B0A0
:109BD00087211A46FEF756FB20680379012B18D01F
:109BE000022B13D18368DB072A464FF0FF015CBFCD
:109BF0002A46FF21FFF7E2FB30B12379DA07EBD4E5
:109C000016B1C3F34013337002B070BD002002B030
:109C100070BD8268417C90F9100002F00102CDE92C
:109C20000052FF22F9F7DCFDE6E700BF70B57821AE
:109C300082B00446164600680022FEF723FB10B9E6
:109C4000002002B070BD251D20680379012B14D0BF
:109C5000022BF5D18368DB072A464FF0FF015CBF7A
:109C60002A46FF21FFF7AAFB0028E9D02379DA076B
:109C7000EAD45B09337002B070BD8268417C90F910
:109C8000100002F00102CDE90052FF22F9F7A8FD11
:109C9000EAE700BF30B5CC2283B00446A5210068B6
:109CA000FEF7F0FA10B9002003B030BD2068037948
:109CB000012B04F1040514D0022BF4D18368DB07D7
:109CC0002A464FF0FF015CBF2A46FF21FFF776FBD3
:109CD0000028E8D02379DB07E6D520680379012B3B
:109CE000EAD18268417C90F9100002F00102CDE9CE
:109CF0000052FF22F9F774FDEAE700BF30B5B42245
:109D000083B00446FF210068FEF7BCFA10B90020BA
:109D100003B030BD251D20680379012B22D0022B12
:109D2000F5D18368DB072A464FF0FF015CBF2A4666
:109D3000FF21FFF743FB0028E9D02379DA07EAD4B3
:109D4000CC212046FFF712FE0028E0D002E0237964
:109D5000DB07DDD520682A46FF21FFF783FB0028BB
:109D6000F5D1D4E78268417C90F9100002F001023D
:109D7000CDE90052FF22F9F733FDDCE72DE9F04F82
:109D800089B00446CDE90623002004F1040B0490B9
:109D9000029103905D462046049FFFF7B3FD069BAA
:109DA000FE0003EBC70B20B90AE0237913F0010A88
:109DB0000DD020682A46FF21FFF754FB0028F4D17C
:109DC000079B1A46049B137009B0BDE8F08F9B07F0
:109DD000F6D5F0212046FFF7C9FD0028F0D0069BFC
:109DE000083E334401270593D0463E46029B002B94
:109DF0004AD0082E48D806F1FF3943FA09F909F08C
:109E0000010920684FEAC9127821FEF73BFA0028C1
:109E1000D6D020680379012B47D0022B43D1836829
:109E2000DB072A464FF0FF015CBF2A46FF21FFF700
:109E3000C5FA0028C4D0237913F00102E9D103F058
:109E4000600160294FEAD31C51D0029919B1082E44
:109E500001D8E145B4D1BCF1000F3AD01BF808306D
:109E60003B430BF808307F00013617F0FF07F6B2CE
:109E7000BCD108F101085FFA88F8B8F1080F36D0B4
:109E8000029B0127002BB4D1049BD3B1039BB342A7
:109E900017D9059B13F808301F4214BF4FF0010972
:109EA0004FF00009ADE700208AE78268417C90F915
:109EB000100002F00102CDE90052FF22F9F790FCF8
:109EC000B7E7039BA3EB0609B9FA89F94FEA5919D9
:109ED00097E71BF8081021EA07010BF80810990909
:109EE00041EA531313F0010F08BFB246BBE7402EFF
:109EF00006D8079B049A1B7893423FF64CAF5FE766
:109F00009BF807C00BF1FF370BF1060B17F8011F89
:109F1000082382EA010616F0010F4FEA520218BF29
:109F200082F08C0203F1FF3318BFD2B213F0FF03AB
:109F30004FEA5101EDD1BB45E8D19445D9D1049BFD
:109F40000133DBB20493BAF1000F3FF439AFCDF81F
:109F50000CA0CEE730B505682B79012B85B00446FF
:109F600000F09280022B08D1AB68DB0702AA4CBF3D
:109F7000082188212846FFF721FA9DF8083013F0C0
:109F8000100302D1184605B030BD2068062302AA8E
:109F90000021FEF739FF0028F5D09DF809209DF833
:109FA00008109DF80A309FED3F6A120202EB014251
:109FB0001344140248BF03F17F4307EE903AF8EED2
:109FC000E77A9DF80C109DF80B409DF80D20364B5C
:109FD000C7EE866A090201EB04410A44090248BF40
:109FE00002F17F42B3F92E1007EE902AB3F9402018
:109FF00003EE902AB3F93C20F8EEE77A07EE102A38
:10A00000C7EE864AB3F93820F8EEE33AB8EEC77ADD
:10A01000D3ED0D7AA6EEA37AF8EEE75A05EE102AF4
:10A02000E6EE875AB3F93E20D3ED0C7A04EE102AFF
:10A03000F8EEE77AB3F93A20E6EEA57A06EE102AB2
:10A04000B8EEC55AB8EEC44AB3F92C2007EE101A80
:10A05000B8EEC66AE4EE857AA6EE846A05EE902A2A
:10A06000B8EEC77AF8EEE55A66EEA46A24EE877A6F
:10A07000B6EE005AA5EE857AE6EE867A83ED127A80
:10A08000C3ED117A05B030BDAA68697C95F910005E
:10A0900002F00102019202AA00920822F9F7A0FB45
:10A0A0006BE700BF00007848D870002030B5056825
:10A0B0002B7987B00022012B04468DF80F2035D074
:10A0C000022B12D1AB68DB070DF10F024CBF272129
:10A0D000A7212846FFF772F928B19DF80F3013F039
:10A0E000080305D1184607B030BD104607B030BD93
:10A0F0002068062304AA2821FEF786FE20B3BDF9B6
:10A100001030BDF91220002BB8BF03339B10E3863B
:10A11000BDF91430002AB8BF0332002BB8BF033397
:10A1200092109B102287638707B030BDAA68697CB4
:10A1300095F9100002F0010201920DF10F02009258
:10A140002722F9F74DFBC7E7E086A06307B030BDD3
:10A1500030B5054600240068EC86AC630379012B1A
:10A1600087B02AD0022B0ED18368DB070DF10F02D6
:10A170004CBF21468021FFF721F928B19DF80F40FF
:10A1800014F0080402D1204607B030BD2868062329
:10A1900004AA0121FEF738FE0028F5D0BDF81430DE
:10A1A000BDF81010BDF812205BBA49BA52BA5B4232
:10A1B000E9862A876B8707B030BD22468468417CD8
:10A1C00090F9100004F0010401940DF10F040094C3
:10A1D000F9F706FBD1E700BF30B50446002025683B
:10A1E000E086A0632B79012B87B027D0022B10D1FA
:10A1F000AB68DB070DF10F024CBF06218621284614
:10A20000FFF7DCF828B19DF80F3013F0040302D1FA
:10A21000184607B030BD2068062304AA0021FEF7C7
:10A22000F3FD0028F5D0BDF81010BDF81220BDF8E0
:10A230001430E1862287638707B030BDAA68697C45
:10A2400095F9100002F0010201920DF10F02009247
:10A250000622F9F7C5FAD5E710B50368DA6B82B0C4
:10A26000044612B1904740B123685B6B1BB1214695
:10A2700001A8984718B9FF23638202B010BDBDF84A
:10A280000630013B9BB2F7E7F0B585B004461846AF
:10A290000D461646039361F095F828442768A0728E
:10A2A000E672204600240094039B7C6932462946CE
:10A2B000A04705B0F0BD00BF38B504468B6801600B
:10A2C0000D46984700230B4AE26023742B6B13B1B1
:10A2D000204698472074084B93F8703F1BB1237CAD
:10A2E00023F001032374002363822046BDE8384035
:10A2F000B2E700BF0001FF00D87000202DE9F04157
:10A30000264ED6F8645F84B09DB1B02280212846E5
:10A31000FDF7B8FF402280212846FDF7B3FF002259
:10A3200080212846FDF7AEFF102280212846FDF748
:10A33000A9FF4FF480644FF000080DF10F0795B1AD
:10A340002B79012B15D0022B0DD1AB6813F0010333
:10A350004FF000024FF04001284602BF1A4640214C
:10A360002846FDF73DFF013CA4B29CB1D6F8645FDE
:10A37000E5E7AA6895F91000697C8DF80F8002F076
:10A380000102013CCDE90072A4B24022F9F75CFA67
:10A39000002CEBD104B0BDE8F08100BFD8700020E4
:10A3A0000B4B10B5D3F8644F8CB15038C2B280213A
:10A3B0002046FDF767FF002280212046FDF762FF5F
:10A3C00020461022BDE810408021FDF75BBF10BD84
:10A3D000D8700020F0B5204C204F203800EB8000D2
:10A3E000661DD7F8645F85B004440644E5B12B7957
:10A3F0002278012B1DD0022B0AD1AB6813F0010F7C
:10A400004FF04001284604BF40212846FDF7E8FEF2
:10A410000134B442EAD155B100224021284605B0AA
:10A42000BDE8F040FDF72EBF0134B442F0D105B0D5
:10A43000F0BD8DF80F20AA6895F91000697C02F034
:10A44000010201920DF10F0200924022F9F7FCF98E
:10A45000D7F8645FDCE700BF7C300708D8700020C5
:10A460002DE9F041734ED6F8645F84B0002D00F002
:10A470009680D42280212846FDF704FF80221146D1
:10A480002846FDF7FFFEA82280212846FDF7FAFEA8
:10A490003F2280212846FDF7F5FED3228021284661
:10A4A000FDF7F0FE002280212846FDF7EBFE40225A
:10A4B00080212846FDF7E6FE8D2280212846FDF703
:10A4C000E1FE142280212846FDF7DCFEA122802136
:10A4D0002846FDF7D7FEC82280212846FDF7D2FE88
:10A4E000DA2280212846FDF7CDFE1222802128465F
:10A4F000FDF7C8FE812280212846FDF7C3FECF224A
:10A5000080212846FDF7BEFED92280212846FDF78E
:10A51000B9FEF12280212846FDF7B4FEDB2280211E
:10A520002846FDF7AFFE402280212846FDF7AAFE0F
:10A53000A42280212846FDF7A5FEA62280212846D8
:10A54000FDF7A0FEAF2280212846FDF79BFEA62244
:10A5500080212846FDF796FEAE2280212846FDF791
:10A5600091FE202280212846FDF78CFE00228021CA
:10A570002846FDF787FEB02280212846FDF782FE9F
:10A58000402280212846FDF77DFE002280212846BA
:10A59000FDF778FE102280212846FDF773FE4FF468
:10A5A00080644FF000080DF10F0755B32B79012B94
:10A5B0002FD0022B0DD1AB6813F001034FF0000236
:10A5C0004FF04001284602BF1A4640212846FDF7B9
:10A5D00007FE013CA4B2002CE7D175B18122802195
:10A5E0002846FDF74FFEC82280212846FDF74AFE87
:10A5F000AF2280212846FDF745FE012004B0BDE8CA
:10A60000F081013CA4B2002CE3D1012004B0BDE8EC
:10A61000F081AA6895F91000697C8DF80F8002F02E
:10A620000102CDE900724022F9F70EF9D6F8645F15
:10A63000CFE700BFD8700020FAF7A8BDFAF7A6BD93
:10A64000FAF7A4BDFAF7A2BDFAF7A0BDFAF79EBDCE
:10A650002DE9F041174DD5F8B83006463BB31B6ADB
:10A6600098470746D5F8BC307488012BB38813D0BF
:10A670009C420FD87868D5F8B83004FB00F0DB684E
:10A680009847D5F8B83000209B689847B3880134C4
:10A69000A342EFD2BDE8F08139885A1C121B8A42CE
:10A6A000E6D1D5F8B830BDE8F0411B69184705F68A
:10A6B0007477D7E7D870002038B50409013C032C23
:10A6C0001BD8104D05EB440200F00F03B2F828151B
:10A6D00041FA03F212F0010211D001209840013832
:10A6E00008402C4461F0C8FC94F83035064A184400
:10A6F00000EB400002EB800038BD002038BD104662
:10A7000038BD00BFF82D0708C82A00202DE9F04FFA
:10A710003C2204460021BA4893B067F050FCB94A85
:10A72000611EE01C144611F8013F5D1E032D88BF19
:10A730000023814244F8043BF5D102F11003114695
:10A7400051F8040B012800F050818B42F8D1002011
:10A75000114651F8044B022C00F03D818B42F8D198
:10A76000114651F8044B032C00F02B819942F8D18B
:10A7700052F8041B042900F01A819342F8D1DFF843
:10A7800080B2DFF8A482A04F5C460F250026002887
:10A790003CD0FFF791FF94F90D908246C0B107239A
:10A7A0008371002303720368984AC57103F13F4324
:10A7B00003F57E039B0AD05C5DF0B8FBBAF8043069
:10A7C0000393934B0493DAF8000003A9F8F74CF9CC
:10A7D000217B0023302201E018F8332091422ED053
:10A7E0000133102BF8D1002209EB490907EBC9030B
:10A7F0002261D3F8982022750132C3F898200721EE
:10A800000122A175627583F8942016440135EDB2DA
:10A81000132D04F10C0401D0207BB8E766B17D4C08
:10A82000DFF808920025237C7BB90135032D04F164
:10A83000180409F1C809F6D113B0BDE8F08F764AC3
:10A8400002EBC303D3F83825CEE760795DF06EFBE9
:10A8500020795DF06BFBA068F8F770F82368A068BA
:10A86000CDF814904C3304936369142202FB03F374
:10A8700007930023CDE90E33CDE9103306930893F7
:10A88000E36803934FF480624FF40063CDE909233A
:10A890004FF400514FF48073CDE90B134FF40033A4
:10A8A00003A90D935DF078FDA2685C49136843F03D
:10A8B000010313605A4A536823F4733323F4477334
:10A8C00023F0030343F44033536022686369506804
:10A8D0000194012B20F0407020F48070D4BF00263A
:10A8E000012640EA062050609068014041F00201D4
:10A8F0009160D16A013B21F47001DBB241EA03535C
:10A90000D3620BF130075B4601214FFA85FC4FF013
:10A91000070A587D18B193F90D00604514D00C3327
:10A92000BB42F6D19368019C43F400739360936833
:10A9300043F480739360936843F0010393609368DA
:10A9400043F08043936070E7187C4E1C09285FFA3F
:10A9500086F89E7D1CD8146900EB400E06FA0EF6B0
:10A960000AFA0EFE24EA0E0E46EA0E0616610629C3
:10A970005ED8013901EB8101D2F834E01F2404FADA
:10A9800001F688402EEA0606304341465063C6E78A
:10A99000A0F10A0ED4680EEB4E0E06FA0EF60AFA75
:10A9A0000EFE24EA0E0E46EA0E06D660DFE71D4BC9
:10A9B00093F8042D3021013283F8F81C83F8042D1C
:10A9C000DDE61849202481F8EC4C91F8044D01345F
:10A9D00081F8044DCCE61349352481F8E04C91F818
:10A9E000044D013481F8044DBAE60E4991F8044D46
:10A9F0003420013481F8D40C81F8044DA8E600BF5E
:10AA0000A07D0020907D002014120020C0210708A6
:10AA10000300010098120020F82D0708FDF7FFC081
:10AA200000230140D87000202C330708E07D00206F
:10AA30000C290ED8073901EB8101D2F830E01F2430
:10AA400004FA01F688402EEA0606304341461063B8
:10AA500065E70D3901EB8101D2F82CE01F2404FADF
:10AA600001F688402EEA060630434146D06256E79A
:10AA700010B503681A79022A044603D00023237113
:10AA8000236010BD987AFFF717FE0028F6D040F635
:10AA90001D610022C18002722021FAF70DFF002300
:10AAA0002371236010BD00BF70B506461C48336893
:10AAB00003F13F4303F57E039B0A82B0C05C0C4662
:10AAC00015465DF033FAB2880092B2FA82F304F0D0
:10AAD00003028DF80420C4F3810230688DF805204C
:10AAE000C3F11F03C4F3001264098DF80740C3F3D8
:10AAF000CC0400EB840403F007038DF806209B00D0
:10AB0000226A0F269D4006FA03F322EA030323621A
:10AB1000226A154369462562F7F7A6FF02B070BDA9
:10AB2000C02107082DE9F04FAB4CAC4DAC4283B0CF
:10AB300050D21E4602E00C34AC424BD294F805C011
:10AB40008C45F8D194F804C0844501D00028F2D196
:10AB500094F807C09445EED12568002D3BD0002322
:10AB60006B60AB60EB602B616B61AB61EB612C6088
:10AB700022792A71A779AF60217AE960012A33D05E
:10AB8000022A27D1E07AFFF797FD94F90980A8619E
:10AB9000A07A85F81080FFF78FFD6861F8B1904CBE
:10ABA00008EB880A04EB8A0A4FEA8809DAF834309D
:10ABB000ABB19AF8463003B30E2200238671C271FE
:10ABC00003720921FAF778FE6B6923B11A689B8832
:10ABD000138300E00025284603B0BDE8F08F284627
:10ABE000FFF746FF0025F6E7E07AFFF765FD627A9A
:10ABF000A37A6B74A8612A74EDE79AF83C005DF0C3
:10AC000095F99AF83C104A09012301F01F01023A14
:10AC10008B40032A08D8DFE802F0ADB3A7027149E0
:10AC20004A6922EA03034B6109EB080304EB83033F
:10AC300008F1010A93F83900FFF73EFD5FFA8AFA3E
:10AC4000014620B140F60D3380F808A0C38009EB1F
:10AC5000080304EB8303009193F83B00FFF72CFDFE
:10AC60000099034620B140F60D5280F808A0C2803A
:10AC700009EB080204EB8202CDE9001392F83A00D6
:10AC8000FFF71AFDDDE90013834620B140F60D42BF
:10AC900080F808A0C28009EB080204EB820217F0DA
:10ACA000040A92F83D2071D039B108464A21019337
:10ACB0000092FFF7F9FEDDE900232BB118462A21A7
:10ACC0000092FFF7F1FE009ABBF1000F03D0584647
:10ACD0000A21FFF7E9FE09EB080B04EB8B0B9BF84D
:10ACE0003870002F6DD109EB080304EB83033E4A53
:10ACF0005B6B934200F09A803C4A934200F0AC8038
:10AD00003B4A934200F09D803A4A934200F0838090
:10AD1000394A934274D0394A934200F0A8801A8885
:10AD2000BAF1000F02F441510CBF032200220A4382
:10AD300042F445721A809A8B22F400621204120CBB
:10AD40009A8307221A821A8892B242F040021A802D
:10AD500077BBC844686904EB8804012384F8463053
:10AD600000283FF42EAF27E71E490A6922EA0303B1
:10AD70000B6159E71B494A6A22EA03034B6253E716
:10AD800018490A6A22EA03030B624DE739B1084603
:10AD90000A2101930092FFF787FEDDE90023002BD3
:10ADA00092D018460A210092FFF77EFE009A8BE7A8
:10ADB0003846FFF781FC0028CBD0036882881A83CD
:10ADC000C7E73846FFF778FC00288CD09BF83D2079
:10ADD0000921FFF769FE86E7843008080432080875
:10ADE00014120020003802400030014000380040BA
:10ADF000003C00400034014000500140005401403C
:10AE000002F56842516A41F480115162516A21F49D
:10AE10008011516283E702F58232516A41F4005198
:10AE20005162516A21F40051516278E702F584328F
:10AE3000516A41F480515162516A21F4805151624A
:10AE40006DE702F5FE32116A41F400411162116AA8
:10AE500021F40041116262E702F50032116A41F407
:10AE600080411162116A21F48041116257E702F5B5
:10AE70006442516A41F400115162516A21F4001197
:10AE800051624CE7F0B5C2B283B0102330210220EA
:10AE9000FFF748FE6A4FC7F8480100286BD003212E
:10AEA000FDF750F99F230093322604F007FB044678
:10AEB0000D4604F003FB031B61EB0502B3F57A7F3B
:10AEC00072F10003F5D3013EEFD1D7F848515D4C44
:10AED00095F910308DF8056003EB830304EB8303D1
:10AEE000586BAB689A0740F1848004230DEB030193
:10AEF0006A4660F0C7F8AB689B0763D59DF80630DB
:10AF00009DF805109DF807201B0243EA01431343F7
:10AF10004D4A934200F08E800FDD4C4A934200F37D
:10AF20008280053A934237DD494A1A44042A7AD886
:10AF3000DFE802F042792C0F3800A2F52202013A34
:10AF4000934239D019DD434A93421FD001329342D4
:10AF500069D14FF480732380A3816288120202FBBF
:10AF600003F30021B3F1807FC4E90123A17353D817
:10AF7000012087F84C0103B0F0BD374A9342E8D076
:10AF800002F5D61202F6FF72934212D180234FF4DB
:10AF900080722380A281E0E7304A9342F6D00232E9
:10AFA000934240D14FF400734FF480722380A2810A
:10AFB000D3E72B4A934236D120234FF4807223806B
:10AFC000A281CAE7274B28491A68284B48684FF4E2
:10AFD000FA7606FB02F2A3FB023292094B681B1AB7
:10AFE0009A42FBD26B69002B88D01A689B88138326
:10AFF00084E76B6913B11A689B885383194B1A490C
:10B000001A681A4B4E68D200A3FB023292094B68B1
:10B010009B1B9A42FBD268E70123B72087F8543183
:10B02000FAF7EEF9A4E70020C4E901002080A0812E
:10B0300003B0F0BD40234FF480722380A2818CE7DF
:10B04000D8700020141200201620C2001940EF0012
:10B05000EBBF10FF17BA2000186001001720C200D4
:10B06000154001007C360020001000E0D34D621036
:10B0700038B500231A4635210120FFF753FD154D41
:10B080000446C5F8840FD8B1FEF780FB48B1012310
:10B090002046A5F88C3F0022BDE838404021FDF74E
:10B0A000F1B895F8883F1A2B08BF0223204608BF45
:10B0B000C5F8903FFFF7DCFC002385F88C3F38BDD6
:10B0C00095F8883F85F88C0F1A2B04BF0123C5F82B
:10B0D000903F38BDD8700020074B53F8203021B185
:10B0E0004BB11A689B8853837047002BFCD01A68B9
:10B0F0009B88138370477047E82D07082DE9F04FB0
:10B100008A4B8B4C93F8B09F93F8B18F93F8B27F32
:10B11000DFF820A283B003F6B475002605F1800B9A
:10B1200001964FF0010EAB78E978C3F1FF039BB2B3
:10B13000002B49D10B460F468C4600918846894624
:10B1400001210191009A100240EA0340172240EACF
:10B150000C0006EB020CACEB02030EFA02F19BB200
:10B16000014204EB830314BF02210121013A43F899
:10B17000C41C531CEFD104351836AB45B6B2D2D13E
:10B180004FF44073A4F8E43B2023A4F8E63B019B72
:10B1900033B1664B83F8B09F83F8B18F83F8B27FE9
:10B1A00094F8E83B6BB1D4F8EC0B50B140F22A3183
:10B1B000F7F710FAD4F8EC0B03B0BDE8F04FF7F74F
:10B1C0003DBA03B0BDE8F08FB5F800C00091C3F1FF
:10B1D000FF03AAFB0C2001FB03F340091B12052807
:10B1E00000F29E80DFE800F08B6E54371C03AAFB50
:10B1F0000C277F09C7EB0717ACEB8707BFB2C81A4C
:10B20000C7F13C0700FB07F7AAFB07275FFA83F8A3
:10B2100008EB57178946FFB20121BC46019191E71F
:10B22000AAFB0C025209C2EB0212ACEB820292B2F0
:10B23000A1EB030902FB09F9AAFB09295FFA83F8CC
:10B2400008EB59198C465FFA89F90F460121CDF8B0
:10B250000090019176E7AAFB0C025209C2EB0212A0
:10B26000ACEB82081FFA88F8CA1AC8F13C0802FB46
:10B2700008F85FFA83F9AAFB082809EB58188C46EE
:10B280005FFA88F80F46012100930191434659E780
:10B29000AAFB0C025209C2EB0212ACEB820292B280
:10B2A000CF1A02FB07F7AAFB07275FFA83F909EB1E
:10B2B00057171A46FFB20B46884601210092BC463A
:10B2C00001913FE7AAFB0C025209C2EB0212ACEB60
:10B2D00082091FFA89F9CA1AC9F13C0902FB09F966
:10B2E000DFB2AAFB092907EB59195FFA89F99C46D5
:10B2F00088460B460121CDF80090019122E7A1EB91
:10B3000003080CFB08F8DFB2AAFB082807EB581863
:10B310005FFA88F89C46012301938946434611E76A
:10B320004346CDF80090BC460CE700BFD870002023
:10B33000D0810020898888882DE9F041284F002499
:10B340003B461D79212D03F1140304D001340F2C49
:10B35000F7D1BDE8F08104EB840007EB8000F6F73D
:10B360001DFFDFF888800646C8F8EC0B0028F0D0F7
:10B370002846FFF7A1F9C8F8F00B58B1142202FBD8
:10B38000047440F21722C28000220272227A4A21FB
:10B39000FFF78AFB134A03213046F6F79BFFD8F8E4
:10B3A000EC0B0021F7F712F80F49D8F8EC0B40F23C
:10B3B0002A325DF01DF810B988F8E80BC9E740F6AD
:10B3C000A8420948002166F0FAFDD8F8EC3B1B7C46
:10B3D000012288F8E82B002BBBD1BDE8F0418DE6B7
:10B3E00080100020009F24000C810020D0810020CC
:10B3F000437913F0010306D0D0E90731C268581A27
:10B40000531E184070471846704700BF437913F029
:10B41000020307D0D0E9093200699B1A013820EAFB
:10B4200003007047184670474379024613F0010045
:10B4300018D010B4D168146AD369481E1B1B03408E
:10B440000CD053691B5D04F1010CD8B2BCFBF1F3C5
:10B4500001FB13C15DF8044B1162704718465DF89B
:10B46000044B7047704700BF43799B070AD5436A76
:10B470008269D154436A02690133B3FBF2F102FBE2
:10B4800011334362704700BF41717047D0E9092012
:10B49000101AB0FA80F04009704700BF014B1B68DA
:10B4A0005B68184710C80020024B1B6808309B6877
:10B4B000184700BF10C800200120704701207047C6
:10B4C000012070470120704731B10C4BD3ED017A58
:10B4D000F8EEE77AC1ED007A72B1084BDFED086A49
:10B4E0009B68A3F5D543333B07EE903AF8EEE77A35
:10B4F00087EEA67A82ED007A704700BF10C8002060
:10B500000000C8420120704701207047704700BF0B
:10B51000044B03EBC00040F2FF739942A8BF1946E9
:10B520000182704710C80020174B184A9B7982F897
:10B530006C30032B1DD9191F022917D8052B10B405
:10B540001AD0062B14BF4FF47A614FF47A519FED55
:10B550000C7B00240E480F4BD467B3FBF1F382ED54
:10B56000207B5DF8044B1067936770470A4B1367A5
:10B5700070470A4B136770474FF4FA51E7E700BF73
:10B5800000000000000000006890002010C80020AB
:10B5900011B5000840420F000DB5000839CB000876
:10B5A000044B03EB8000D0F888300BB19B68196026
:10B5B000704700BF10C8002010B5D94C04EB8003C1
:10B5C000D3F888300BB19B6819600F282ED8DFE8BC
:10B5D00010F02E0049006C009300B600D900000165
:10B5E000230141015C017F01AB01CE01F101180291
:10B5F0001000C900CB48A1F5DB511C3980FB01309C
:10B60000C917C1EB600040F21472AD21FAF712FFC6
:10B6100094F8DD3000F0070203F01F0343EA421301
:10B62000C0F3C70084F8DD3084F8DE0010BDC90027
:10B63000BC48A1F5DB511C3980FB0130C917C1EBB7
:10B64000600040F21472AD21FAF7F4FE94F8CA30AB
:10B6500084F8C900C0F3022223F00703134384F8DF
:10B66000CA3010BDC900AF48A1F5DB511C3980FBC1
:10B670000130C917C1EB600040F21472AD21FAF736
:10B68000D9FE94F8CA2094F8CB3000F01F0102F0E4
:10B690000702C0F3451023F03F0342EAC1021843FA
:10B6A00084F8CA2084F8CB0010BDC9009D48A1F5DC
:10B6B000DB511C3980FB0130C917C1EB600040F23F
:10B6C0001472AD21FAF7B6FE94F8CB2094F8CD3081
:10B6D00000F0030102F03F0242EA811223F001036D
:10B6E000C0F380210B43C0F3870084F8CB2084F89B
:10B6F000CC0084F8CD3010BDC9008A48A1F5DB51DB
:10B700001C3980FB0130C917C1EB600040F2147294
:10B71000AD21FAF78FFE94F8CD2094F8CE3000F0EA
:10B720007F0102F00102C0F3C31023F00F0342EACD
:10B730004102184384F8CD2084F8CE0010BDC90022
:10B740007848A1F5DB511C3980FB0130C917C1EBEA
:10B75000600040F21472AD21FAF76CFE94F8CE202E
:10B7600094F8CF3000F00F0102F00F02C0F3061082
:10B7700023F07F0342EA0112184384F8CE2084F8B4
:10B78000CF0010BDC9006748A1F5DB511C3980FB13
:10B790000130C917C1EB600040F21472AD21FAF715
:10B7A00049FE94F8CF2094F8D13000F0010102F066
:10B7B0007F0242EAC11223F00303C0F341210B438D
:10B7C000C0F3470084F8CF2084F8D00084F8D1304B
:10B7D00010BDC9005348A1F5DB511C3980FB013075
:10B7E000C917C1EB600040F21472AD21FAF722FED6
:10B7F00094F8D12094F8D23000F03F0102F0030217
:10B80000C0F3841023F01F0342EA8102184384F836
:10B81000D12084F8D20010BDC9004248A1F5DB5107
:10B820001C3980FB0130C917C1EB600040F2147273
:10B83000AD21FAF7FFFD94F8D23000F0070203F0D3
:10B840001F0343EA4213C0F3C70084F8D23084F8E0
:10B85000D30010BDC9003348A1F5DB511C3980FB72
:10B860000130C917C1EB600040F21472AD21FAF744
:10B87000E1FD94F8D53084F8D400C0F3022223F01F
:10B880000703134384F8D53010BDC9002548A1F53E
:10B89000DB511C3980FB0130C917C1EB600040F25D
:10B8A0001472AD21FAF7C6FD94F8D52094F8D6307D
:10B8B00000F01F0102F00702C0F3451023F03F0320
:10B8C00042EAC102184384F8D52084F8D60010BD9E
:10B8D000C9001448A1F5DB511C3980FB0130C917A0
:10B8E000C1EB600040F21472AD21FAF7A3FD94F8A9
:10B8F000D62094F8D83000F0030102F03F0242EA6B
:10B90000811223F00103C0F380210B43C0F38700B1
:10B9100084F8D62084F8D70084F8D83010BD00BF52
:10B9200010C8002067666666C9004748A1F5DB516C
:10B930001C3980FB0130C917C1EB600040F2147262
:10B94000AD21FAF777FD94F8D82094F8D93000F0BB
:10B950007F0102F00102C0F3C31023F00F0342EA9B
:10B960004102184384F8D82084F8D90010BDC900DA
:10B970003548A1F5DB511C3980FB0130C917C1EBFB
:10B98000600040F21472AD21FAF754FD94F8D9200A
:10B9900094F8DA3000F00F0102F00F02C0F3061045
:10B9A00023F07F0342EA0112184384F8D92084F877
:10B9B000DA0010BDC9002448A1F5DB511C3980FB19
:10B9C0000130C917C1EB600040F21472AD21FAF7E3
:10B9D00031FD94F8DA2094F8DC3000F0010102F037
:10B9E0007F0242EAC11223F00303C0F341210B435B
:10B9F000C0F3470084F8DA2084F8DB0084F8DC30F8
:10BA000010BDC9001048A1F5DB511C3980FB013085
:10BA1000C917C1EB600040F21472AD21FAF70AFDBC
:10BA200094F8DC2094F8DD3000F03F0102F00302CE
:10BA3000C0F3841023F01F0342EA8102184384F804
:10BA4000DC2084F8DD0010BD67666666F0B54D4EFB
:10BA500096F8E13083B03BB196F8E250012D0446F0
:10BA60005ED0022D3ED00DB103B0F0BD0122802189
:10BA70000068454FFCF706FC01223870FF21206862
:10BA8000FCF700FC2A46387029462068FCF7FAFBD0
:10BA900096F8E320387091212068FCF7F3FB2946E3
:10BAA000387001222068FCF7EDFB2A463870FF2130
:10BAB0002068FCF7E7FB2A46387080212068FCF7F5
:10BAC000E1FB29460346012220683B70FCF7DAFBC4
:10BAD0002E4A38701268C6F8E420012386F8E23056
:10BAE00003B0F0BD0068284F01AA1321FDF7BAFC8E
:10BAF0009DF8043038705B0725D1D6F8E830002B6C
:10BB0000B2D0224AD6F8E410126892B2521A934286
:10BB1000AAD24FF0FF3200237A6086F8E230A3E722
:10BB200001AA0068184F0021FDF79CFC9DF8043025
:10BB30003870DA07E1D4154A02231268C6F8E42007
:10BB400086F8E23090E720682B4601AA1E21FDF717
:10BB50005BF9BDF8043002460B2120683A700122DF
:10BB60005CBAFCF78FFB0A4B3870A4B2A3FB043419
:10BB7000E408012200237C6086F8EC2086F8E2309D
:10BB800072E700BF10C80020481400205435002080
:10BB9000CDCCCCCC0C4A13787BB10C4B93F8E11094
:10BBA00059B193F8EC1059B150680022FA2883F883
:10BBB000EC20A8BF4FF0FF3070476FF001007047D6
:10BBC0006FF00200704700BF4814002010C800202A
:10BBD0002DE9F041114C04F1F00884F8F1101746FA
:10BBE000002502234246FF21064684F8F050FDF767
:10BBF00093F880B1424630460223FF21FDF704F955
:10BC000048B194F8F02094F8F13003EB0223284671
:10BC10003B80BDE8F0816FF00C00FAE710C800200F
:10BC20000B4B93F8F02182B193F8F12152B10949FD
:10BC300088680022B0F5967F83F8F121A8BF4FF005
:10BC4000FF3070476FF0020070476FF001007047DF
:10BC500010C8002048140020024BD3F8F4315B6870
:10BC6000184700BF10C80020024BD3F8F4319B687E
:10BC7000184700BF10C80020024BD3F8F431DB682E
:10BC8000184700BF10C80020014BD868704700BF9C
:10BC900048140020044B93F8F83113B1034B186992
:10BCA00070476FF00100704710C800204814002052
:10BCB000437A5A1C0344D2B242729972037A934275
:10BCC00000D97047002AFCD010B5044604F10A01DF
:10BCD000D0E9003098470023637210BD08B5284BA7
:10BCE000284ED3F8FC51B0682CF042FB28462CF0CB
:10BCF0003FFBB06841798B073BD500210846FFF731
:10BD0000EBF900210120FFF7E7F91F4CB068036849
:10BD10005B689847C8B92B6828465B689847002835
:10BD2000F4D0D4F89C202B68B4F8A010DB685183C1
:10BD3000284698470146B068026813689847D4F8C7
:10BD40009C30B4F8A0201A83E0E7B068D4F8A820AB
:10BD50000368B4F8AC10DB68518398472B68014640
:10BD60001B6828469847D4F8A830B4F8AC201A834A
:10BD7000D1E7036841F002019B699847BDE700BF26
:10BD800010C80020E8910020C82A00202DE9F04FBB
:10BD9000B44D002605F5007C95F84412A5B00A24A0
:10BDA0003346E64637469BE002EBC70205EB42000E
:10BDB000C2F30727B0F8480210F0040F5FFA82FEC2
:10BDC000C6B24FEA102900F0C480480614D403F12B
:10BDD0000208B8F18C0F41F0400100F2FC800DF137
:10BDE000900A581C53444FF0040A03F88CAC24AB5F
:10BDF000034403F88C1C434603F10208B8F18C0F8E
:10BE000047F0020B00F2E78024A8184400F88BBC2E
:10BE10004FF0050B00F88CBC03F1040BBBF18C0F49
:10BE200000F2D9800DF1900AD044B6004FF0060A16
:10BE300008F88CAC5FFA86F89E1D8C2E00F889EC11
:10BE400000F2C9800DF1900AD3444FF0070A0BF8B5
:10BE50008CAC00F8878C03F10808B8F18C0F00F265
:10BE6000BA800DF1900B5E444FF0050B06F88CBCC8
:10BE700003F10A068C2E00F8857C00F2AC8024AF1A
:10BE8000B8444FF0060A08F88CAC00F883EC03F1D4
:10BE90000C008C2800F29F800B333B443E444FF053
:10BEA000070A06F88CAC03F88C9C0346570902F08D
:10BEB0001F00012686405CF82700013C20EA0600AE
:10BEC0004CF8270000F08A80561CB6F5F07F80F011
:10BED000858072090CEB820E9700634A96457DD2ED
:10BEE00006F01F024FF0FF30DEF8006000FA02F2A9
:10BEF000324092FAA2F2B2FA82F2D2B2202A7FF44F
:10BF000053AF594A0EF1040090421AD2574AA2EB9D
:10BF10000E0727F003070EF1080E774401E0B84240
:10BF20000FD006460430326892FAA2F2B2FA82F2D8
:10BF3000D2B2202AF3D0A6EB0C0612EBC6027FF594
:10BF400035AF85F844121846002B49D125B0BDE81D
:10BF5000F08F11F0400F03D101F03808B04513D035
:10BF600021F078019E1C01438C2EC9B233D80DF10B
:10BF70009008581C43444FF0040803F88C8C24AB01
:10BF8000034403F88C1C3346981C8C2823D824AE19
:10BF900006EB03084FF0050608F88C6C1E1D8C2E6E
:10BFA00008F88B7C17D824AF38444FF0060700F808
:10BFB0008C7C981D8C2808F889EC0CD824AF3E4462
:10BFC0004FF0070706F88C7C053324AE334403F8A2
:10BFD0008C9C03466AE76FF0004367E785F84412DC
:10BFE000D5F83C42224894F91020A16802EB820265
:10BFF00050F822008A0722D501AA00215FF042F8FA
:10C00000A3689B0703D5012025B0BDE8F08F194B2D
:10C0100019491A68194B4FF4FA7000FB02F2A3FB9E
:10C020000232486892094B681B1A9A42FBD2636934
:10C03000002BE8D01A689B881383012086E7626989
:10C0400012B1116892884A830A4A0B4D11680B4A53
:10C050006E68C900A2FB012189096A68921B91429E
:10C06000FBD2C9E710C800204CCA002047CA0020F4
:10C07000481200207C360020001000E0D34D6210F2
:10C08000F0B541F0010285B000212A4F2A4D2B4E18
:10C090000446FCF7F7F83B68C6F8E430287016E071
:10C0A000A368DB070DF10F024FF0130120465EBFBE
:10C0B0000DF10F0293212046FDF780F99DF80F3016
:10C0C000287013F007030ED1D6F8E8204ABB237975
:10C0D000012B18D0022BE3D09DF80F30002013F075
:10C0E00007032870F0D001220B212046FCF7CAF884
:10C0F00000220346114620462B70FCF7C3F8287037
:10C10000012005B0F0BDA268617C94F9100002F036
:10C11000010201920DF10F0200921322F7F760FB6A
:10C12000CCE73968D6F8E40089B2091A8A42CED23F
:10C130001846E6E7543500204814002010C80020B7
:10C140002DE9F04F7E4B93F84252C7B005B1FEE7A0
:10C150007B4A92F84372012382F8423207F0F707D4
:10C16000D2F83C3282F8437203931B79012B0446C8
:10C170000E4600F0A280022B40F09D800398836859
:10C1800013F0010118BF29463A46FCF729F86C4B19
:10C19000D3F83C32039305ADFF2C4FF009036C70CC
:10C1A00088BFA4082B708CBF04F0C0084FF00008B3
:10C1B000022300204FF00A0B0DF1150A4FF00B0976
:10C1C00012E0BEF5827F05F803B016F800C00AF849
:10C1D000032015D80130362805F8049001F1060136
:10C1E00005F807C0734612D09C1C48EA0002B4F55B
:10C1F000827F03F1040E1946D2B203F10307E0D99E
:10C2000001306FF0004E36284E497346ECD1B1F53F
:10C21000827F00F2918008210DF1150205F80E10C1
:10C22000A021D1540233039C474994F9102002EB1A
:10C23000820251F82200A26892076AD52A4600219C
:10C240005EF020FF039B9B689B074AD53C4B3F4D0C
:10C25000D3F83C020379012B0DF1130419D0022B02
:10C2600008D12246A021FDF7A9F818B1237813F0D0
:10C2700020031AD0D5F8A830B5F8AC2059690A4285
:10C2800014BF5A831A832E4BD3F83C020379012B37
:10C29000E5D18268417C90F9100002F00102CDE9FD
:10C2A0000042A022F7F79CFADFE7254A82F84232E3
:10C2B00047B0BDE8F08F05AD6EE7039881682A4668
:10C2C00001F00105014690F91000497C019505AD8A
:10C2D0002F700095F7F7B8FA194BD3F83C32039357
:10C2E0005AE71B4B1B491A681B4B48684FF4FA74FA
:10C2F00004FB02F2A3FB023292094B681B1A9A421A
:10C30000FBD2039B5B69002BA0D01A689B88138328
:10C310009CE7626912B1116892884A830C4A0D4CFD
:10C3200011680D4A6668C900A2FB0121890962688B
:10C33000921B9142FBD281E76FF0004373E700BF8D
:10C3400010C800200100008048120020C82A0020E8
:10C350007C360020001000E0D34D621038B58368B1
:10C360001C686379DB0748D5A37994F85C2203F055
:10C3700001010D461ABB94F85F32012B3ED0002B11
:10C3800040D194F85E3294F85DC263450DD2B4F8A2
:10C3900066224FF0010E0EFA03F001330243D8B2C9
:10C3A000604592B2F7D3A4F86622012384F85F3285
:10C3B000E06B85EA0301BDE838405BF01FBEE06B2F
:10C3C00043681A68D36AC3F34E03536294F86D321C
:10C3D000012B07D094F8613223B1B4F868320133ED
:10C3E000A4F8683285F001015BF008FE00224FF0EE
:10C3F0008073A4F86622C4F85C3238BD94F85D32CC
:10C4000084F85E32002384F85F32E06BBDE8384088
:10C410005BF0F4BD30B5032083B00D461446FBF746
:10C4200033FE01909DB107EE900A9FED0B7AF8EE76
:10C43000677AF0EE006A67EE877AB8EE047AA7EEC4
:10C44000A67ADFED067A67EE277AC5ED007A0CB1A1
:10C45000034B236003B030BD6740533A00007A4479
:10C460003313904300B500680379012B85B00DD0DC
:10C47000022B07D1012303AAFF21FCF76FFC05B0B3
:10C480005DF804FB002005B05DF804FB8268417C88
:10C4900090F9100002F00102019203AA0092FF221B
:10C4A000F7F79EF905B05DF804FB00BF30B5044610
:10C4B00000680379012B85B029D0022B1ED1826838
:10C4C00012F0010F18BF512103AA08BFD121FCF7B8
:10C4D00045FC98B1BDF80C30194A5BBA9BB2D360E9
:10C4E000D368B3F5C87F0EDC1649174AD1F8083671
:10C4F00015683233AB4218D305B030BD104B6FF026
:10C500000102DA60F0E74FF0FF33D360ECE78368B5
:10C51000417C90F9100003F00103019303AB0093F9
:10C5200051220223F7F75CF9D3E701F20C62C1F85C
:10C530000856206800235121FCF7EEFB05B030BD02
:10C540004814002010C800205435002000B50068B1
:10C550000379012B85B008D0022B2FD0204B00226D
:10C5600083F8F82105B05DF804FB8368417C90F9FD
:10C57000100003F0010303AACDE9002302230022E7
:10C58000F7F72EF9164B83F8F8010028EAD0BDF82A
:10C590000C305BBA9BB2B3F5FA6F1AD21149124A4A
:10C5A000A1FB0313DB0807EE903AF8EEE77AFDEE05
:10C5B000E77AC2ED047A05B05DF804FB826812F0F8
:10C5C000010F18BF002103AA08BF8021FCF7C6FB9A
:10C5D000D8E7054B4FF0FF321A6105B05DF804FB58
:10C5E00010C80020CDCCCCCC4814002010B5006879
:10C5F0000379012B84B00C461DD0022B18D1826820
:10C6000012F0010F14BF0021802103AAFCF7A6FB42
:10C6100060B15CB19DF80D309DF90C20DB0903EB96
:10C62000830302EB820203EB4203238004B010BDBC
:10C63000002004B010BD8368417C90F9100003F025
:10C640000103019303AB009300220223F7F7C8F81C
:10C650000028DED1EAE700BF70B50668F56982B050
:10C660000446002D50D000232B7004230DEB030251
:10C670003046FF21FCF7C8FB10B9002002B070BDA6
:10C68000206804236A46FF21FCF7BEFB0028F4D093
:10C690009DF804108A09023A012AEED99DF8053066
:10C6A0009DF800409DF8012003EB012302EB0422DA
:10C6B000C3F30D03C2F30D02991A0029B8BF494212
:10C6C000FF29DADC9DF802409DF803109DF8066012
:10C6D00001EB04214C119DF8071001EB0621C4EB7E
:10C6E0005116002EB8BF7642FF2E4FEA6111C4DC0E
:10C6F000134421445B104910C5F805300123C5F8E7
:10C7000001102B7002B070BD0C211420FAF730FE1E
:10C71000F06105462668A6E770B50568E8690C462D
:10C720001646A0B3D0F80130CCB1D0F805209FED6B
:10C730001B7ADFED1B5ADFED1B6A07EE902AF8EE3D
:10C74000677AB7EE006A77EEC77A77EEA77A87EE58
:10C75000A57A77EE467A67EEE67AC4ED007AAEB156
:10C7600007EE903A9FED107ADFED106A9FED106AA8
:10C77000F8EEE77A67EE877A87EEA67ADFED0D6A44
:10C7800077EE467A77EEA67AC6ED007A70BD0C2178
:10C790001420FAF7EDFDE861C4E700BF9AC9CC4464
:10C7A0009AC94C460E76D7450000484300E0FF4446
:10C7B000000048423393884370B52DED048B344B11
:10C7C0001B7E022B0C46154618D0DFED327A7CB169
:10C7D0009FED317A9FED316ADFED316A67EEA77A1E
:10C7E00067EE877A87EE867A77EE267AC4ED007A4E
:10C7F0000DB12C4B2B60BDEC048B70BD2A4B93F814
:10C800001C2622B9D3F81836D3ED357ADFE703F2C8
:10C810000C63D3ED008A93ED019A244EF0EE680A82
:10C82000B0EE490AF9F722FDB5EEC00AF1EE10FAB2
:10C8300048BFDFED1F7AB0EE408AF0EE490A48BFEC
:10C8400030EE278AB0EE680AFAF7D8FBDFED196AF6
:10C850009FED197AD6F8E82328EE268AC8EE077AE3
:10C86000B0EE408AFCEEE77A17EE903A9BB29B1A44
:10C8700007EE903AF8EEE77A87EEA60A20EE070A6E
:10C88000F9F718FBD6EDFE7AE0EE487A9FE700BF95
:10C8900060A6002000000000CDCC9C3F00409C46DC
:10C8A00082E6C5473313904310C8002000B800202B
:10C8B000DB0FC9400000C84235FA8E3C2DE9F04F2D
:10C8C00087B099469DF84430BDF840B001930746C3
:10C8D0008A469046F5F762FC0446002800F09480F2
:10C8E000594E96F81D560A2D00F29E805C2303FBDC
:10C8F00005630022C3F8202683F824263A79130919
:10C90000691C013BC9B2032B86F81D16029102F087
:10C910000F0C42D84D4A039332F8130040FA0CF240
:10C92000D3073AD5012202FA0CF2013A10405FF027
:10C93000A3FB474A039B0299D35C464A184400EB89
:10C94000400002EB80034FF0020C1972019983F84A
:10C9500006A083F807C000FA0CFA002958D15AF84B
:10C9600002103D48019301F13F4101F57E01890A22
:10C97000405C5BF0DBFA019B364A998804914FF0EA
:10C98000011152F80A00059104A9F6F76DF8314A31
:10C99000019B5AF802209B8853835C2707FB05679D
:10C9A000424649462046C7F82046F5F793FC5946CB
:10C9B000D7F82006F5F70AFDD7F8203659680B6836
:10C9C000B3F844206FEA42426FEA524292B2A3F8AF
:10C9D00044201A8892B242F001021A804A79032A4E
:10C9E00029D8DFE802F01B1D1F02403305EB45008C
:10C9F0005C22C5EBC000194C02FB05650022C5F89E
:10CA0000283604EB80041A60204607B0BDE8F08F9A
:10CA10003A7A61461846FEF747F8BEE73433E5E751
:10CA20003833E3E73C33E1E70D4A00210420FAF70D
:10CA3000BFFB0024E8E75C22002302FB0565C5F884
:10CA400028361B60FFDE00BF10C800202033070817
:10CA500028330708C82A0020C021070830CE00204C
:10CA600068C4070830B503682F4C2DED028BA34234
:10CA700083B0F0EE408AB0EE608A13D004F5806493
:10CA8000A3420FD004F57054A3420BD004F5806488
:10CA9000A34207D004F58064A34203D0234B1C6853
:10CAA000640801E0214B1C680192B4FBF1F202F52D
:10CAB0007F420023FF32120C0093B4FBF2F4B4FB6C
:10CAC000F1F52246ABB20421FFF7F8FED0B1B5EE86
:10CAD000408AF1EE10FA19D0DFED150A07EE904A00
:10CAE00068EE200AF8EE677A60EEA70A9FED117AE9
:10CAF000C0ED040A27EE607A0123A8EEA77A03713D
:10CB000080ED037A03B0BDEC028B30BD07EE905A86
:10CB1000DFED070AB8EE677A07EE904A67EE200A63
:10CB2000F8EE677AE2E700BF000001407C0E0020CB
:10CB30006F12833A00007A4410B50B4B03EBC00030
:10CB400082B0C46801916CB107EE901A94ED047A3A
:10CB500094ED030AF8EEE77AA7EE870A62F008F888
:10CB6000A368186002B010BD10C800202DE9F04382
:10CB7000324E96F86C3083B00D46062B59D8DFE85C
:10CB800003F029473B4204040400052B45D02C49FF
:10CB90002C4C062B08BF21464FF000080192CDF81F
:10CBA00000800A4614230421FFF788FE0746002868
:10CBB0003DD08146122259F8140B49465BF018FC0F
:10CBC000044660BB012406EBC505EF60204603B0B8
:10CBD000BDE8F083DFED1C0A4FF4C871B0EE600AC7
:10CBE000FFF740FF06EBC505041E18BF0124E860EF
:10CBF000204603B0BDE8F083DFED140A9FED140A70
:10CC00004FF4FA61ECE7134BDFED130A9988E5E77F
:10CC1000DFED120A4FF47A71E0E71149BCE74146B3
:10CC20004846482265F0CBF901233B71CBE7044627
:10CC3000C9E706EBC5050024EC60C7E710C8002073
:10CC4000C0C62D00001BB7006F12833AACC5A737D2
:10CC5000ACC5A73668900020000000006F120339B1
:10CC6000808D5B0010B5174C84F8F110017984F8C1
:10CC7000F22001294FF0000282B084F8F02012D097
:10CC800002290CD1032304F1F002FF21FBF7EEFF90
:10CC9000002814BF00206FF00C0002B010BD6FF030
:10CCA0000C0002B010BD8268417C90F91000F03495
:10CCB00002F00102CDE900420323FF22F6F7C4FD92
:10CCC000E6E700BF10C8002000680379012B0BD0F5
:10CCD000022B08D183680F4A13F0010316D00023FA
:10CCE0005121FBF7C3BF704700B58368094A417CF7
:10CCF00090F9100083B003F00103CDE90023002375
:10CD00005122F6F7A1FD03B05DF804FBD121FBF73A
:10CD1000ADBF00BF1CCE002030B5184D95F8F031E6
:10CD200083B00BB903B030BD04460DF105010068B6
:10CD30005DF0B0F99DF8053073B901212068104A03
:10CD400085F8F2104FF406440323FF21A5F8F040C4
:10CD5000FBF7E2FF03B030BD0DF10602962120681B
:10CD6000FEF736FF074ABDF806300749A2FB03234A
:10CD7000DB0801228B6085F8F121DEE710C8002076
:10CD800000C90020CDCCCCCC481400202DE9F041C6
:10CD9000DFF8608004460F46164600252046202115
:10CDA00065F024F90446E0B103461C4613F8010B74
:10CDB0002028FAD02046FAF75DFF40F634024FF4FF
:10CDC0006171F9F737FBA0F5617088FB0023C0178C
:10CDD000C0EBE300302804D84DB1787033780133CC
:10CDE00033700DB90125D9E72046BDE8F0813870D0
:10CDF000F4E700BF1F85EB51084B93F841224AB17D
:10CE000093F8433213F0400F14BF4FF4F0704FF417
:10CE1000C37070474FF4F070704700BF10C8002017
:10CE2000054B93F8410230B193F8433213F0400FB1
:10CE30000CBF0D201020704710C800202DE9F041D4
:10CE400013238CB00446002229210220FDF76AFE3C
:10CE5000704DC5F83C02002800F0A3800221FBF7CA
:10CE600071F902220021D5F83C02FBF70BFA0023EE
:10CE700085F8443285F8404205F5127305F5C16125
:10CE80004FF0202243F8042B8B42FBD1624FDFF896
:10CE90008C813E683236D5F83C422379012B00F074
:10CEA0008380022B11D1A3685C4ADB074FF080011D
:10CEB00020465EBF594A80212046FCF77FFA10B118
:10CEC0003B689E42E7D8D5F83C4211224FF0100E45
:10CED0004FF0120C132714261525162017218DF854
:10CEE0000E20192201238DF80CE08DF810C08DF86A
:10CEF00012708DF814608DF816508DF818008DF8AA
:10CF00001A101E201F218DF81E204FF0180E4C22E3
:10CF10004FF01A0C1B271C261D258DF80D308DF89F
:10CF20000F308DF811308DF813308DF815308DF8E5
:10CF300017308DF819308DF81B308DF81D308DF8B5
:10CF40001F308DF821308DF823308DF825308DF885
:10CF500027308DF828008DF829308DF82A108DF8AB
:10CF60002B308DF81CE08DF820C08DF822708DF8E4
:10CF700024608DF826508DF82C308DF82D2094F9F2
:10CF80001030A268264903EB8303920751F823006F
:10CF90002DD5222303AA00215EF074F8A3689B0715
:10CFA0000ED50CB0BDE8F081A268617C94F9100048
:10CFB00002F00102CDE900828022F6F711FC7EE743
:10CFC000184B19491A6848684FF4FA7303FB02F2C8
:10CFD0004FF47A73B2FBF3F24B681B1A9A42FBD2FE
:10CFE0006369002BDDD01A689B881383D9E76369D6
:10CFF00013B11A689B8853830A4B0B491A684D6812
:10D00000D2004FF47A73B2FBF3F24B685B1B9A4287
:10D01000FBD2BEE710C800205435002053CA0020C0
:10D02000481200207C360020001000E0104A70B545
:10D03000002302F570744FF40056A2F146054FF03C
:10D04000010E32F8020F03F01F01B0F5005F4FEA46
:10D05000531C0EFA01F103F1010305D055F82C0021
:10D060001680014345F82C10A242EAD170BD00BFE2
:10D0700056CA00204FF01E0C43EA0223FF2A0CFB85
:10D0800001011BB288BF43F00403B1F5F07F07DA5A
:10D090000C4A02EB41009BB2B0F848C29C4500D15B
:10D0A00070474FEA511C02F50072A0F8483201F0B7
:10D0B0001F0152F82C30012000FA01F10B4342F815
:10D0C0002C30704710C800204FF01E0C0CFB0101E3
:10D0D000B1F5F07F01DB002070470B4800EB410108
:10D0E000B1F84812080AC9B210801970490709D569
:10D0F000118841F4807111801A7822F00402012015
:10D100001A7070470120704710C800202DE9F047C1
:10D110001E2404FB010114787CB31D282DDC184E5D
:10D120000FFA83FE06EB410CC1F10105483E0127D1
:10D1300001E01D2B21DCB1F5F07F4EEA042405EB64
:10D14000010311D2BCF800A001F01F08A2454FEA6C
:10D15000511907FA08F807D0ACF8004056F82940F2
:10D1600044EA080446F8294012F8014FDBB20CF1FA
:10D17000020C03440131002CDBD1BDE8F08700BF75
:10D1800058CA0020F0B5534CD4F83C5285B015B1C4
:10D1900094F842320BB105B0F0BD012384F842325D
:10D1A0002B79012B7BD0022B37D128460DF10E02B3
:10D1B0008421FCF703F9D4F83C522B7994F84422EB
:10D1C000012B42F004027BD18DF80F20AA6895F95B
:10D1D0001000697C02F0010201920DF10F02009231
:10D1E0000422F6F731FB15E0022B0ED1AB6813F0E9
:10D1F000010F0DF10E024FF08401284602BF0DF120
:10D200000E0284212846FCF7D9F89DF80E3013F061
:10D21000040616D0D4F83C522B79012BE4D1AA682D
:10D22000697C95F9100002F0010201920DF10E02E5
:10D2300000928422F6F7D4FA9DF80E3013F004061B
:10D24000E8D1254D254884F8443231463C2264F02B
:10D25000B6FE05F570773146A5F1460E012635F884
:10D26000023F1A0A22F0200203F0040301F01F001B
:10D2700013434FEA511C06FA00F001F1010104D0FA
:10D280005EF82C3018434EF82C00BD42E7D1FEF773
:10D290007DFD0028FBD184F8420205B0F0BDAA68EC
:10D2A000697C95F9100002F0010201920DF10E0265
:10D2B00000928422F6F794FAD4F83C522B797DE759
:10D2C000022BAAD128460421FAF78AFFD4F83C524F
:10D2D0002B79A2E710C8002056CA002010CA0020EF
:10D2E00070B54A4DD5F83C4284B08CB395F84032C5
:10D2F000012B40D0022B2DD1082294F91030444844
:10D3000085F8432203EB8303042150F823008DF8B2
:10D310000D2000238DF80C30A3688DF80E109A07AD
:10D320008DF80F1040D5042303AA00215DF0AAFE5A
:10D33000A3689B0721D537483C22FF2164F03FFEBC
:10D3400095F8413223B9FFF71DFF012385F84132DB
:10D3500004B070BD2379012B4AD0022B37D09DF841
:10D360000B3003F00503012B3ED0002B36D1D5F84E
:10D370003C420822C1E74822BFE7274B27491A68E9
:10D38000274B48684FF4FA7606FB02F2A3FB023201
:10D3900092094B681B1A9A42FBD26369002BCAD0D0
:10D3A0001A689B881383C6E7636913B11A689B8860
:10D3B0005383194B19491A68194B4E68D200A3FBC5
:10D3C000023292094B689B1B9A42FBD2ABE70DF1EC
:10D3D0000B02A0212046FBF7F1FFC0E7114A1268BB
:10D3E00040F2DC539A42B3D9D5F83C42482284E754
:10D3F000A268617C94F9100002F0010201920DF123
:10D400000B020092A022F6F7EBF9A8E710C8002063
:10D410004812002010CA00207C360020001000E0D6
:10D42000D34D62105435002030B5484CD4F83C52EE
:10D4300085B095B194F84332180702D594F842327A
:10D440006BB194F8413243B9FFF74AFF94F8413287
:10D45000002B40D1002384F8423205B030BD94F84F
:10D460004132012284F84222002BEDD02B79012B8E
:10D4700034D0022BE8D10DF10E0280212846FBF7B3
:10D480009DFF0028E0D094F843229DF80E309A4288
:10D49000DAD194F84032002BD8D12D4AD4F8143A7E
:10D4A0001568EB1AB3F57A7FD0D9D4F83C0203792A
:10D4B000012B34D0022B04D10DF10F02A021FBF778
:10D4C0007DFF9DF80F30590716D50023C4F8183A90
:10D4D000C4F8145ABAE7FEF759FCBBE7AA68697C9E
:10D4E00095F9100002F0010201920DF10E02009276
:10D4F0008022F6F775F9C4E703F00503012B1CD071
:10D50000002BE5D194F843325B06E1D5D4F8183A04
:10D51000C3B1EB1A642BDBD9FFF7E2FED8E78268D0
:10D52000417C90F9100002F0010201920DF10F020E
:10D530000092A022F6F754F9C3E794F843325A0652
:10D54000E4D5C5E7C4F8185AC2E700BF10C80020E8
:10D55000543500202DE9F0439E4ED6F83C4285B06C
:10D56000002C6DD096F84292B9F1000F00D0FEE782
:10D5700096F843C201230CF0F70C86F843C286F8F4
:10D5800042322379012B05460F4600F0DB80022B47
:10D5900000F09680B0F5807F0DF10F0800F0FA8062
:10D5A000012B00F0E580022B07D1204650220821F4
:10D5B000FAF716FED6F83C422379874D012B1AD094
:10D5C000022B0AD142462046A021FBF7F7FE20B1EC
:10D5D0009DF80F4014F0200451D0D5F8A830B5F8CC
:10D5E000AC205969D6F83C420A4214BF5A831A83C8
:10D5F0002379012BE4D1A268617C94F9100002F038
:10D600000102CDE90082A022F6F7EAF8DFE7B9F1DE
:10D61000000F12D196F84342D6F83C5204F0F704BA
:10D6200086F843422B79012B00F0C080022B04D1F5
:10D63000224649462846FAF7D3FD002386F84232AF
:10D6400005B0BDE8F083022B16D162460A212846B8
:10D65000FAF7C6FDD6F83C020379012B07EB04026A
:10D6600028D18568417C90F9100005F00105CDE9CD
:10D670000025C022F6F7B4F80134362CC7D0D6F80E
:10D680003C522B79012B5FFA84FCDCD1AA6895F916
:10D690001000697C8DF80FC002F00102CDE9008214
:10D6A0000A22F6F7D1F8D6F83C020379012B07EBF2
:10D6B0000402D6D0022BDFD1C021FBF77FFEDBE7CF
:10D6C000494620466246FAF78BFDD6F83C4223795C
:10D6D00081460DF10F08012BEAB229D1A16894F916
:10D6E000100001F0010C617C8DF80F20CDF804C012
:10D6F000CDF800800922F6F7A7F8D6F83C42237946
:10D70000B5F5807F7FF44CAF012B43D1A26894F92B
:10D710001000617C02F00102CDE9008240228DF808
:10D720000F200A22F6F790F8D6F83C42237937E723
:10D73000022B49D120460921FAF752FDD6F83C4286
:10D740002379DDE7A16894F9100001F0010E0DF1D5
:10D750000F08617CCDF804E04A46CDF800808DF8D2
:10D760000FC0F6F771F8D6F83C4281462379B2E74C
:10D77000A26894F91000617C02F00102CDE90082F8
:10D7800050228DF80F200822F6F75EF8D6F83C42BA
:10D79000237912E7022B7FF410AF204640220A21A2
:10D7A000FAF71EFDD6F83C422379F9E6A96895F907
:10D7B000100001F001074A46697C8DF80F40CDE961
:10D7C0000087F6F741F838E7B5F5807F7FF4EBAED8
:10D7D0009AE700BF10C80020C82A0020034BD3F8E6
:10D7E0003C320BB1FEF7ACBC704700BF10C8002044
:10D7F00010B58379C26B13F0010F0446406B20D043
:10D8000013F0200F526814BF0221422120B1127A76
:10D81000FDF74AF9E36B5A68012384F86032A4F8F3
:10D820005C3250790B4C1168205C0A8C83409BB2AF
:10D8300092B222EA03020A840A8C92B213430B8446
:10D8400010BD13F0200F526814BF022122210028BE
:10D85000DDD1E1E79039070838B583681C68637942
:10D86000990745D4D90700D438BD94F85C32002B11
:10D87000FAD194F85D320133DBB2092B84F85D32C2
:10D8800000F0AC800A2BEFD194F85F52002D00F02D
:10D89000C480B4F86602820500F0010302D4002BB4
:10D8A00040F0C480B4F86A320133A4F86A3201232C
:10D8B0009D42A4F85C32D7D1A179E06B002384F8B3
:10D8C0005F3201F001015AF099FBE36B76485B6827
:10D8D0005A791968835C0A8C05FA03F39BB292B2F9
:10D8E00022EA03020A840A8C92B213430B8438BDE5
:10D8F00094F86112002967D1D4E90902904200F03E
:10D900009E80501CA569A062AA5C25695200A842AD
:10D9100034BF05460D4694F86002A56242F40072D9
:10D920000A254FF0010CA4F8642284F8625284F8AE
:10D9300061C2002850D0A07905071CD410F0400522
:10D9400090D009214FEA520CC00702F0010248BFF3
:10D9500082F00102A4F864C2002A57D1A26B12B16E
:10D9600010689288428384F86212002D3FF47AAFE7
:10D9700000292DD076E7E36B4B485D686B792A6808
:10D98000C35C606B0CFA03FC138C9BB223EA0C0C97
:10D99000A2F820C0138C9BB2138410B12A7AFDF731
:10D9A00083F8236CA06B002284F86022002B64D0E3
:10D9B00020B15B6801211A7AFDF776F8A37913F09C
:10D9C000400F63793FF44EAF94F9621200294CD1B5
:10D9D000002284F8612245E7A079AFE794F85F322E
:10D9E000002B7FF441AF94F85E32082B3FF63CAF3A
:10D9F000B4F86622012000FA03F101330A43D9B2D8
:10DA0000082992B2F7D9A4F8662238BDA26B002A81
:10DA1000A9D0106892880283A5E7B4F8663243F073
:10DA200001009B05A4F866023FF53CAFE36A40089D
:10DA30003BB3216BC0B2984794F85F5237E794F834
:10DA4000601200297FF40EAFA27912077FF50AAFAA
:10DA5000236CA06B23B318B15B681A7AFDF724F826
:10DA60002046FFF7C5FE6379FCE6A079B4F864228E
:10DA7000013949B200F0400564E70121F7F71CFFC6
:10DA80009CE7E3696269C0B2D054E369E26894F844
:10DA90005F520133B3FBF2F102FB1133E36106E79E
:10DAA0001946F7F709FFDBE79039070838B54368EF
:10DAB000344A1B68934204462BD002F5806293429D
:10DAC00027D002F57052934223D002F58062934230
:10DAD0001FD002F5806293421BD02B4B1A6852086C
:10DAE0001346B3FBF1FCBCF5803F15D21FFA8CF155
:10DAF0002046F4F7EFFB23681A6853790BBB937940
:10DB000073B963681A6813889BB243F001031380EA
:10DB100038BD1D4B1A68E3E7012BE4D95B08E0E749
:10DB20005AB2002A1FDB19480121851803F01F0390
:10DB3000520901FA03F3302185F8001340F822302E
:10DB4000DFE759B2002915DB104D012005EB010C70
:10DB500003F01F03490900FA03F330208CF8000397
:10DB600045F82130CBE70A4A03F00F031A4430236B
:10DB70001376C6E7064903F00F03194430230B76EA
:10DB8000BDE700BF000001407C0E002000E100E086
:10DB9000FCEC00E00346C06B996087E7002ABCBF3D
:10DBA00080185242002B30B53BDB5D180028B7BF10
:10DBB000121A841814460020A4F11D0C0029BCBFC1
:10DBC0002B460021BCF1000FC8BFA2EB0C04A5F14D
:10DBD0000F02C8BF2418002AC4BF9B1A5D188442D4
:10DBE0001EDBC1F1010C114AAC44C1EB0113CCEBBB
:10DBF0000C1C00EB430301344FEA4C0C02EB4302D4
:10DC00004FF0200E8D42A8BF002304DB22F813E062
:10DC10001E339C45FAD10130A04202F10202F1D13B
:10DC200030BD5C180D465B422146BFE758CA002054
:10DC30001B4B1C48196C1C4A10B441F08051012444
:10DC4000196404625321FF24CA2054625062516255
:10DC50005B6FDB0085B013D400231449029302915B
:10DC6000029A134804320292029A136003930391BA
:10DC7000039B0393039B186005B05DF8044B70474A
:10DC80000A4B002201920193019B0193019A084BD8
:10DC900012689A42E0D105B05DF8044B704700BFAE
:10DCA0000038024000000E4200280040502800408A
:10DCB00076614E692DE9F04F0023DFF8C492A84E3B
:10DCC000A84FDFF8C0A283B0C0E900330546019138
:10DCD00009F596789B464C46B279022A00F0B68048
:10DCE000012A00F0C480A04800228446014691F930
:10DCF0000430012B01F10C0140D00132082AF6D189
:10DD00009949002291F90430022B01F10C0142D013
:10DD10000132082AF6D19449002291F90430032BEC
:10DD200001F10C0144D00132082AF6D18E490022BB
:10DD300091F90430042B01F10C0146D00132082A7C
:10DD4000F6D1002290F90430052B00F10C0000F010
:10DD50009F800132082AF5D1844A1068410640F1BB
:10DD6000AD80494600220B79122B01F1140100F01D
:10DD7000CF8001320F2AF6D10022CDE002EB420221
:10DD80005CF82220002A3FD1774991F90430022B18
:10DD900001F10C01BCD102EB42025CF82220002A06
:10DDA0003ED1714991F90430032B01F10C01BAD134
:10DDB00002EB42025CF82220002A3CD16A4991F928
:10DDC0000430042B01F10C01B8D102EB42025CF8E3
:10DDD0002220002AB6D0664B227993F83D1093F8A2
:10DDE0003CE0914201D07245ABD1624A5B460121D1
:10DDF0000420F9F7DDF9143444450BF1010B7FF4ED
:10DE00006BAF03B0BDE8F08F5B4A217992F83DE03B
:10DE100092F83C208E45E8D091427FF471AFE4E760
:10DE2000227997F83D1097F83CE09142DDD0724599
:10DE30007FF471AFD9E722799AF83D109AF83CE067
:10DE40009142D2D072457FF471AFCEE7E2685007BD
:10DE500004D522F0040242F00802E26091067FF548
:10DE600042AF22F0200242F04002E2603BE7E2686B
:10DE7000130704D522F0080242F00402E2605006C3
:10DE80007FF531AF22F0400242F02002E2602AE743
:10DE900002EB42025CF82220002A3FF45DAF374AD1
:10DEA000217992F83D0092F83C2088429DD0914221
:10DEB0009BD02E4A106841063FF553AFC20363D48E
:10DEC0002279A2F1340101298FD902F0EF02202A30
:10DED0008BD072786AB1032A0BD0E26851060DD458
:10DEE000930688D52A68911C01322A6045F82140A2
:10DEF00081E7019BE26843B1130706D56A6805EB29
:10DF0000820101326A604C6375E75007EAD472E718
:10DF100002EB820209EB820249464FF0000C0B79BA
:10DF2000122B01F114010BD00CF1010CBCF10F0FFD
:10DF3000F5D1002AC2D0116822689142BED154E7BF
:10DF4000002A39D01268216891423FF44EAF142262
:10DF500002FB0CFC59F80C208A42AFD145E700BF08
:10DF6000089300204C0500200898002014000010A1
:10DF7000E4090020A4C4070800030020300C00209E
:10DF80008010002098070020494600220B79212BA1
:10DF900001F1140107D001320F2A91D00B79212B06
:10DFA00001F11401F7D1142101FB02F2216859F8A3
:10DFB0000220914284D118E72168C8E7F0B583B008
:10DFC000054619F075FC0C2806462BDCFDF7ACFA6B
:10DFD000214A224B927903EB42031B79002B32D06A
:10DFE0002B68B3422BDB002E27DD1D4F04350024A8
:10DFF00002E00134A64220D03A6855F8040FE1B29D
:10E00000C2F30072FEF7B2FD0028F2D1154D164A98
:10E0100005260146234604202E7003B0BDE8F040DB
:10E02000F9F7C6B80F49114A0C2301200093087074
:10E03000334600210420F9F7BBF803B0F0BD0949CD
:10E040000B4A0320F2E70B4A0221042003B0BDE88B
:10E05000F040F9F7ADB800BF68900020903907088C
:10E06000140000107690002044C50708BCC40708BF
:10E0700008C50708E8C40708014B00221A75704755
:10E0800048140020014B01221A75704748140020E3
:10E09000034A044B92F86C2003EB42035879704713
:10E0A00010C80020903907080F49104B91F86C20D8
:10E0B00003EB42035B7903B9704710B50C4B1C7836
:10E0C0008CB10C31002301EBC00E4FF0010C51F864
:10E0D00033202AB112791AB1984208BF8EF806C0CF
:10E0E00001339C42F3D110BD10C8002090390708BD
:10E0F0002810001010B5154CD4F82C2AD4F8303A5A
:10E10000D4F8241A82B002FB03F38B428DF8070087
:10E110001AD0D4F8203AD4F8280A0DF1070118448F
:10E1200063F014FDD4F8203AD4F82C2AD4F8241A39
:10E130001344D4F8302AB3FBF1F0013201FB103361
:10E14000C4F8203AC4F8302A02B010BD10C800202C
:10E150000B4B10B4002203F6342408200121C3F82D
:10E16000284AC3F8240A5DF8044BC3F82C1AC3F8F4
:10E170001C2AC3F8202AC3F8302AC3F8402A704763
:10E1800010C800200F4B93F86C30062B17D8DFE82F
:10E1900003F00416070A0D1013004FF4C8707047FF
:10E1A0004FF4FA607047084B988870474FF47A60D4
:10E1B00070474FF4FA5070474FF47A5070474FF45D
:10E1C0007A70704710C8002068900020044B03EB61
:10E1D000C000C06810B103685B681879704700BF61
:10E1E00010C8002008B50C4B1B7A012B06D0022B5F
:10E1F0000BD00A4B0A4AC3F8442A08BD5BF0F2F977
:10E20000064B084AC3F8442A08BD5BF0EBF9034B00
:10E21000054AC3F8442A08BD7890002010C80020A1
:10E22000A1B5000855C00208B9B500082DE9F04FA6
:10E2300085B09A469DF83830009381468B469046CB
:10E24000F3F7ACFF0446002800F08980584E96F89A
:10E250001D760A2F7ED85C2303FB07630022C3F8D8
:10E26000202683F8242699F8042013097D1C013BFD
:10E27000EDB2032B86F81D5602F00F0139D84D4A36
:10E28000019332F8130040FA01F2D30731D501228D
:10E290008A40013A10405DF0EFFE474A019BD35C93
:10E2A000464A184400EB400002EB800340F205218F
:10E2B000D98000991D728500002944D1A958404891
:10E2C000009301F13F4101F57E01890A405C59F05C
:10E2D0002DFE009B394A998802914FF00111505947
:10E2E000039102A9F4F7C0FB344A009BAA589B880B
:10E2F00053835C2505FB0765324AC5F82046B2FB0F
:10E30000F8F1204689B2F3F7E5FF5146D5F820062B
:10E31000F4F75CF8D5F8203659680B68B3F8442058
:10E320006FEA42426FEA524292B2A3F844201A883E
:10E3300092B242F001021A804A79032A30D8DFE80B
:10E3400002F0292B2D1299F8082018460221FCF71B
:10E35000ABFBCEE71C4A00210420F8F729FF002080
:10E3600005B0BDE8F08F40335C2000FB0760002162
:10E37000C0F82836154A196007EB470306EB8B06F1
:10E38000C7EBC30702EB87070120C6F8887005B00A
:10E39000BDE8F08F3433E7E73833E5E73C33E3E7B4
:10E3A0005C22002302FB0766C6F828361B60FFDEEE
:10E3B00010C800202033070828330708C82A002087
:10E3C000C021070840420F0068C4070830CE002073
:10E3D000034BD3F8442A12B10F2800D810477047D6
:10E3E00010C80020084AD2F8483A5BB140B1996899
:10E3F000B2F84C2A054BB3FBF2F35B100B6070478D
:10E400009B681860704700BF10C8002040420F0092
:10E4100010B50379012B84B00C4621D0022B1DD1FD
:10E420008368DB070DF10F024CBF01218121FAF750
:10E43000C5FF9DF80F30114A1070C3F3C002C3F33B
:10E44000001CC3F38001A270C3F38012DB0984F8BF
:10E4500000C06170E270237104B010BD0020E8E7D5
:10E4600082680DF10F0102F00102CDE900121A4697
:10E47000417C90F91000F5F7B3F9DAE74814002071
:10E480002DE9F04383B014460F4601AA50210546FA
:10E49000FAF7E8FF9DF804303C4EDFF8F490307056
:10E4A00001335B00DBB201AA238046212846FAF73C
:10E4B000D9FF2378DFF8DC80307009FB03F303F524
:10E4C000FA73A8FB03239DF8042099090132DB09A4
:10E4D00002FB0133A280A8FB03239B0901AAE3608E
:10E4E000512102232846FAF78FFC2378BDF8041047
:10E4F000307009FB03F349BA03F5FA73A8FB032351
:10E50000CAB2C1F307218A40013292B29909DB09EC
:10E5100002FB0133E280A8FB03239B09238201AAAB
:10E5200070212846FAF79EFF9DF8043030700133C1
:10E530005B00DBB201AA6380712102232846FAF74F
:10E5400063FCBDF80420F978307052BAD3B2C2F33C
:10E550000722934001339AB2228119B1E388D31A7A
:10E560009AB22281A1780A4B0A4803FB01F101F516
:10E57000FA71A0FB01139909DB0902FB0133A0FB2F
:10E5800003239B09638203B0BDE8F0834814002095
:10E59000002F3A00D34D62102DE9F043A84FA94C4B
:10E5A000DFF8A4828FB006464FF000094FF4FA73EB
:10E5B00009AA89210068C7F8E83087F8E190FAF7DE
:10E5C00051FF9DF82420207042F00102892130681B
:10E5D000F9F758FE4A46207088213068F9F752FE54
:10E5E0000122207080213068F9F74CFE0122207052
:10E5F000FF213068F9F746FE4A46207049463068E8
:10E60000F9F740FE09AA207091213068FAF72AFF35
:10E610009DF82430207001224946306887F8E330A5
:10E62000F9F730FE4A462070FF213068F9F72AFEDC
:10E630004A46207080213068F9F724FE09AA20702C
:10E6400060213068FAF70EFF9DF82420207042F018
:10E65000120260213068F9F715FE20250223207090
:10E6600009AA442130688DF825508DF82490FAF7D6
:10E6700053FBFF22207001213068F9F703FE356853
:10E680002070012280212846F9F7FCFD012220702C
:10E69000FF212846F9F7F6FD4A46207049462846EC
:10E6A000F9F7F0FD06222070FF212846F9F7EAFD70
:10E6B00009AA207083212846FAF7D4FE9DF8242069
:10E6C000207042F0040283212846F9F7DBFD07227F
:10E6D0002070FF212846F9F7D5FD01222070812105
:10E6E0002846F9F7CFFD0122207080212846F9F74E
:10E6F000C9FD6B22207094212846F9F7C3FD4A46D4
:10E70000207083212846F9F7BDFDD8F8003020702D
:10E71000C7F8E43014E0AB68DB0709AA4FF08301C7
:10E7200028465EBF09AA83212846FAF747FE9DF8CE
:10E730002430207083B9D7F8E830002B40F00F83E5
:10E740002B79012B00F0FE82022BE4D09DF82430BF
:10E7500000202070002BEED0012283212846F9F7FB
:10E7600091FD09AA207092212846FAF77BFE00222B
:10E770002070812128469DF82490F9F783FD062218
:10E780002070FF212846F9F77DFD09AA207083211A
:10E790002846FAF767FE9DF82420207002F0FB025D
:10E7A00083212846F9F76EFD01222070FF212846BB
:10E7B000F9F768FD0122207000212846F9F762FD73
:10E7C00000222070FF212846F9F75CFD002220700E
:10E7D00080212846F9F756FD0623207007AAB021AC
:10E7E0003068FAF711FB01222070FF213068F9F739
:10E7F00049FD002220704F213068F9F743FD2C229B
:10E8000020704E213068F9F73DFD00222070FF2175
:10E810003068F9F737FDB4222070B6213068F9F777
:10E8200031FD4FEAD918B8F1000F4FF00005207004
:10E8300018BF4FF00C0809F07F0EAC46012017E01E
:10E8400010C800204814002054350020F44503F07F
:10E85000070317D011F81C2C42FA03F3DB070CF165
:10E86000010105F1010548BF5FFA81FC302D12D08E
:10E87000EBB20EAA02EBD301984503F0070200FAAF
:10E8800002F2E3D911F81C3C013523EA0202302DD3
:10E8900001F81C2CECD1062307AAB0213068FAF746
:10E8A0003BFA01222070FF213068F9F7EBFC0022CF
:10E8B000114620703068F9F7E5FC00222070FF2136
:10E8C0003068F9F7DFFC0022207009213068F9F781
:10E8D000D9FC0022207010213068F9F7D3FC002207
:10E8E000207011213068F9F7CDFC0122207024211D
:10E8F0003068F9F7C7FCFF22207025213068F9F74E
:10E90000C1FC0022207075213068F9F7BBFC0122A0
:10E910002070FF213068F9F7B5FC2C2220704E21C1
:10E920003068F9F7AFFC0022207048213068F9F711
:10E93000A9FC2946207020223068F9F7A3FC0022A8
:10E940002070FF213068F9F79DFC294620700922CC
:10E950003068F9F797FC0022207054213068F9F7ED
:10E9600091FC0422207031213068F9F78BFC0322DE
:10E97000207032213068F9F785FC83222070402115
:10E980003068F9F77FFC2522207046213068F9F7BE
:10E9900079FC0022207060213068F9F773FC0022B6
:10E9A000207027213068F9F76DFC06222070502175
:10E9B0003068F9F767FC0022207051213068F9F7C0
:10E9C00061FC9622207052213068F9F75BFC082226
:10E9D000207056213068F9F755FC2A4620705721DF
:10E9E0003068F9F74FFC0022207061213068F9F798
:10E9F00049FC0022207062213068F9F743FC0022B4
:10EA0000207064213068F9F73DFC002220706521F8
:10EA10003068F9F737FCA022207066213068F9F7DA
:10EA200031FC01222070FF213068F9F72BFC3222E3
:10EA3000207022213068F9F725FC1422207047212C
:10EA40003068F9F71FFCFF22207049213068F9F780
:10EA500019FC002220704A213068F9F713FC0022CB
:10EA60002070FF213068F9F70DFC0A2220707A210E
:10EA70003068F9F707FC002220707B213068F9F735
:10EA800001FC2122207078213068F9F7FBFB01227C
:10EA90002070FF213068F9F7F5FB34222070232124
:10EAA0003068F9F7EFFB0022207042213068F9F757
:10EAB000E9FBFF22207044213068F9F7E3FB2622AE
:10EAC000207045213068F9F7DDFB052220704621D2
:10EAD0003068F9F7D7FB4022114620703068F9F70B
:10EAE000D1FB062220700E213068F9F7CBFB1A22E9
:10EAF000207020213068F9F7C5FB402220704321A7
:10EB00003068F9F7BFFB00222070FF213068F9F769
:10EB1000B9FB0322207034213068F9F7B3FB44229B
:10EB2000207035213068F9F7ADFB01222070FF21FC
:10EB30003068F9F7A7FB0422207031213068F9F71B
:10EB4000A1FB092220704B213068F9F79BFB0522BD
:10EB500020704C213068F9F795FB042220704D217C
:10EB60003068F9F78FFB00222070FF213068F9F739
:10EB700089FB0022207044213068F9F783FB2022B2
:10EB8000207045213068F9F77DFB0822207047216D
:10EB90003068F9F777FB2822207048213068F9F7B0
:10EBA00071FB0022207067213068F9F76BFB0422AB
:10EBB000207070213068F9F765FB01222070712107
:10EBC0003068F9F75FFBFE22207072213068F9F798
:10EBD00059FB0022207076213068F9F753FB0022A0
:10EBE000207077213068F9F74DFB01222070FF215A
:10EBF0003068F9F747FB012220700D213068F9F7E2
:10EC000041FB00222070FF213068F9F73BFB012215
:10EC1000207080213068F9F735FBF822207001213F
:10EC20003068F9F72FFB01222070FF213068F9F7D7
:10EC300029FB012220708E213068F9F723FB012285
:10EC4000207000213068F9F71DFB00222070FF21A1
:10EC50003068F9F717FB0022207080213068F9F73F
:10EC600011FB042220700A213068F9F70BFB35688C
:10EC7000207009AA84212846FAF7F4FB9DF8242085
:10EC8000207002F0EF0284212846F9F7FBFA0122F6
:10EC900020700B213068F9F7F5FA05A9207030686B
:10ECA0000390FFF7B5FB039809AA05A9FFF7E8FB56
:10ECB0009DF81430002B65D00C9B03F684539DF80F
:10ECC0001620002A55D00C9A02F2B22203EB42031E
:10ECD0009DF8172022B1BDF8342002F525721344A7
:10ECE0009DF8182022B1BDF8362002F226221344E6
:10ECF00001213068C7F8503AE822F9F7C3FAD7F88B
:10ED0000501A207044F61F639942306802D95BF0B4
:10ED1000FBF9306801221146F9F7B4FA402120705E
:10ED20003068FDF7ADF950B1012130680222F9F7E2
:10ED3000A9FA002120703068FDF7A2F928BB0FB0B6
:10ED4000BDE8F083AA68697C95F9100002F0010221
:10ED5000019209AA00928322F4F742FDE7E4D8F871
:10ED60000020D7F8E41092B2521A9342BFF4E8ACF4
:10ED7000E5E79DF81520002AAAD00C9A02F5257225
:10ED80001344A5E740F6363399E7E82201213068BD
:10ED9000F9F778FA002502234FF0200C09AA207019
:10EDA000442130688DF825C08DF82450F9F7B4FF60
:10EDB000D6F80080207005A94046FFF729FB09AA74
:10EDC00005A94046FFF75CFB502257214046F9F762
:10EDD00059FA0822207056214046F9F753FA0822C2
:10EDE000207050214046F9F74DFABDF834202070CC
:10EDF0004FF47A7148F20E6301FB02337C4A93426E
:10EE000040F2F2807B4AA2FB03231B0C5A1E32F015
:10EE1000FF0309D02B465208013322F0FF019BB2B9
:10EE20000029F8D11B029BB21343C3F30722DBB2C4
:10EE30008DF810208DF8113004AA0223512140468C
:10EE4000F9F76AFF0C9A20704FF47A7148F20E635A
:10EE500001FB0233684A934200F2C480654AA2FB78
:10EE60000332120C013AD2B246214046F9F70AFAAF
:10EE7000D7F8501A207044F61F63994202D94046D1
:10EE80005BF042F904AA01214046FAF7EBFA0222AC
:10EE90002070012140469DF81050F9F7F3F9002148
:10EEA00020704046FDF7ECF82A4601214046F9F76C
:10EEB000E9F93568207005A92846FFF7A9FA09AADB
:10EEC00005A92846FFF7DCFA482211462846F9F73B
:10EED000D9F90822207047212846F9F7D3F90322EF
:10EEE000207032212846F9F7CDF907222070302111
:10EEF0002846F9F7C7F901222070FF212846F9F7C3
:10EF0000C1F92022207030212846F9F7BBF90022F0
:10EF10002070FF212846F9F7B5F9062220707021EC
:10EF20002846F9F7AFF9BDF83610344A207046F696
:10EF300044034FF47A7000FB0133A2FB03239DF8D6
:10EF400017201B0B1AB1BDF82A2013449BB2002BCB
:10EF500046D05A1E32F0FF0309D000235208013375
:10EF600022F0FF019BB20029F8D11B029BB2134390
:10EF7000C3F30722DBB28DF810208DF81130712118
:10EF8000022304AA2846F9F7C7FED7F8501A2070C2
:10EF900044F61F63994202D928465BF0B5F804AAEB
:10EFA00001212846FAF75EFA022220700121284644
:10EFB0009DF81060F9F766F9002120702846FDF7EA
:10EFC0005FF8324601212846F9F75CF964220123F3
:10EFD0002070C7F8E82087F8E1300FB0BDE8F08373
:10EFE0001A46C8E7FF223FE72B462A4620E700BF24
:10EFF0001B0C0100950370F41B280D014963A41339
:10F0000010B5174C84F8F110017952BAA4F8F22027
:10F0100001294FF0000282B084F8F02012D00229BA
:10F020000CD1042304F1F002FF21F9F71FFE0028A0
:10F0300014BF00206FF00C0002B010BD6FF00C0088
:10F0400002B010BD8268417C90F91000F03402F0EB
:10F050000102CDE900420423FF22F4F7F5FBE6E7C5
:10F0600010C800202DE9F04FA24FA34D06680021E3
:10F070003C4685B0834685F8F0115A37C4F12D0916
:10F0800005F1F00A884615E0022A0FD1B26812F0A5
:10F09000010F4FF0030352464FF0FF01304601BF0E
:10F0A00003235246FF213046F9F7E0FDBC421AD057
:10F0B00014F8011F327985F8F21009EB0403012AD4
:10F0C00085F8F08085F8F130DED1B368717C96F96F
:10F0D000100003F00103CDE900A3FF220323F4F79E
:10F0E000B3FBBC42E4D14FF40743A5F8F030402312
:10F0F00085F8F23052460323FF213046F9F70CFE23
:10F1000000238DF80E300DF10E0130465AF0C2FF8B
:10F110009DF80E30002BF6D04FF40640A5F8F00015
:10F120000120764A85F8F2000323FF213046F9F7E3
:10F13000F3FD4FF40740714AA5F8F00000240323C3
:10F14000FF21304685F8F240F9F7E6FD4FF4006004
:10F15000A5F8F0000920694A85F8F2000323FF2191
:10F160003046F9F7D9FD4FF43063A5F8F030634A23
:10F1700085F8F24030460323FF21F9F7CDFD002842
:10F180007FD0DBF800600DF10E025E213046FCF707
:10F190001FFDBDF80E30B3F5D77F00F0A38079D8FE
:10F1A000512B75D040F29480AD2B00F09B80D62B74
:10F1B00040F08A80212408BB0A224B213046FDF70B
:10F1C00051FD0F2260213046FDF74CFD0D226321D9
:10F1D0003046FDF747FDB82269213046FDF742FD74
:10F1E00040F60D7278213046FFF70AFF40F60E62B6
:10F1F0007A213046FFF704FF002875D0DBF80000C5
:10F2000021215AF097FEDBF800400DF10E02DE21BD
:10F210002046FCF7DDFCBDF80E309FED397AC3F3D4
:10F220000903ADF80E3003EB8303DB0007EE903AE1
:10F23000F8EEE77A204667EE877A0623FCEEE77A57
:10F240004FF4D84417EE902A110E85F8F210110CE5
:10F2500052BA85F8F310A5F8F420FF215246A5F81C
:10F26000F040F9F759FD4FF407414023DBF8000067
:10F27000A5F8F01085F8F23052460323FF21F9F784
:10F280004BFD85F8F00105B0BDE8F08F1E2BB5D120
:10F29000142490E740F2E132934221D00AD940F29F
:10F2A0008F42934203D040F291529342A6D14FF441
:10F2B000FA7480E740F2D922934211D040F2E12261
:10F2C000934209D1642476E7602B3FF473AF95E74E
:10F2D0001D2BDBD10F246EE7B3F5E67FF2D08DE76F
:10F2E000C82468E7322466E7214630465AF022FEF9
:10F2F00084E700BFA439070810C8002000C9002017
:10F300009A99893F03682DE9F041DF691FB13B46B7
:10F31000BDE8F0411847002A164611DD04460D46A7
:10F320000E4400E023689B68204698470028F9D0E7
:10F33000236815F8011B1B6820469847AE42F1D19F
:10F34000BDE8F081DEE700BF0B4B9A7A03468AB92D
:10F350000A490B4A0978126849B13AB11BB11368DE
:10F3600092881A837047136892885A83704780F096
:10F370000103F2E7FFF736B85491002050910020C6
:10F380004C910020BFF34F8F0549064BCA6802F429
:10F39000E0621343CB60BFF34F8F00BFFDE700BFB8
:10F3A00000ED00E00400FA0508B572B600224FF047
:10F3B000FF31930003F1604303F561430132082AF2
:10F3C000C3F88010C3F88011F3D1FFF7DBFF00BF53
:10F3D000012108B50846F4F79BFBFFF7E5FF00BFE6
:10F3E00000B583B00D49002200920091009B0433C8
:10F3F0000093009B1B68012B02D003B05DF804FB57
:10F4000001920191019B064904330193019B1A600B
:10F410000B6883F308884B689847FEE75028004044
:10F420000000FF1F10B4EFF31183102282F3128843
:10F43000094C0A4822684FF0E021013222608A69B3
:10F44000C0F8542A0022C0F8582A0A69DBB283F3B4
:10F4500011885DF8044B70475435002010C8002017
:10F4600030B4EFF31182102383F312884FF0E023BE
:10F47000D2B29969186910F4803F0D481EBF01216E
:10F48000C0F8581A99690B4B1D68D0F8583A82F3A6
:10F490001188094804684FF47A7202FB04F02B4487
:10F4A000401A0021B0FBF4F030BCE3FB02017047CE
:10F4B00010C80020543500207C360020124B5B68B9
:10F4C000C3F30803FBB9EFF31183E3B930B40F4A78
:10F4D0000F4C4FF0E02C1168DCF8180013688B42D9
:10F4E000F9D1D4F8541A8142F5D30A4A15684FF479
:10F4F0007A7404FB05F20021101AB0FBF5F0E3FB6F
:10F50000040130BC7047ABE700ED00E0543500204B
:10F5100010C800207C36002090B170B5461EFFF761
:10F52000CDFF04460D46FFF7C9FF031B61EB050243
:10F53000B3F57A7F72F10003F5D3013EEFD270BDCF
:10F54000704700BF70B5006801220921F8F79AFEE4
:10F550006426FFF7B3FF04460D46FFF7AFFF031B1A
:10F5600061EB0502B3F57A7F72F10003F5D3013E3A
:10F57000EFD170BD2DE9804885B0431C0393DFF8BF
:10F580009C81DFF89CB10A230293D8F89C10D8F82C
:10F59000A830B8F8A000B8F8AC20039C48830194C8
:10F5A0001A834FF0320A4FF005094C69204214BF0C
:10F5B0004883088359690A4214BF5A831A839BF807
:10F5C0000A30002B6DD1534B1A78534B1B68002A1D
:10F5D00061D013B11A689B88138356465746FFF7CC
:10F5E0006DFF04460D46FFF769FF001B61EB050147
:10F5F000B0F57A7F71F10003F5D3013FEFD1D8F870
:10F600009C30B8F8A02059690A4214BF5A831A8363
:10F61000D8F8A830B8F8AC2059690A4214BF5A8308
:10F620001A839BF80A30002B3FD13A4B1A783A4B99
:10F630001B6852BB13B11A689B881383FFF73EFF08
:10F6400004460D46FFF73AFF001B61EB0501B0F5DC
:10F650007A7F71F10003F5D3013EEFD1B9F1000FCC
:10F660000BD0B9F1010924D0B8F8A000D8F89C104B
:10F67000B8F8AC20D8F8A83097E7019B013B01937C
:10F68000019B6BB34FF00009EEE7002BD6D01A6850
:10F690009B885383D2E7002B9FD01A689B885383A3
:10F6A0009BE70120FEF79EFE97E70020FEF79AFEFB
:10F6B000C4E74FF4FA76FFF701FF04460D46FFF763
:10F6C000FDFE031B61EB0501B3F57A7F71F10003C9
:10F6D000F5D3013EEFD1019B4FF0FA0A002BD1D1B7
:10F6E0004FF47A76FFF7EAFE04460D46FFF7E6FE92
:10F6F000031B61EB0501B3F57A7F71F10003F5D3CC
:10F70000013EEFD1029B013B02937FF43EAFFFF736
:10F710005FFE00BF509100204C910020C82A0020BD
:10F72000549100200178F9B1F8B5104F0546002634
:10F7300002E015F8011FB1B1D7F85C4A637A5A1C90
:10F740002344D2B262729972237A9342F1D8002A8A
:10F75000EFD004F10A01D4E900309847667215F839
:10F76000011F0029E8D1F8BD704700BF10C8002074
:10F7700030B583B00F4C01900F480091FFF7D2FFD6
:10F78000DDE900320D49D4F85C0A58F0C3FCD4F826
:10F790005C5A6A7A32B12B68686805F10A019847A9
:10F7A00000236B7294F8603A13B1012384F8613A34
:10F7B00003B030BD10C800206CC50708B1BC0008FC
:10F7C0002DE9F041404F3B68002B7AD01B6A9847E7
:10F7D0008368002B59D03D48DFF80081FFF7A2FF76
:10F7E0003B48FFF79FFFB8F8626A1EBBD8F8640A6F
:10F7F000FAF72EFF002388F8683A88F8693AC8F8C3
:10F800006C3A3B6813B15B68984710BB6426FFF7FE
:10F8100055FE04460D46FFF751FE031B61EB050143
:10F82000B3F57A7F71F10003F5D3013EEFD1E8E73C
:10F83000013EDBD0FFF742FE04460D46FFF73EFED9
:10F84000031B61EB0501B3F57A7F71F10003F5D37A
:10F85000EEE72048FFF766FF1D48FFF763FFB8F8A3
:10F86000626A1EB9BDE8F081013EFBD0FFF726FEBB
:10F8700004460D46FFF722FE031B61EB0502B3F5BC
:10F880007A7F72F10003F5D3EEE71348FFF74AFFE2
:10F890000F48FFF747FF114BB3F8626A002EE1D023
:10F8A000FFF70CFE04460D46FFF708FE031B61EB55
:10F8B0000502B3F57A7F72F10003F5D3013EEFD173
:10F8C000D0E7074884E700BF907100208CC5070887
:10F8D000B8C8070898C5070878C5070810C80020E9
:10F8E0004C80002080B51948194DFFF71BFF1948BF
:10F8F000FFF718FFD5F85C4A627A32B1214660689A
:10F9000051F80A3B984700236372D5F8FC713B68B5
:10F9100038465B699847B0B90A26FFF7CFFD044621
:10F920000D46FFF7CBFD031B61EB0502B3F57A7FB4
:10F9300072F10003F5D3013EEFD13B6838465B69B5
:10F9400098470028E8D001200FF0CEFCA0C507089A
:10F9500010C80020BCC50708194B1A78012A00D02E
:10F9600070475B790D2B01D01648DBE600B5164ACF
:10F9700087B00023CDE9013392F815C08DF814301B
:10F98000CDE903334122EB2315214FF0A60E684643
:10F990008DF801208DF80330B22203238DF800E0AA
:10F9A0008DF802108DF804C08DF805208DF8063012
:10F9B0002AF0C4FF054807B05DF804EBB2E600BFCB
:10F9C0005C940020C8C5070848140020D8C5070863
:10F9D000F8B52F482F4FFFF7A5FE2F48FFF7A2FEDF
:10F9E000B7F8626A002E43D1D7F85C4A627A32B126
:10F9F0002146606851F80A3B98470023637200254E
:10FA000087F8705AC7F8B05A87F8B45A17F08CFFC5
:10FA10002248FFF787FED7F85C4A627A2AB121466E
:10FA2000606851F80A3B98476572D7F8FC713B68EB
:10FA300038465B699847B0B90A26FFF73FFD044690
:10FA40000D46FFF73BFD031B61EB0502B3F57A7F23
:10FA500072F10003F5D3013EEFD13B6838465B6994
:10FA600098470028E8D000200FF03EFC013EBBD0B4
:10FA7000FFF724FD04460D46FFF720FD031B61EB55
:10FA80000502B3F57A7F72F10003F5D3EEE700BF0C
:10FA9000F4C5070810C80020B8C80708BCC5070887
:10FAA00070B50C48FFF73EFE0B4BB3F8626A16B90F
:10FAB00070BD013EFCD0FFF701FD04460D46FFF787
:10FAC000FDFC031B61EB0502B3F57A7F72F10003C5
:10FAD000F5D3EEE7B8C8070810C8002070B5044693
:10FAE0000F48FFF71FFE2046FFF71CFE0D48FFF7EB
:10FAF00019FE0D4BB3F8626A16B970BD013EFCD019
:10FB0000FFF7DCFC04460D46FFF7D8FC031B61EB56
:10FB10000502B3F57A7F72F10003F5D3EEE700BF7B
:10FB200020C60708B8C8070810C80020800601D5FD
:10FB3000002933D10CB470B5194C1A49D4F85C0AB9
:10FB400082B007AB069A019358F0E4FAD4F85C5AF5
:10FB50006A7A32B12B68686805F10A019847002378
:10FB60006B721148FFF7DEFDB4F8626A3EB90120FE
:10FB700002B0BDE8704002B07047013EF7D0FFF719
:10FB80009DFC04460D46FFF799FC031B61EB050243
:10FB9000B3F57A7F72F10003F5D3EEE700207047EA
:10FBA00010C80020B1BC0008B8C8070810F0400019
:10FBB00031D00CB470B50C4682B029B1002002B02F
:10FBC000BDE8704002B07047194ED6F85C5A6B7AA7
:10FBD0005A1C2B44D2B223216A7299722B7A934217
:10FBE0001AD9069A134907AB2846019358F092FA9E
:10FBF000D6F85C4A627A32B1D4E9003004F10A01E5
:10FC0000984700236372FFF74BFF012002B0BDE865
:10FC1000704002B070477047002AE2D0D5E900304A
:10FC200005F10A0198476C72D6F85C5AD9E700BF13
:10FC300010C80020B1BC00080FB410B582B004ABEE
:10FC40000C4C53F8042BD4F85C0A0B49019358F080
:10FC500061FAD4F85C4A627A32B1D4E9003004F136
:10FC60000A0198470023637202B0BDE8104004B057
:10FC7000704700BF10C80020B1BC00080FB470B5B9
:10FC800082B006AB174C53F8042B1749D4F85C0A22
:10FC9000019358F03FFAD4F85C5A6A7A32B12B6873
:10FCA000686805F10A01984700236B720F48FFF757
:10FCB00039FDB4F8626A36B902B0BDE8704004B0EC
:10FCC0007047013EF8D0FFF7F9FB04460D46FFF7F9
:10FCD000F5FB031B61EB0502B3F57A7F72F10003BC
:10FCE000F5D3EEE710C80020B1BC0008B8C807087B
:10FCF0002DE9F04F474B1B6883B0002B00F0848048
:10FD00001B6A98478246DAF80800002875D0BAF8CE
:10FD10000C30DAF80420BAF800100190BAF80200AA
:10FD200000903D48DFF8FC80DFF810B1FFF7A6FF38
:10FD300000264746002E42D0DBF800309E4212DA01
:10FD40003B78062B39D8354A02EB83031A6FBB8800
:10FD500000937B88324831460136FFF78FFF092E2A
:10FD600007F10607E6D1002304E00133092B08F16F
:10FD700006084CD098F80020022AF6D1294A2A48D1
:10FD8000DAF8041003EB430302EB430390F8692A0B
:10FD90009C885B88E41A90F8683A9A428ABFC2F15C
:10FDA00080029B1A9B18D0F86C2A204804FB011192
:10FDB0001A4403B0BDE8F04F60E70022C7E71C48D3
:10FDC000FFF7B0FC1B48FFF7ADFC174BB3F8623AE6
:10FDD000002BB1D09946FFF771FB04460D46FFF7A3
:10FDE0006DFB001B61EB0501B0F57A7F71F100033B
:10FDF000F5D3B9F10109EED19EE70F48FFF792FC68
:10FE000003B0BDE8F04F4BE6DFF834A07BE70023FA
:10FE10009B88FFDE9071002028C6070890390708EC
:10FE200084C607085871002010C8002094C607082F
:10FE300078C60708B8C8070878C507089471002075
:10FE40004C8000202DE9F84F06465BF0BBFADFF846
:10FE50007CA10446DAF80080002839D14D484E4E86
:10FE60004E4DDFF86091FFF75DFC012754234C49AC
:10FE700007FA04F24BB9013485B12B78294607FA09
:10FE800004F256F8045F002BF5D012EA080FF2D006
:10FE90004846FFF7D1FE0134002DEED14148FFF76F
:10FEA00041FC414BB3F8626A1EB9BDE8F88F013ED0
:10FEB000FBD0FFF703FB04460D46FFF7FFFA031BD9
:10FEC00061EB0502B3F57A7F72F10003F5D3EEE73B
:10FED000024636493046F7F715FB00283DD0337807
:10FEE000DFF8EC902E4D2D2B03BF013604F1FF34CB
:10FEF0004FF0010B4FF0000B002703E059F8045FAF
:10FF00000137C5B1294622463046F7F7FBFA0028EB
:10FF1000F4D1012303FA07F7BBF1000F32D028EA2E
:10FF200007072348CAF80070FFF7FCFB2946214861
:10FF3000BDE8F84FA2E62048FFF7F4FB1F48FFF7A3
:10FF4000F1FBFFF7ADFD184B93F8602A002AACD007
:10FF5000012283F8612ABDE8F88F19480E4D0F4C35
:10FF6000184EFFF7DFFB0E49542330460BB1FFF765
:10FF700063FE24B12378214655F8044FF5E7BDE828
:10FF8000F84F8DE547EA08070F48CAF80070FFF7F9
:10FF9000C9FBCBE7CCC60708203A0708B4C6070858
:10FFA000BCC60708B8C8070810C80020DCC6070888
:10FFB00000C7070808F307086CC50708F0C607085C
:10FFC000E4C60708D8C607080CC70708DC7000207D
:10FFD0001C3A07082DE9F84F06465BF0F3F9DFF805
:10FFE00084910446D9F80870002840D14F48504EFB
:10FFF000DFF86891DFF870810125FFF793FB224657
:020000040801F1
:100000002C4604FA02F23A424A490CD16B1C2A46A9
:10001000DDB208EB850386B104FA02F23A423146BA
:10002000D3F81061F2D04846FFF706FE6B1C2A4653
:10003000DDB208EB8503002EEED13F48FFF772FBDF
:100040003E4BB3F8626A1EB9BDE8F88F013EFBD0A3
:10005000FFF734FA04460D46FFF730FA031B61EB55
:100060000502B3F57A7F72F10003F5D3EEE702469D
:1000700033493046F7F746FA00283FD03378DFF8A7
:10008000D8A02C4D2D2B03BF013604F1FF344FF0C7
:10009000010B4FF0000B4FF0000804E05AF8045F2A
:1000A00008F10108C5B1294622463046F7F72AFA79
:1000B0000028F3D1012303FA08F8BBF1000F2DD07B
:1000C00027EA08071F48C9F80870FFF72BFB2946E5
:1000D0001D48BDE8F84FD1E51C48FFF723FB1C483D
:1000E000FFF720FBFFF7DCFC144B93F8602A002A93
:1000F000AAD0012283F8612ABDE8F88F1548164C72
:10010000164DFFF70FFB0B492846FFF795FD54F8F6
:10011000041F0029F8D1BDE8F84FC1E447EA0807F9
:100120000F48C9F80870FFF7FDFAD0E7CCC60708FA
:1001300014C707081CC70708B8C8070810C800205C
:10014000DCC6070800C7070808F307086CC50708DE
:10015000F0C60708E4C60708A03A0708D8C607088B
:100160000CC7070860910020903907082DE9F84F67
:1001700080465BF027F9DFF8A0A1DAF80060E0B96B
:100180005648574CDFF87881FFF756FD012304F5F8
:100190008A771D4601E014F80C3F013B05FA03F392
:1001A0003342404602D0A168FFF746FDBC42F2D17F
:1001B000002E37D0BDE8F84F72E4074602464949A1
:1001C0004046F7F79FF998B398F80030444DDFF8B0
:1001D00034912D2B03BF08F1010807F1FF374FF0D1
:1001E000010B4FF0000B002401E0D5F808904946C0
:1001F0003A464046F7F786F90C3568B301341A2CB5
:10020000F3D13948FFF78EFA3848FFF78BFAFFF73A
:1002100047FC374B93F8602A12B1012283F8612A18
:10022000BDE8F88F3348FFF77DFABDE8F84F37E4B3
:10023000314C3248324EFFF775FA04F59C7531495E
:1002400001E054F80C1C30460C34FFF7F5FCAC42CE
:10025000F7D1BDE8F84F23E4BBF1000F18D0182CFC
:1002600034D0192C2AD0284A04EB440402EB84022F
:10027000012392F83821013A93401E43CAF80060E6
:100280002248FFF74FFA49462148BDE8F84FF5E408
:10029000182C20D0192C16D01B4B04EB440403EB74
:1002A0008404012394F83821013A934026EA030696
:1002B000CAF800601748FFF735FAE4E7DAF80430C7
:1002C000CAF80030DCE7CAF80460F3E76FF07F4358
:1002D000CAF80030D4E7CAF800B0EBE738C707081F
:1002E000C83A0708DCC607086CC50708F0C6070847
:1002F00010C8002044C70708DC3A070854C707089D
:100300004CC7070824C707089039070800C7070823
:1003100008F307080CC70708549100202DE9F8439B
:1003200008B1037883BB364881694C1C192C3ED830
:10033000344E04EB440306EB83034FEA4408D3F83E
:100340004091B9F1000F32D02F4F84610020054653
:10035000FEF7FAFF87F8B50A29F048F82146444429
:1003600006EB8406294887F8B65A4A46C7F8B85AB1
:10037000A7F8BC5AC7F8C05AFFF780FC96F83801B6
:10038000BDE8F84323F052BDF7F774FC1928044682
:1003900030D81C4E04EB440306EB83034FEA4408B9
:1003A000D3F84091B9F1000F24D01548CCE7154D92
:1003B00006E004EB440305EB83030BD9914212D012
:1003C00022460134192CF4DD0024DFF84C900D4E48
:1003D000A046B9E7D3F840912E464FEA4408B9F158
:1003E000000FEBD0B0E70A48FFF79CF9BDE8F843EF
:1003F000FFF756BB21460748BDE8F8433EE400BF7F
:10040000481400209039070810C800208CC707083E
:1004100060C7070874C7070824C7070810B518B3D2
:1004200003780BB3F7F726FC0138022828D8C4B2AA
:10043000204605F0C5F9F0B9601CC0B2114B41F27D
:1004400002420128A3F8C42A4FEA400105D004293A
:10045000A3F8C62AC8BFA3F8C82A0B44FF220F205E
:1004600083F8C42A23F0E2FC074B08481978BDE85A
:100470001040013102E404F043FF06F069F8DBE7C5
:1004800010BD00BF10C80020F08D0020ACC70708C9
:10049000F8B500283CD00378002B39D0F7F7EAFBF9
:1004A000013802283ED8204D204E00EB800105EB9C
:1004B0000113C4B293F8FC3A77787470013B05F5E8
:1004C0002E62D8B202EB01120128C5F8DC2A26D927
:1004D000BC421FD1601CC0B241F202430128A5F802
:1004E000C43A4FEA400205D0042AA5F8C63AC8BF6C
:1004F000A5F8C83A1544FF230F2085F8C43A23F025
:1005000095FC71780A48BDE8F8400131FFF7B6BBA9
:10051000064EF6E704F0F4FE06F01AF8DAE705F006
:100520004FF9D5E7F8BD00BF10C80020F08D0020BE
:10053000A4C707082DE9F041384F3948B97ADFF8E8
:100540001481FFF79BFB3748FFF7ECF83648FFF7BD
:10055000E9F8B8F8626A002E3FD1B9793348FFF75D
:100560008DFBF9793248FFF789FB397A3148FFF77B
:1005700085FB797A3048FFF781FB3048FFF7D2F8E6
:100580002948FFF7CFF8B8F8626ABEBB2C4C2D485B
:10059000B4F91030B4F90E20B4F90C10FFF76EFB6B
:1005A000B4F91C30B4F91A20B4F918102648FFF732
:1005B00065FBB4F91420B4F912102448B4F91630CC
:1005C000FFF75CFBB4F92020B4F91E102048BDE809
:1005D000F041FFF753BB013EBFD0FEF76FFF04466B
:1005E0000D46FEF76BFF031B61EB0501B3F57A7F48
:1005F00071F10003F5D3EEE7013EC7D0FEF75EFFD1
:1006000004460D46FEF75AFF031B61EB0502B3F5E6
:100610007A7F72F10003F5D3EEE700BF000000100F
:10062000B8C70708D4C70708B8C80708E8C7070845
:10063000F0C70708FCC7070804C807080CC8070864
:1006400010A8002020C8070830C8070840C80708BD
:1006500050C8070810C800202DE9F04300F10047FA
:100660009F4D8DB0013F662205E09E421BD1B842EE
:1006700012D015F8012F10F8013BA3F14104192CF9
:10068000A2F1410198BF2033192902F12006ECD9CB
:100690009A4208D1002AEAD1924D2B78012B00F022
:1006A000B780022B03D00DB0BDE8F04342E7002332
:1006B000012206A93D208DF81830F7F7DDFB19243B
:1006C000FEF7FCFE06460F46FEF7F8FE831B61EBC5
:1006D0000702B3F57A7F72F10003F5D3013CEFD145
:1006E000814E824F30683C700368AA211B6898478E
:1006F0003068036801211B689847306803685521FA
:100700001B6898473068036816211B6898474FF0AC
:100710003209FEF7D3FE04468846FEF7CFFE031BE0
:1007200061EB0801B3F57A7F71F10003F5D3B9F1FC
:100730000109EED16E480DF11C0E0624A31FDBB299
:100740007146C21892F801C0C25C0233DBB242EAC1
:100750000C22A34221F8022BF3D10633DCB2182C71
:100760000EF1060EEAD1B0F91290B0F9148030689B
:1007700000243C700368AA211B689847306803680E
:1007800021461B689847306803683D211B689847DD
:100790003068036801211B689847306803680C21A2
:1007A0001B6819279847FEF789FE04460E46FEF798
:1007B00085FE031B61EB0601B3F57A7F71F100033F
:1007C000F5D3013FEFD1BDF91CE0BDF91EC0BDF965
:1007D0002070BDF92260BDF92440BDF92600BDF9A5
:1007E0002810BDF92A20BDF92C30A5F818E0A5F88D
:1007F0001AC0AF836E82AC82E882A981EA812B8223
:10080000A5F81E90A5F820800DB0BDE8F04391E654
:10081000DFF8E0800022D8F800003D21F7F732FD34
:100820001927FEF74BFE04460E46FEF747FE031B54
:1008300061EB0601B3F57A7F71F10003F5D3013F57
:10084000EFD1162306AA5521D8F80000F8F7DCFAF4
:10085000D8F800000C223D21F7F714FD1927FEF708
:100860002DFE04460E46FEF729FE031B61EB060231
:10087000B3F57A7F72F10003F5D3013FEFD101AFF9
:100880000624A31FDBB238460CAAD118023311F894
:10089000176C11F8182CDBB242EA0622A34220F8AA
:1008A000022BF1D10633DCB2182C07F10607E8D190
:1008B000BDF92A90BDF92C80BDF904E0BDF906C050
:1008C000BDF90870BDF90A60BDF90C40BDF90E0014
:1008D000BDF91010BDF91220BDF9143085E700BF35
:1008E00060C8070810A800208C7D0020D871002067
:1008F000E4710020388000200FB470B582B006A9E2
:1009000051F8040B0191FEF733FF0E48FEF70AFF82
:100910000D4BB3F8626A36B902B0BDE8704004B05E
:100920007047013EF8D0FEF7C9FD04460D46FEF7BC
:10093000C5FD031B61EB0502B3F57A7F72F100037D
:10094000F5D3EEE7B8C8070810C8002000283DD04E
:100950000378002B3AD02DE9F04F87B0584905AA0B
:1009600061F0D3FA0446002800F09F804FF0000B9E
:10097000DFF87C91DFF87C81DFF87CA15D465F4683
:100980004FF0FF360BE0BBF1000F26D04C4905AA13
:10099000002061F0BAFA0BF1010B044610B3BBF171
:1009A000010F15D0BBF1020FEDD14946204661F091
:1009B0008CFB00286BD045F001054146204661F0D4
:1009C00084FB00285CD045F00205DFE73D4893E753
:1009D0002046F7F74FF90746D8E72046F7F74AF9D8
:1009E0000646D3E770B2384900230C4694F900203C
:1009F000824224D00133082B04F10C04F6D1002FDD
:100A00004CD0002D08BF03250023EDB2CDE90153E2
:100A100000971A46194627F073FA044600284AD070
:100A20002A483A463146F6F78FFB31462848F6F712
:100A30008BFB284B2146D3F8FC0155F0AFF803EBB4
:100A4000430301EB83035C68002CD8D02248314675
:100A5000F6F77AFB5DB16179A94208D01F482A46B2
:100A6000F6F772FB2368E9B29B6920469847E36A70
:100A7000002BDAD01A48F6F767FB0023E362D4E7CD
:100A80002046514661F021FB00289CD17EE71549A4
:100A9000204661F01AFB00288DD18EE712483146BE
:100AA000F6F752FB07B0BDE8F08F4FF0FF30254658
:100AB0002746064697E731460C48F6F745FBF1E72F
:100AC0000C1208085CC90708088E0020BCC807087B
:100AD0002CC9070810C80020DCC80708F4C807089C
:100AE00014C90708BCE7070874C807089CC80708AA
:100AF00068C807086CC8070870C80708F0B504463E
:100B000083B070B302785AB300F10040424D2146E1
:100B10000238722307E0974237D1884214D011F887
:100B2000012F15F8013FA2F1410EBEF1190FA3F1FB
:100B3000410C98BF2032BCF1190F03F12007EAD90C
:100B4000934222D1002BE8D1344B354AC3F8D02B45
:100B5000C3F8D42BC3F8D82BC3F8DC2B03B0F0BDFB
:100B60001446304D304E35F8241005EB84033246E0
:100B70005888CDE900100120234600210444FEF7E7
:100B8000D5FF042CEFD103B0F0BD2046F7F772F883
:100B9000032805462ED82046202161F027FA044676
:100BA000002837D003461C4613F8012B202AFAD020
:100BB0002046F7F75FF8012706462021204661F01E
:100BC00015FA034688B1184601330278202AFAD074
:100BD000F7F750F84FB1A6F2EE2240F2DC539A42FA
:100BE00003D8A0F2EE229A420CD9104803B0BDE817
:100BF000F04081E60E490F480323002203B0BDE810
:100C0000F04079E6054B03EB8505A5F8D06BA5F818
:100C1000D20BA3E70746D0E768C9070810C8002031
:100C2000E803D007E0D3002070C907085CC90708B3
:100C300084C907088CC907082DE9F04387B040B381
:100C4000037807462BB300F10040554E3946023871
:100C5000722207E09C4532D1814212D011F8013F47
:100C600016F8012FA3F14105192DA2F1410498BFF7
:100C70002033192C02F1200CECD99A421FD1002A02
:100C8000EAD148486022002107B0BDE8F04361F096
:100C900096B9444D444F0024D5E9010615F80C1BC4
:100CA0000091CDE90106012023463A460444002183
:100CB000FEF73CFF082CEFD107B0BDE8F0833846C3
:100CC000F6F7D8FFC3B2072B054646D82021384691
:100CD00061F08CF90446002854D003461C4613F8F2
:100CE000012B202AFAD02046F6F7C4FF071E18BFB2
:100CF000012701262046202161F078F904460028CA
:100D00004CD003461C4613F8012B202AFAD020466B
:100D1000F6F7B0FF01368046F6B22046202161F09A
:100D200065F9034688B39946013399F80020202AD3
:100D3000F9D04846F6F79EFF013604462021484682
:100D4000F6B261F053F908B10136F6B2032E0CD0B9
:100D5000164807B0BDE8F043CEE51549154807230E
:100D6000002207B0BDE8F043C6E5134B6DB205EBBA
:100D7000450503EB850383F8E07BC3F8E48BC3F8F8
:100D8000E84B99E706460746B4E72021059061F055
:100D90002DF9059B1C460028D6D1D9E78046BCE733
:100DA00068C90708F0D30020ACC907085CC9070868
:100DB000C4C907088CC9070810C80020002862D0E1
:100DC0002DE9F04F90F800C085B00446BCF1000F4B
:100DD00030D000F10047574E8646023F0146634639
:100DE000722207E098452CD18F4212D011F8013FB2
:100DF00016F8012FA3F14105192DA2F1410098BF6A
:100E00002033192802F12008ECD99A4219D1002A7E
:100E1000EAD1494B1B6813F0040308D1474AA2F8F2
:100E2000D03F82F8D23F82F8D73FA2F8D83F05B032
:100E3000BDE8F08F0021012005B0BDE8F04F54F06F
:100E400019BF3F4E214663466C2207E098451ED1EC
:100E5000B94212D011F8013F16F8012FA3F1410554
:100E6000192DA2F1410098BF2033192802F1200862
:100E7000ECD99A420BD1002AEAD1012005B0BDE895
:100E8000F04F4BF02DBD0021012054F0F3BE2D4852
:100E9000732307E065455BD1BE4513D01EF801CF33
:100EA00010F8013FACF141011929A3F1410298BFAB
:100EB0000CF1200C192A03F12005EBD9634547D129
:100EC000002BE9D11D4B002293F9D60F83F8D02FC8
:100ED0001C46164693F890140129A1F1030509D088
:100EE000052D07D90EB184F8D60F174805B0BDE817
:100EF000F04F01E593F8A614A52903F1180303D0D8
:100F00000132782AE6D1EDE7012803D0013840B25A
:100F10000126F5E70D4984F8D00F0023013284F84B
:100F2000D12F81F8403C84F8D63F05B0BDE8F04FA2
:100F30004BF082BD68C907081000001000B80020FF
:100F4000D4C9070870DF07085CC9070810C800206B
:100F5000DFF884A22046F6F78DFE9AF9407C07FA66
:100F600080F5772D064600F2D1802046202161F0E1
:100F70003DF88046002800F01D810346984613F88E
:100F8000012B202AFAD04046F6F774FE01245FFABE
:100F900080F94046202161F029F88046002800F0C1
:100FA0000E810346984613F8012B202AFAD04046BA
:100FB000F6F760FE01340090E4B24046202161F073
:100FC00015F88046002800F0F8800346984613F88C
:100FD000012B202AFAD04046F6F74CFE013401904E
:100FE000E4B24046202161F001F88046002800F07C
:100FF000C0800346984613F8012B202AFAD04046B9
:10100000F6F738FE01340290E4B24046202160F049
:10101000EDFF8046002800F0AA800346984613F8AA
:10102000012B202AFAD04046F6F724FE01340FFAAD
:1010300080FBE4B24046202160F0D8FF0246002841
:1010400000F0B68003461A4613F8011B2029FAD097
:1010500010460392F6F70EFE0134039A0FFA80F859
:10106000E4B21046202160F0C1FF002857D00346AB
:101070001A46013311782029FAD010460392F6F768
:10108000F9FD039A03461BB210462021039360F03A
:10109000ADFF039B002800F0948002461046013209
:1010A00001782029FAD00393F6F7E4FD04F0FD045B
:1010B000042C039B08BFC2B27FF417AFB9F1010F34
:1010C00004D9A9F1030105293FF60FAF22B1A52AE2
:1010D00030D0482A7FF409AF45B33C4905EB4505BC
:1010E00001EBC50181F890940098C1F8940401982F
:1010F000C1F898040298C1F89C04A1F8A0B4A1F822
:10110000A284A1F8A43481F8A62490E6304931489D
:101110007723002205B0BDE8F04FFFF7EDBB5FFA83
:1011200088F203468046062CC8D0DEE6274981F8BF
:10113000D65FD7E7FDB9254C0099C4F894140199FE
:10114000C4F898140299A4F8A43484F89094C4F8CC
:101150009C14A4F8A0B4A4F8A28484F8A6240123C3
:1011600001373E448AF8406C84F8D63F5FE68346F8
:1011700060E7029049E7154C009805EB450504EB44
:10118000C501A1F8A43494F8D63FC1F8940401989D
:10119000C1F898040133029881F89094C1F89C0436
:1011A000A1F8A0B4A1F8A28481F8A6245BB2D7E785
:1011B000804656E704468146EBE6019011E7009031
:1011C000FBE60134E4B20246ADE700BF00B8002000
:1011D000DCC907088CC9070810C800202DE9F04FAA
:1011E0008BB010B103780446BBB97B4E7B4F002413
:1011F00005AD56F8043F0493294604A854F07CFC3E
:1012000001202346009504443A460021FEF78EFC57
:10121000202CEED10BB0BDE8F08FF6F72BFD1F2888
:10122000064632DC2046202160F0E0FE044628B16C
:1012300003461C4601332278202AFAD0684BDFF897
:10124000B881002543F8265001272C200395AA4693
:101250000295A946AB46237807F1FF3C5FFA8CFC68
:10126000E3B105A9002205E001F8013B14F8013FB4
:101270000132A3B1984200F092800A2AF4D1594871
:101280000BB0BDE8F04FFFF737BB574957481F2356
:1012900000220BB0BDE8F04FFFF72EBB1A460AAB99
:1012A0001A4402F814BC0028E9D10CF1FF330134D0
:1012B000032B79D8DFE803F06547200205A8F6F78D
:1012C000D9FC0F2876DC800405F00F03029A43EA6C
:1012D0008953034343EA0223039A120143EA0A3380
:1012E000D2B21343424A02EB8606C6F8443C0BB026
:1012F000BDE8F04F39F056B99DF814200DF1140EE9
:10130000E2B13C480023432101E010F8011B8A426E
:101310003CD00133082BF8D1542A39D04F2A4DD074
:10132000422A4FD04E2A4FD0492A51D0572A08BFBF
:1013300005232ED01EF8012F002AE2D1013718F81C
:10134000010BFFB287E79DF8143005AA83B9F5E7D2
:10135000452B31D0532B33D0572B37D0552B39D089
:10136000442B08BF052306D012F8013F002BE5D01F
:101370004E2BEDD10023012101FA03F349EA0309C1
:10138000F2E705A8F6F776FC0546D7E70293C3E730
:101390000023012202FA03F34AEA030ACAE70AAB6E
:1013A0001A4402F814BC80E705A8F6F763FC052F81
:1013B0000390C3D1002087E70123DCE70123E8E79E
:1013C0006346D8E70223E4E76346E2E70323D2E774
:1013D0000423DEE70423CEE750D40020E8C9070841
:1013E00054D400205CC90708F4C907088CC9070851
:1013F00010C80020093C0708013C07082DE9F0410E
:1014000084B010B103780446CBB9384C384F00256E
:1014100094F8820094F88360B4F880100091CDE9CC
:10142000010601202B463A4605440021FEF77EFBCB
:10143000102D04F10404EBD104B0BDE8F081F6F7FF
:1014400019FC0F2805462CDC2046202160F0CEFD3B
:10145000044628B103461C4601332278202AFAD0DC
:10146000244B254F2035012603EB85082046F6F74F
:1014700001FC37F8021B8842034606F1FF3219DCF3
:10148000012A4FF02C01204626D0022A1CD0A8F8B1
:10149000443C60F0ABFD441C60B1032ECCD001365F
:1014A000E4E7164916480F23002204B0BDE8F041D6
:1014B000FFF722BA0D4B1348002243F8252004B051
:1014C000BDE8F041FFF718BA0A4A02EB850585F836
:1014D000473C04B0BDE8F08188F8463C60F086FDEA
:1014E0000028E7D0441C0136C0E700BF54D40020D8
:1014F000FCC9070810C80020103C0708F4C90708F9
:101500008CC907085CC9070870B508B103786BB9C6
:10151000174C18480023A4F8623AFEF703F916485E
:10152000FEF700F9B4F8626A76B970BDF6F7A2FB6F
:101530000146C0B10E4B1148A3F8621ABDE87040D5
:10154000FEF79CBB013EF0D0FDF7B8FF04460D4608
:10155000FDF7B4FF031B61EB0502B3F57A7F72F16F
:101560000003F5D3EEE7BDE870400548FFF7C4B9C6
:1015700010C8002028CA0708B8C8070810CA0708FA
:101580005CC907082DE9F04188B0002841D00378F4
:101590000446002B3DD000252D2B5CD0A3F130025A
:1015A000092A58D9202B50D163780134002BF3D16C
:1015B000052D4AD1BDF914309AB20F2A45D8BDF98C
:1015C0001610A1F5FA7292B2B2F5FA6F3DD8BDF9D4
:1015D0001800A0F5FA7292B2B2F5FA6F35D8BDF9DB
:1015E0001A40A14231DCA0422FDB81422DDCBDF943
:1015F0001C5005F17D0292B2FA2A26D8204A22F820
:10160000331002EBC30358809C809D7108B0BDE885
:10161000F0811B4CDFF870800025B4F9020094F9CA
:101620000670B4F9046034F9081BCDE900100120FC
:101630002B46CDE90267054442460021FEF776FAC3
:10164000102DEAD108B0BDE8F0810E4808B0BDE821
:10165000F041FFF751B9042DF7DC2046F6F70AFBFD
:1016600008AB03EB4503013523F80C0C14F8013FDC
:10167000A3F13002092AF9D9002B8DD198E700BFD8
:10168000448F00205CC9070840CA0708F0B58BB03A
:10169000074659F097FE10F0FF0432D03C4E07F198
:1016A000050C3946722205E098423FD1614512D0BF
:1016B00016F8012F11F8013BA3F14105192DA2F1F4
:1016C000410498BF2033192C02F12000ECD99A4232
:1016D0002CD1002AEAD12F482F4A904238BF40F23D
:1016E000FF3103D320E0143090421DD20388C3F3AE
:1016F0000B038B42F7D129490BB0BDE8F040F6F758
:1017000087BB264D264FA968D5E90006CDE901061D
:1017100001202346009104443A460021FEF706FAD0
:10172000082C05F10C05EED10BB0F0BD1D4905AA42
:10173000384660F0EAFB78B11A4E06AD0024F6F7A1
:1017400099FA05AA45F8040B31460020013460F0EF
:10175000DCFB30B1042CF2D11348FFF7CDF80BB00D
:10176000F0BD042CF8D1069B072BF5D80F4A104882
:10177000DDE9074103EB430302EB8303099AC3F856
:101780003C4DC3F8341DC3F8382DFFF77FFFCBE77E
:1017900068C907081C270808082C080844D5002039
:1017A00058CA07080C1208085CC9070810C80020AE
:1017B000B41908082DE9F04782B0404901AA60F049
:1017C000A4FB002875D04FF0000A4FF0FF343B4DCA
:1017D000D1465646D0462746BAF1040F09D8DFE86D
:1017E0000AF0453F390E03000378482B47D0562BAB
:1017F00042D03348FFF780F802B0BDE8F087F6F733
:1018000039FA3F280646F4D8002001AA294660F09C
:101810007CFB0AF1010A0028DED1BAF1040F3BD0AB
:1018200030DDBAF1050FE4D1264A3901B30103F4E2
:101830007C6308F03F0843EA0803B9F1000F01D0C8
:1018400043F40053394404EBC10402EB4404A4F80C
:10185000943DD1E7F6F70EFA3F288046D4D9C8E781
:10186000F6F708FA87280446CED9C2E7F6F702FA57
:1018700003280746C8D9BCE74FF00109C4E74FF079
:101880000009C1E7BAF1020FB3DC0F4923463A461B
:10189000012054F073FAAFE70A4A07EB071304EB91
:1018A000C30302EB43033901B3F8949DC9F34039F4
:1018B000BCE74FF0FF373C46E7E700BF0C120808D3
:1018C0005CC9070810C80020A4D500202DE9F0410C
:1018D00084B0044659F076FD042827D010BB324D61
:1018E0003248FDF71FFF6878A978EA782B7904ACB5
:1018F0002044234421442244412400F8084C452438
:1019000001F8084C5220542402F8080C02A90022C5
:1019100003F8084C26488DF80C20FEF7AFF904B008
:10192000BDE8F0812348FEF7E7FFD8E7621E2546B1
:10193000E01C12F8013FA3F1610119299CBF203B73
:10194000DBB290421370F4D11B4E271D15F8011B1A
:101950000191304660F04AFB03460199284613B1D5
:1019600060F044FB28B1134804B0BDE8F041FEF735
:10197000C3BFBD42EAD121780029B0D0DFF838805A
:10198000094D274608F10406404660F02FFB30B1B0
:10199000B042A0EB080302D22B443A1B5A7017F84E
:1019A000011F0029F0D19BE75C9400206CCA070856
:1019B00090DE07085CC90708183C0708002832D0E9
:1019C000037883B3F0B583B001AA284960F09DFA8B
:1019D000024600283CD00024244D264627462CB33E
:1019E000012C03D11046F6F745F9064601AA00205E
:1019F000294660F08AFA013402460028EFD10B2F05
:101A00001FD8022C17D1A6F57A73B3F57A7F24D8A4
:101A1000174B03EB470332B29A8016483946FEF75C
:101A20002DF903B0F0BD1448FEF766BF1046F6F777
:101A300021F90746DAE70E4B03EB4703B3F904201D
:101A4000EBE70E490E480B23FEF756FF03B0F0BD3F
:101A5000074B1746B3F90420DFE70A4908484FF45B
:101A6000FA634FF47A72FEF747FFDAE70C120808C0
:101A7000281000107CCA07085CC90708F4C90708C9
:101A80008CC9070874CA0708F8B53049052204460E
:101A900060F0C2FA18BB2E4E96F8603A23B90122C4
:101AA00086F8602A86F8613A2A48FDF73BFE2A4804
:101AB000FDF738FEB6F8626A16B9F8BD013EFCD0F3
:101AC000FDF7FCFC04460D46FDF7F8FC031B61EB3B
:101AD0000502B3F57A7F72F10003F5D3EEE71F49F3
:101AE0000322204660F098FA50BB194E96F8603AEF
:101AF00013B196F8613AFBB91948FDF713FE164881
:101B0000FDF710FEB6F8627A3FB9002386F8603A16
:101B100086F8613AF8BD013FF7D0FDF7CFFC0446E7
:101B20000D46FDF7CBFC031B61EB0502B3F57A7F95
:101B300072F10003F5D3EEE70A48FEF7DDFEE4E7B5
:101B4000BDE8F8400848FEF7D7BE00BF8CCA0708BA
:101B500010C8002094CA0708B8C8070888E007081A
:101B6000E4CA0708ACCA0708F8CA070870B5837941
:101B7000044603F00F008CB01546062800F2A28040
:101B8000DFE800F00A1333353841040053480CB045
:101B9000BDE87040FEF750B80E7813F0C00309D0CE
:101BA000402B00F084800CB070BD13F0C00391F99D
:101BB0000060F5D14A483146FEF73EF8002DF2D0DC
:101BC000A37913F0C00FEED1E179464B227A464853
:101BD00003EB820203EB8103D2F89022B3F9901257
:101BE0000CB0BDE87040FEF727B80E88D5E7B1F914
:101BF0000060D2E7096813F0C0030E4637D13B48B6
:101C0000FEF71AF8DAE791ED000A01A8F5F7E0FE11
